:10000000986E0020A5160000A1160000A1160000A1
:1000100000000000000000000000000000000000E0
:10002000000000000000000000000000A116000019
:100030000000000000000000A116000059010000AF
:10004000A1160000A1160000A1160000A1160000D4
:10005000A1160000A1160000A1160000A1160000C4
:10006000A1160000710D0000810D0000910D00002F
:10007000A10D0000B10D0000C10D0000A11600008F
:10008000A1160000A1160000A1160000A116000094
:10009000A1160000A1160000A1160000A116000084
:1000A000A1160000A1160000A1160000A116000074
:1000B0000000000010B5064C2378002B07D1054B3B
:1000C000002B02D0044800E000BF0123237010BDC4
:1000D000D80000200000000060B10200084B10B5FD
:1000E000002B03D00749084800E000BF0748036819
:1000F000002B00D110BD064B002BFBD09847F9E731
:1001000000000000DC00002060B1020060B10200CD
:100110000000000010B5402200210A480A4B984711
:100120000A4A002010600A4B53600A4C236A1B02E3
:100130001B0AC02109060B4323629060072313604A
:1001400010BDC046B04C002071C6010010E000E0B8
:100150003F1F000000ED00E070B506490A684B68DB
:100160000124002512196B410A604B600120024BEB
:10017000984770BDF8000020DD0E0100F0B5DE46A6
:100180004F464646C0B586B0214B1E685F6818686A
:100190005968204B9B46FA2292000023D84704005E
:1001A000402200211C481D4B98471D4B99461D4974
:1001B00005942000984708001B4DE1210901A8473C
:1001C000FF2420408046FA229200002330003900AC
:1001D000D84792B202923C21059E3000C847214088
:1001E0000191E12109013000C84708003C21A847DE
:1001F0000440009443460D4A402107480C4CA04758
:10020000054806B01CBC90469946A346F0BDC046C2
:10021000F800002091C30100B04C002071C601001D
:10022000B1C1010080510100A5C001004CCF010007
:1002300081C6010030B58DB0224B98470122224B78
:100240001A70BFF35F8F62B6204B9847204B9847D8
:10025000204B9847204B9847204B9847204B984776
:10026000204C96235B0100221F4920001F4DA84708
:1002700001A81F4B98471F4B0493029401A81E4BE3
:10028000984700201D4B9847040000211C4B9847BD
:1002900005001C491C4B98470022002128001B4DDB
:1002A000A847002120001A4B9847040023225A2116
:1002B000A84718492000184B9847184B98470DB08D
:1002C00030BDC046751600000C00002035BF01008F
:1002D000C5BE0100FDBD010015010000651D000047
:1002E00051AF01008026002000010020010C010018
:1002F0009D0B0100DDBA0100210C01004518000032
:100300005D95010064CF0100C992010079290000C8
:10031000C5A80100CC5402009DA5010079C00100D0
:1003200010B50020084B9847020000230748002121
:1003300080185941064A0023064CA047064B9847AF
:10034000064B984710BDC046FD130000571B000028
:10035000581B000091C3010001000020A1360100DC
:10036000F0B5DE4657464E464546E0B587B0804676
:10037000049116001F000022002300218B463F2419
:1003800001202100009601975C46039444460594A1
:1003900013E02024641A0500E540A84614E0009C00
:1003A000019D121BAB415C464D462C43A346039C6A
:1003B00045462C430394013925D3202464420C196B
:1003C000E7D40500A540A84604008C40A146921839
:1003D0005B4114001D00059E4F463E40B446049EFE
:1003E00047463E40B246664657463E4303D0060067
:1003F000264332002B00009C019D9D42DBD8CED1CC
:100400009442D8D8CBE7039B5846190007B03CBCB0
:1004100090469946A246AB46F0BD10B54908402328
:100420000024814202D2180010BD1C00091A631C6E
:100430009BB28842F9D94023FF2CF4D814800023C2
:10044000F1E70000F0B583B00F00160008AA11789C
:1004500004004C434022BC4202D9100003B0F0BD5E
:10046000002B14D1020008000021194CA047010004
:100470003A0000230020174CA04700220123121A43
:100480008B41120C1B041A4332800022E5E7002244
:10049000012BF9D10A00002300210D4CA0470200D6
:1004A0000B0000920193380000210A4CA047050080
:1004B00080239B0140229842CFD8790FF800009A00
:1004C000019BA047EA00821AD2B252032A43DBE71B
:1004D000D1C301006103000010B582B004000E4BCF
:1004E0001B78002B07D0002905D10B4B5B7883428A
:1004F00010D01D200CE001A90C701320074B984769
:100500001320074B9847044B5C7001221A7000209F
:1005100002B010BD0020FBE7A42600201515000046
:1005200089140000404B984231D00AD93F4B984281
:100530004DD03F4B98425AD03E4B984237D0002086
:1005400070473D4B98420CD03C4B9842F7D1012963
:1005500017D000295DD0022915D0032915D000201D
:10056000EEE7012907D0002951D0022905D003293F
:1005700005D00020E4E73248E2E73248E0E73248BD
:10058000DEE73248DCE73248DAE73248D8E70129CB
:1005900007D000293FD0022905D0032905D000202B
:1005A000CEE72D48CCE72D48CAE72D48C8E70129FA
:1005B00007D0002931D0022905D0032905D0002019
:1005C000BEE72848BCE72848BAE72848B8E7012929
:1005D00007D0002923D0022905D0032905D0002007
:1005E000AEE72348ACE72348AAE72348A8E7012958
:1005F00007D0002915D0022905D0032905D00020F5
:100600009EE71E489CE71E489AE71E4898E71E484A
:1006100096E7032094E71D4892E71D4890E71D48A0
:100620008EE71D488CE7C0460010004200180042CB
:10063000001C00420014004200080042000C00426E
:10064000030005000300060003000700030001008B
:1006500003001E0003001F000300090003000A003E
:1006600003000B000300110003001200030013003D
:1006700003000D0003000E0003000F00030017002D
:100680000300180003001900030004000300080021
:100690000300100003000C000300160030B587B003
:1006A0000B4B6A4632CB32C232CB32C2009B834202
:1006B0000BD001239A0069465258824206D001337A
:1006C000062BF7D1002007B030BD0023D8B2FAE7DF
:1006D000D8540200F0B5DE4657464E464546E0B5D2
:1006E00091B005000C00160029600800BA4B98472D
:1006F000020023680520DB0706D511B03CBC9046FC
:100700009946A246AB46F0BD236817309B07F4D448
:10071000B249086A971C0123BB4003430B620FA92F
:100720002D27F35D0B701432D3B202931800AC4B3B
:1007300098470298AB4B9847F05D0021AA4B984729
:10074000F37A6B712423F35CAB712523F35CEB71BB
:10075000F37E2B72337F6B722B68984618009E4B8A
:100760009847143000220E2306A98C4663441A8051
:10077000328A02928023DB019A4200D19AE00FD99B
:10078000C023DB01029A9A4200D18EE080231B0233
:100790009A4200D01BE1032306930023079308E04D
:1007A00080239B019A4200D011E1102306930F3B56
:1007B000079333680593F3689B4673690393337E0D
:1007C00004932623F35C9A4673689946002B00D164
:1007D0009CE080235B05994500D180E0737E002B6F
:1007E00002D0B37E424693730E2306AA9446634416
:1007F0001B8842469381059B5A461343039A134331
:100800004A461343029F1F43049B1B021F43534648
:100810005B071F432723F35C002B01D104331F43E5
:10082000737E9B02327F52021343727F1202134384
:100830002422B25C520413432522B25C12041343F7
:10084000B17AF27A114319433389FF2B00D181E049
:1008500080225204174319432C23F35C002B03D14D
:10086000624B9B789B0701D580231F432A68D3697D
:10087000002BFCD1434659602A68D369002BFCD178
:1008800043461F600EAB80221A7000225A70DA7045
:100890009A70336B0A93736B0B93B36B0C93F36B7C
:1008A00002930D9300270AAE63E008230693073BEB
:1008B00007937EE733680593F3689B467369039358
:1008C000337E04932623F35C9A4673689946002B83
:1008D00018D080235B05994501D0002025E027230F
:1008E000F35C002B00D079E7336A1F00C0B2404BA5
:1008F000984701000E2206AB9C46624438003D4BEF
:10090000984712E008230693002307932723F35CFC
:10091000002B0ED0069B0093079B0E2206A98C4647
:100920006244B16A306A344FB847002800D0E4E628
:1009300054E7336A1F00C0B22D4B98470100069B55
:100940000093079B0E2206A88446624438002A4F73
:10095000B847EAE7F37E002B00D17DE78023DB0474
:100960001F4379E72000254B984707E00137042F04
:100970000DD0F9B2BB0098590028F3D0431CF5D034
:100980000EA90870000CC0B21D4B9847EEE700237B
:10099000EB602B616B61AB61EB612B62AB626B62F5
:1009A0000022EB85AB853033EA540133EA5401333E
:1009B000EA540133EA542868074B98470400114968
:1009C000114B9847A400114BE550002095E61023E9
:1009D000069300230793ECE69D0600000004004008
:1009E0001515000089140000D90400000020004102
:1009F000311500001B04000045040000250500001F
:100A00000D1600006D0B0000050D0000F04C0020DD
:100A1000C2791C23002A01D118007047C28D92B2FE
:100A2000173B002AF8D1026811850221137E0B4280
:100A3000FCD00023F0E70000F0B5CE46474680B575
:100A400083B0050001911720002A04D103B00CBC2B
:100A500090469946F0BDEB790530002BF6D02C6816
:100A6000013A93B2994600260127204B984611E09F
:100A7000731C9BB2019A915D6A79012A17D089B2E1
:100A80001E0028001A4B98474B46013B9BB29946E3
:100A9000434513D0237E3B42EAD1144B227E3A4297
:100AA000E6D1012B19D0013B002BF7D1E0E702364C
:100AB000B6B2019AD35C1B021943E2E7237E9B077F
:100AC0000DD40A4B0221227E0A420AD1012B0AD000
:100AD000013B002BF7D10020B8E71220B6E7002039
:100AE000B4E70020B2E71220B0E7C046FFFF0000E5
:100AF000110A0000F8B504000D00160007680F4B3E
:100B00009847A38D9BB2002B03D00D4B984705202F
:100B1000F8BDA6850A4B9847656205223223E25448
:100B20002E3BBB75237A002B01D02023BB75637A43
:100B30000020002BECD00823BB75E9E7D10D0000A5
:100B4000110E0000931C9B00C31859603021012333
:100B500093401A00435C13434354704710B501227D
:100B6000014B984710BDC046F50A0000F8B580005B
:100B7000624BC5582C68E369002BFCD1237EA67D0F
:100B80001E403023EB5C3122AF5C1F40F30722D5BF
:100B9000EB8D9BB2002B1CD0AA6A1378DBB2511CE0
:100BA000A962697901290ED09BB2DB05DB0D238593
:100BB000EB8D013B9BB2EB85002B0CD101332375F0
:100BC0000133A37507E0517809020B430232AA6290
:100BD000EBE701232375B30706D502232375002213
:100BE0003133EA54FB071AD4730765D5AB8D9BB23A
:100BF000002B5FD0638BDBB21A0714D43F22134063
:100C0000002B34D09A0711D51A223223EA54303BF4
:100C100063837B0750D528006B6998474CE0280018
:100C2000EB689847E0E737221340E9E75A0705D514
:100C30001E223223EA542E3B6383EAE7DA0705D506
:100C400013223223EA54313B6383E2E7DA0605D507
:100C500042223223EA54223B6383DAE720221A42FB
:100C6000D7D021323223EA54123B6383D1E7238D5C
:100C7000DB05DB0DDAB2696A0A706A6A511C6962C7
:100C80006979012910D0AB8D013B9BB2AB85002B5C
:100C900012D10433237500222E33EA54BB070BD53F
:100CA00028002B69984707E01B0A53706B6A0133D1
:100CB0006B62E8E704232375F30604D5102323753C
:100CC0002376FB060ED4B30604D5202323752376A2
:100CD0003B070BD4330704D5082323752376BB06C3
:100CE00008D4F8BD2800EB699847ECE72800AB6909
:100CF0009847EFE72B6A28009847F2E7F04C00206E
:100D000070470000F0B50A4B1B78002B0CD1094F3F
:100D1000094E0A4D0024DE515A1914600433182B71
:100D2000F9D10122024B1A708000024BC150F0BD74
:100D3000A6260020A8260020010D0000F04C00206F
:100D400000B583B009236A46137001335370013331
:100D500093700133D3700133137101335371034B1B
:100D600098476B46185603B000BDC0469D0600006C
:100D700010B5024B1B680020984710BDA826002024
:100D800010B5024B5B680120984710BDA8260020D3
:100D900010B5024B9B680220984710BDA826002082
:100DA00010B5024BDB680320984710BDA826002031
:100DB00010B5024B1B690420984710BDA8260020DF
:100DC00010B5024B5B690520984710BDA82600208E
:100DD0000C4B1B68002B06D1EFF31083002B07D0C0
:100DE0000022094B1A70074A1368013313607047D9
:100DF00072B6BFF35F8F0022044B1A700132024BB0
:100E00001A70F0E7C0260020C42600200C00002045
:100E1000084B1A68013A1A601B68002B09D1064B6F
:100E20001B78002B05D00122044B1A70BFF35F8F93
:100E300062B67047C0260020C42600200C000020A7
:100E4000F0B583B001AC012565700027A77025704F
:100E500021003E20064EB0478022D205054B9A6104
:100E60002770657021000F20B04703B0F0BDC04669
:100E7000790E00008044004100B583B001AB8022B0
:100E80001A700A785A704A789A708A78DA7019005B
:100E9000014B984703B000BD0D16000010B582B09D
:100EA00001AB80241C7014785C7054789C7092782C
:100EB000DA701A00014B984702B010BD3D160000D1
:100EC00010B5082803D880001C4B1B589F460020F3
:100ED00032E01B4B18692FE01A4B1B6A9B059B0FD6
:100EE0001948D84028E0164B586925E0144B1B6878
:100EF00000209B0720D513491022CB681A42FCD052
:100F00000F4B1A6824231340042B01D00F4813E021
:100F100000200F4B98470A4B9B681B041B0C58433F
:100F20000AE05023074AD35C00205B0704D5044B3A
:100F3000D86801E08020000210BDC046F0540200D5
:100F4000C82600200008004000127A00006CDC0275
:100F50003115000070B50C490B6A0478857840782B
:100F60000122104080014026B34303432A40D201AE
:100F7000802083431343032222401202034803408C
:100F800013430B6270BDC04600080040FFFCFFFF2A
:100F9000F0B5DE4657464E464546E0B50100264BC5
:100FA0009B469B8A45780078424242419146887828
:100FB000CA7894460A7990464E7B0F7B8C7B8A6870
:100FC0001E494A6101214A469200914604229343F8
:100FD0004A46134342460A40D200904608229343B1
:100FE0004246134362460A4012019446102293433C
:100FF00062461343084040012022934303430F40BD
:10100000BF01402083433B430E40F6014030834301
:101010003343793805402D02094803402B432140D2
:101020000903084803400B435A4693823CBC904650
:101030009946A246AB46F0BD00080040C8260020F5
:10104000FFF8FFFFFFEFFFFF10B5037A9B061B0CB5
:1010500042899205920D134318494B608379C279F6
:10106000134342888488224313434278D2011343B6
:101070000B600378042B11D0202B0ED1037B9B0631
:10108000028A1343C28912040D490A4013430B4AD2
:10109000936011680B4B0B43136010BD037B9B06E1
:1010A000028A1343C289120405490A401343034AC2
:1010B0009360136804210B431360EEE7C8260020F9
:1010C0000000FF0324040000082803D88000254BFB
:1010D0001B589F46172044E0234A136A02210B4302
:1010E000136200203DE0204A936902210B43936183
:1010F000002036E01C4A138A02210B431382002091
:101100002FE0194A938A02210B439382002028E0A2
:1011100016490B68022213430B60134B9A84190083
:101120000E32CB681A42FCD0104A91680E4BD9623D
:1011300052689A6200229A8419001032CB681A42CF
:10114000FCD00A4B1B689BB2074A9384002008E03E
:10115000054944228B5C022003438B54002000E0AD
:10116000002070471455020000080040C8260020E7
:10117000F0B58FB0C222D2004A4B9A604A4A5368F7
:101180001E218B431A390B435360022201AB1A70A4
:101190000024464DE0B201A9A8470134252CF9D11D
:1011A0000AA800230370802212028260C370012209
:1011B00002718373032141708270437302733C4B4D
:1011C000984705203B4B984736490222CB681A4284
:1011D000FCD0344A938A80210B43938205AB0021D3
:1011E0000022598099809A71DA713F3159813B39D7
:1011F00019705A70304B1B689B0E3F2B4FD005A8BF
:1012000003722E4B0382072303733833C3812C4BA5
:10121000984704A80025457005708570294B9847AC
:101220000620244FB847284B984701AC0126029668
:101230006570657205232370267221000120234BFF
:1012400098470120224B9847267021000020174B19
:10125000984700201F4B98470720B8471149D022D4
:10126000CB681340D02BFBD10E4A938C80210B43CB
:101270009384194A0023137253729372D37201A993
:1012800001224A604B700B724B7207330B700020C7
:101290000E4B984700200E4B98470FB0F0BD203BF7
:1012A000ADE7C046000800400040004115150000B1
:1012B000910F0000C910000024608000B9050000F3
:1012C00049100000550F0000DD120000011300005E
:1012D000B91300008914000000040040064A936915
:1012E00008210B4393610122044B1A7019000B78FB
:1012F0001342FCD17047C04600040040000C00407F
:1013000070B5060004000D782D0205434B78002BC4
:1013100002D08023DB021D434B7A002B02D08023B6
:101320001B031D434868012810D9431E184234D1BD
:10133000022830D90223002201325B009842FBD8F8
:1013400012023243140080235B031D430B7A002BEF
:1013500002D080239B031D43134A53785BB2002BBA
:10136000FBDB124B9847124B1E700F4A53785BB24F
:10137000002BFBDB0C4B9C601A0053785BB2002BFC
:10138000FBDB094A5368802149020B401D4355602D
:10139000084B984770BD0022D2E7040234438023F3
:1013A0009B021D43D2E7C046000C0040D10D000057
:1013B000080C0040110E000010B504000B4A5378D1
:1013C0005BB2002BFBDB0A4B98470A4B1C70074AA9
:1013D00053785BB2002BFBDB044A516880235B022D
:1013E0000B435360044B984710BDC046000C0040AF
:1013F000D10D0000040C0040110E000070B5040077
:101400001A4A53785BB2002BFBDB194B9847194BF8
:101410001C70164A53785BB2002BFBDB134E7068CE
:10142000C004C00E144B98470500124B1C70766820
:10143000F602F60F114B1C700C4A53785BB2002B6E
:10144000FBDB0A4B9C682402240C0D4B9847002EB2
:1014500007D1012C07D9210028000A4B9847050025
:1014600001E00134E540280070BDC046000C00409A
:10147000D10D0000040C0040C10E0000080C00401B
:10148000110E0000A5C0010010B50400064B9847DE
:10149000064B1C70064A53888021C9010B435380B8
:1014A000044B984710BDC046D10D0000020C00400F
:1014B000000C0040110E000010B504000F4B9847BF
:1014C0000F4B1C700F4A53881B05180F53880E4989
:1014D0000B40538053880D490B40538011008022EC
:1014E000D2014B881342FCD106494A8803020648C0
:1014F000024013434B80064B984710BDD10D0000AE
:10150000020C0040000C0040FFF0FFFFFFBFFFFF98
:10151000110E000010B50C7824020443024B9847CA
:10152000A4B2024B5C8010BDB9140000000C004056
:1015300010B50400064B9847064B1C70064B5C88A0
:101540002405240F054B98472000054B984710BDF4
:10155000D10D0000020C0040000C0040110E0000F4
:10156000FD13000030B5D378002B35D11378802BD4
:1015700029D01B0680246402234354780225AC43FF
:1015800006D19478002C20D18024A402234341600A
:101590005478013C012C1CD90D042D0CA024E40529
:1015A0002C431C4384620D0CD02424062C431C4382
:1015B0008462D478002C22D15B031CD59378012B54
:1015C0001ED0416117E00023D7E7C024E402234383
:1015D000DDE70D4C2340DFE741600C04240CA02321
:1015E000DB05234383620C0CD0231B062343836259
:1015F000D378002B03D15378013B012B02D930BDA6
:101600008161F8E78160FAE7FFFFFBFF10B50A0090
:10161000C1090023002904D14309DB0105498C4697
:1016200063441F242040012181401800024B984749
:1016300010BDC0460044004165150000F0B583B000
:1016400000900E00019200240127084D02E00134B1
:10165000202C09D03300E3401F42F8D0019A390012
:10166000A1400098A847F2E703B0F0BD651500005F
:101670007047000010B5054B9847054B9847054B40
:101680009847054B9847054B984710BD71110000CE
:10169000410E000071160000711600007116000066
:1016A000FEE70000F8B52A4A2A4B9A4211D01A00E8
:1016B000294B9A420DD2294A03339B1A9B080133C6
:1016C0009B000022234822498C58845004329A42BD
:1016D000FAD1234A234B9A420AD2D34321495B18B9
:1016E00003218B4304339B18002102C29342FCD197
:1016F0001D4AFF211D4B8B439360FD3990235B00F6
:101700001B4AD1501B4AD3780325AB430224234301
:10171000D370D3780C27BB4308263343D370164BC2
:10172000987B30229043202210439873997BB943D1
:10173000314399739A7BAA4322439A730F4A5368A1
:1017400080210B4353600E4B98470E4B9847FEE7A2
:1017500060B1020000000020D4000020040000203E
:10176000D8000020944E002000ED00E000000000B2
:10177000007000410050004100480041004000411D
:10178000F9C5010091C001000300064A1268002A51
:1017900004D0044A1068C318136070470249014A14
:1017A0001160F6E7E0260020986E0020431E984165
:1017B000C0B2704770B5C2B0040015001B4B98470B
:1017C0000600E52829D80200210002A8184B9847F6
:1017D00002AB9819202303700833437008338370D9
:1017E0004833C370041D5C3B124E0F222900D940C0
:1017F0001140715C21700134043B191DF6D12D3369
:1018000003730023437302AB00930B4BBC220B49C1
:1018100003200B4CA04742B070BD0094064BBF2282
:1018200006490320064CA047F5E7C04609C701005A
:10183000452501004C550200385502006055020054
:101840005921010010B582B0002802D0C06B02B04F
:1018500010BD074B98470028F8D1064B0093064B64
:101860002E2206490230064CA0470020EFE7C04672
:10187000750D010060570200705602002C570200DF
:101880005921010010B582B0002802D0006C02B0CE
:1018900010BD074B98470028F8D1064B0093064B24
:1018A0004B2206490230064CA0470020EFE7C04615
:1018B000750D0100F0560200845602002C570200FC
:1018C0005921010010B582B0002802D0406C02B04E
:1018D00010BD074B98470028F8D1064B0093064BE4
:1018E0005C2206490230064CA0470020EFE7C046C4
:1018F000750D0100B45602009C5602002C570200E0
:1019000059210100F8B5002811D0002534272026E0
:10191000074C02E0A047002804D0C35D1E42F9D066
:101920000500F7E7002D02D02800024B9847F8BDCC
:10193000A5210000ED280000F8B5DE4657464E46CA
:101940004546E0B506008A469046037DDB073CD459
:10195000C468012399460025324F0F339B4615E09A
:10196000337D5A461A4201D1002D2ED14B46002B11
:101970002BD03000D0470400002D4CD000239946D6
:10198000002C03D02068B84700280CD0002CE7D0EA
:10199000002D06D021003000C0470400A842EFD13E
:1019A00013E02500F6E7F368A3420ED0002B16D013
:1019B0001868C369002217219847F3681868002245
:1019C0000E21194B9847012805D03CBC90469946FA
:1019D000A246AB46F8BDF3681868144B9847F4600C
:1019E0002068C369002216219847F368186800220E
:1019F0000D210D4B98470128E7D1F36818680C4B6F
:101A00009847F3681868094B98473369002BDCD076
:101A100030009847D9E70028D7D005000023994621
:101A2000B0E7C04601270000DD1F00006928000064
:101A30000519000010B518210148024B984710BD48
:101A4000744E0020D11D010010B5024A0249034B1B
:101A5000984710BD9D1E0100851E01003919000028
:101A600010B5024A0249034B984710BDC51E01003C
:101A7000911E01003919000070B50400037DDD06D8
:101A8000ED0F1022134303751B0708D5054B98472C
:101A90002D01237D102293432B43237570BD024BF0
:101AA0009847F5E7611A0000491A0000F0B583B0C5
:101AB00005000C00002818D00600274B9847002886
:101AC00015D003689C4208D0244F01003000B8476D
:101AD00000280CD00368A342F7D1214B0093214B7F
:101AE000752221490120214CA04703B0F0BDA36B12
:101AF000002B0FD020001E4B984700280AD0A06B67
:101B00001C4B98471C4B0093164B7F221649012013
:101B1000164EB047A5632800184B98470600184B8F
:101B2000984700280BD0002EDFD0346028000A4BE5
:101B300098478642D9D128000E4B9847D5E7094BE4
:101B40000093852208490330084CA0473200002347
:101B50000C480D498847FEE7851E01009D1E0100C7
:101B6000B05702009C570200205802005921010082
:101B70003D460000791A0000EC570200351E0100B6
:101B8000AD17000054580200B5170000F0B583B03F
:101B90000500866B002E20D0F368002B1DD01B683B
:101BA00098421CD0019630001E4B9847041E14D05A
:101BB00003689D4208D01C4F21000198B847041EBD
:101BC0000BD023689D42F7D121003000174B984776
:101BD0002000174B98470023AB6303B0F0BD337D63
:101BE000DB0703D5337D01229343337530000D4B62
:101BF0009847F368984209D030000E4B9847F36835
:101C00001B689D42CED10023F360CBE730000A4B26
:101C10009847F3689842EFD10068C3690022172102
:101C20009847ECE7851E01009D1E01006D1F010015
:101C3000C9230100791A0000911E0100002804D078
:101C4000C368002B03D0186870470020FCE7002011
:101C5000FAE7002803D0007D8007C00F70470020FE
:101C6000FCE70000014B18687047C046E4260020DE
:101C7000F8B50C00002815D05022835C02210B43DC
:101C80008354184B1B68984205D0002C07D0C36BB7
:101C90009C4204D0F8BD0022134B1A60F5E70023E4
:101CA000C363F7E70020114B98470028F2D00D4F8F
:101CB0000D4D0E4E07E000232B600CE00023C363A4
:101CC000B0470028E6D05022835C02210B438354A6
:101CD0003B688342EFD0002CF0D0C36B9C42EFD125
:101CE000ECE7C046E4260020E8260020B90E0100FB
:101CF00010B500210020014B984710BD711C000059
:101D0000014B18687047C046E8260020F0B585B042
:101D10000D00029116000392031D019318000F4B52
:101D20009847041E18D0ADB2B7B20D4E238AEB18F7
:101D30002382638AFB186382A38AEB18A382E38A57
:101D4000FB18E382039A02992000FFF7DFFF2100CE
:101D50000198B047041EE9D105B0F0BD851E010011
:101D60009D1E010030B585B0214B1B78002B36D16C
:101D7000204B9847204B9847204B9847204B98473B
:101D8000204B984710212048204CA047204B02931D
:101D90000193009302221F211E4800881E4DA84770
:101DA0001E4B98471E4B9847B82149001D48A04735
:101DB00060211D48A0471D4B98471D4B98470120A7
:101DC0001C4B984701220A4B1A701B4B00931B4B6C
:101DD000A1321B4901201B4CA04705B030BD1A4B56
:101DE0000093164B782216490220164CA047F4E7C0
:101DF000F4260020B5220100A5340100451B010096
:101E000065110100351A0000C44D0020D11D0100EC
:101E100030000020625802000D690100CD40010031
:101E20007D540000204D0020144D0020F11C0000C6
:101E3000EDFD00009DF10000745C0200BC58020042
:101E40002C5C0200592101005C5C020030B583B0BB
:101E500004000D000C4B9847002808D03422ED01F7
:101E6000A15C7F230B402B43A35403B030BD074B31
:101E70000093074A07490330074DA8472200002373
:101E8000064807498847FEE7AD170000DC59020005
:101E9000940500002C5C020059210100205D020025
:101EA000B517000030B583B004000D000D4B984706
:101EB000002809D0342201231D40A35C0120834364
:101EC0002B43A35403B030BD074B0093B422D20080
:101ED00006490330064DA84722000023054806495D
:101EE0008847FEE7AD170000F45902002C5C0200A1
:101EF00059210100205D0200B5170000F0B589B03E
:101F000007000C0003921E00002904D00800294B92
:101F1000984700283CD005AB059400221A7107921F
:101F2000254B1B68002B00D0079305AA224B1A6093
:101F3000224B1D681E60224B9847002804D08368FE
:101F4000002B01D003999847002F02D0039920005D
:101F5000B8471A4B1D60184B1A6892681A6005AB97
:101F60001B790020002B11D1002C1FD03433E35CEF
:101F700001305B060AD52068002819D03200039989
:101F8000104B9847013842424241D0B209B0F0BDEF
:101F90000D4B0093DB22D2000C4903300C4DA847B7
:101FA000220000230B480C498847FEE70120EDE79B
:101FB0000120EBE7AD170000F0260020EC26002002
:101FC000651C0000DD1F0000545A02002C5C02005A
:101FD00059210100205D0200B517000070B582B0E4
:101FE00004000D001600002818D00D4B984700285B
:101FF0000CD10C4B00930C4A0C4903300C4DA847F4
:10200000220000230B480C498847FEE7A0693300F3
:102010002A002100094CA04702B070BD0120FBE757
:10202000AD170000445A0200C40600002C5C0200F8
:1020300059210100205D0200B5170000FD1E0000BF
:1020400030B583B004000D00094B9847002802D03A
:10205000E56103B030BD074B0093074A07490330E1
:10206000074DA84722000023064807498847FEE796
:10207000AD170000685A02001B0700002C5C02002C
:1020800059210100205D0200B517000010B500289D
:1020900004D0C369002B03D0984710BD0120FCE792
:1020A0000120FAE730B583B004000D00094B9847D2
:1020B000002802D0256203B030BD074B0093074AC9
:1020C00007490330074DA847220000230648074967
:1020D0008847FEE7AD170000805A0200370700006E
:1020E0002C5C020059210100205D0200B5170000A0
:1020F00030B583B004000D000C4B984700280CD17C
:102100000B4B00930B4A0C4903300C4DA84722009F
:1021100000230B480B498847FEE72900606A0A4BF9
:102120009847002800D0606203B030BDAD170000B2
:10213000985A0200490700002C5C02005921010056
:10214000205D0200B5170000FD26010030B583B008
:1021500004000D4B984700280CD10C4B00930C4AFF
:102160000C4903300C4DA847220000230B480C49B2
:102170008847FEE700236386E369002206212000EA
:10218000984703B030BDC046AD170000B45A0200F6
:10219000590700002C5C020059210100205D02005B
:1021A000B517000030B583B004000A4B98470028EB
:1021B00002D0206803B030BD074B0093074A08499E
:1021C0000330084DA84722000023074807498847E5
:1021D000FEE7C046AD170000F45A02009F0700005A
:1021E0002C5C020059210100205D0200B51700009F
:1021F00030B583B004000D4B9847002801D00C4D3A
:102200000DE00C4B00930C4A0C4903300C4DA847D1
:10221000220000230B480C498847FEE704002000F9
:10222000A8470028FAD1200003B030BDAD17000048
:10223000A5210000D05A02006B0700002C5C0200B0
:1022400059210100205D0200B5170000F0B5C64617
:1022500000B582B00400234B984700280FD02368B4
:10226000002B03D02000204B984704001F48204B30
:102270009847071E2AD01E4B98461E4E12E01E4B52
:1022800000931E4A1E4903301E4DA847220000231A
:102290001D481E498847FEE739001448154B9847EA
:1022A000071E13D03D0030352800C0470028F3D06A
:1022B000844206D001002800B0470028ECD08442B8
:1022C000F8D1380002B004BC9046F0BD104B00932A
:1022D000094BF222D2000A4902200A4CA0470027EB
:1022E000EFE7C046AD170000F1210000204D0020AF
:1022F000851E01009D1E0100E45A02007F070000B8
:102300002C5C020059210100205D0200B51700007D
:10231000305D020030B583B004000D000E4B9847CD
:10232000002807D0002D12D0201D29000B4B984704
:1023300003B030BD0A4B00930A4A0B4903300B4DE2
:10234000A847220000230A480A498847FEE7201DC3
:10235000094B9847ECE7C046AD1700009D1E0100F1
:10236000085B0200AD0700002C5C0200592101004F
:10237000205D0200B5170000851E010030B583B056
:1023800004000D000D4B984700280AD0200018309B
:1023900010342178297001350134A042F9D103B0FD
:1023A00030BD074B0093074A07490330074DA84744
:1023B00022000023064807498847FEE7AD170000C2
:1023C0001C5B0200010800002C5C02005921010086
:1023D000205D0200B517000030B583B004000F4B3C
:1023E000984700280CD10E4B00930E4A0E4903303B
:1023F0000E4DA847220000230D480E498847FEE7EE
:1024000020000D4B9847002805D0238A008A181A0F
:1024100000B203B030BD1023E05EFAE7AD17000054
:10242000305B0200220800002C5C020059210100F0
:10243000205D0200B5170000A521000030B583B073
:1024400004000F4B984700280CD10E4B00930E4A06
:102450000E4903300E4DA847220000230D480E49B7
:102460008847FEE720000D4B9847002805D0638A77
:10247000408A181A00B203B030BD1223E05EFAE7BA
:10248000AD170000405B0200360800002C5C020023
:1024900059210100205D0200B5170000A5210000B0
:1024A00030B583B004000C4B9847002806D0A08AB2
:1024B0000130238AC01A00B203B030BD074B00932D
:1024C000074A08490330084DA8472200002307485F
:1024D00007498847FEE7C046AD170000505B020081
:1024E0004A0800002C5C020059210100205D020016
:1024F000B517000030B583B004000C4B9847002896
:1025000006D0E08A0130638AC01A00B203B030BD41
:10251000074B0093074A08490330084DA84722009B
:102520000023074807498847FEE7C046AD1700006B
:10253000645B0200560800002C5C02005921010077
:10254000205D0200B517000000B583B0002902D15C
:10255000283003B000BD6B461970002301936A4612
:102560000821044B9847012801D10198F1E7002088
:10257000EFE7C0468D200000F0B5DE4657464646E0
:10258000C0B580468A4693461E001D481D4B98479D
:10259000041E2FD0B0422DD01B4F0AE0A3885B450C
:1025A00015D05B46FF2B12D0002D23D02C00AE425D
:1025B00020D021001248B847050020684045F3D1DB
:1025C000A1795145EAD05346FF2BEDD1E6E70F4BF9
:1025D00098470F4B9847A1880E4B98470021200041
:1025E0000D4B9847210006480C4B984720000C4B98
:1025F0009847D9E71CBC90469A46A346F0BDC04612
:10260000C44D0020911E0100C51E01004925000097
:1026100065690000895E0000FD1101006D1F010069
:10262000C923010030B583B004000D000B4B98475F
:10263000002809D00A4B98470023FF2229002000D8
:10264000084CA04703B030BD074B0093074B084A26
:1026500008490230084CA047F4E7C046492500006D
:102660007569000079250000845C0200AC59020005
:10267000920400002C5C020059210100F8B50468A6
:102680001748184B9847002820D00026144D164FA5
:1026900004E001002800B84700280DD08442F8D09B
:1026A000036822689342F4D143681B0262681202F5
:1026B0009A42EED10126ECE7002E07D0210008480F
:1026C0000A4B984720000A4B9847F8BDA17920682B
:1026D000084B9847084B9847A188084B9847EDE767
:1026E000C44D0020851E01009D1E01006D1F0100CC
:1026F000C92301004925000065690000895E0000CA
:1027000030B583B004000B4B9847002805D0342324
:10271000E05CC006C00F03B030BD074B0093074A12
:1027200007490330074DA847220000230648074900
:102730008847FEE7AD170000785B0200410A000001
:102740002C5C020059210100205D0200B517000039
:10275000F0B587B004000E00344B984700280DD127
:10276000334B0093F022520032490330324DA847D8
:1027700022000023314832498847FEE72000314BD0
:102780009847002801D007B0F0BD20002E4B984795
:1027900007002E4B984705002D4B9847874209D0DC
:1027A00028002C4B9847874204D028002A4B984792
:1027B0008742E8D13222A35E20001030002202A915
:1027C000875C57540132082AFAD19BB202AA1188B9
:1027D000C91A11805188C91A51809188591891805D
:1027E000D1885B18D380310004A81C4B984700287F
:1027F000C9D020001A4B9847041E11D0174E220052
:10280000103204A90800B0470028BCD020000D4BAE
:1028100098470028B7D12000114B9847041EEED1ED
:1028200004A928000F4B9847ADE7C046AD1700003C
:10283000E05802002C5C020059210100205D0200DA
:10284000B517000001270000F12100004D22000013
:102850004518000085180000C51800000B14010081
:10286000A52100008154000030B585B00400174B4D
:10287000984700281DD03223E25E25001035002342
:1028800002A8E95C19540133082BFAD193B202A9CA
:102890000A88D21A0A804A88D21A4A808A889A18E4
:1028A0008A80CA889B18CB802000094B984705B0C6
:1028B00030BD084B0093084A08490330084DA8472B
:1028C00022000023074808498847FEE7AD170000AB
:1028D00051270000F85802000D0200002C5C020095
:1028E00059210100205D0200B5170000F0B583B04A
:1028F0000400164B984700280CD1154B0093154A3D
:1029000015490330154DA8472200002314481549E6
:102910008847FEE72000144B98470500061D30004D
:10292000124B984784420FD02800114FB84701231B
:102930002200310030000F4EB04722000121280054
:10294000EB6998472800B84703B0F0BDAD17000009
:102950000C590200620200002C5C020059210100A7
:10296000205D0200B5170000A5210000851E0100B2
:1029700069280000FD1F0100F0B5D6464F464646C7
:10298000C0B584B004000D0017002E4B98470028F6
:1029900041D02668002E4BD0338A228A9B1A5B19BD
:1029A0009BB29A461BB29846758A638AED1AED1956
:1029B000ADB22BB299464346002B02D14B46002BB9
:1029C00023D02000204FB84702A920001F4B984772
:1029D000238A53442382638AEB186382A38A534475
:1029E000A382E38AED18E5824A4641462000184B4F
:1029F000984702AA02212000E3699847F369220060
:102A00000121300098472000B84704B01CBC904614
:102A10009946A246F0BD0F4B00930F4A0F49033071
:102A20000F4DA847220000230E480F498847FEE7B4
:102A30000E4B0093074BA722920008490220084C36
:102A4000A047E2E7AD170000692800007D230000E1
:102A50000D1D000024590200960200002C5C0200AB
:102A600059210100205D0200B5170000545D0200ED
:102A700030B583B004000D000D4B984700280DD1F0
:102A80000C4B0093B32292000B4903300B4DA84727
:102A9000220000230A480B498847FEE720000A4B22
:102AA0009847020029002000084B984703B030BD2A
:102AB000AD170000345902002C5C020059210100BE
:102AC000205D0200B51700003D24000079290000B8
:102AD00030B583B004000D000D4B984700280DD190
:102AE0000C4B0093B62292000B4903300B4DA847C4
:102AF000220000230A480B498847FEE720000A4BC2
:102B0000984701002A002000084B984703B030BDC9
:102B1000AD170000445902002C5C0200592101004D
:102B2000205D0200B5170000D923000079290000BC
:102B3000F0B5D6464F464646C0B586B004000F00F5
:102B4000039299460EAB00229A5E90462D4B984711
:102B500000280CD12C4B00932C4A2D4903302D4DCD
:102B6000A847220000232C482C498847FEE7002F65
:102B700011D03800234B9847002811D1224B0093E5
:102B8000274A23490330234CA0473A000023224818
:102B900022498847FEE72000224B98470700E8E7D4
:102BA00005AD21001031380010302B00039A1E4E65
:102BB000B04720001B4B98471222835E6A8842442C
:102BC00029884944008A091A09B22980D21A12B206
:102BD0006A802000154B984748236A46127BE254CE
:102BE000043B4A46E25202334246E25227644922FB
:102BF000A35C02218B43A35406B01CBC90469946AB
:102C0000A246F0BDAD170000785902006D03000028
:102C10002C5C020059210100205D0200B517000064
:102C200071030000A52100003D1701007929000073
:102C3000F0B5DE4657464E464546E0B585B080467F
:102C40000391924699460EAB00229B5E9B46A84B91
:102C5000984700280CD1A74B0093A74AA7490330F7
:102C6000A74CA04742460023A648A7498847FEE74D
:102C70004046A64B984705004046A54B98470400A0
:102C80004046A44B9847C30F1B185B101EB240462A
:102C9000A14B9847C70F3F187F103FB2039B002BF3
:102CA0000BD00398924B984700280BD05346142B17
:102CB00026D89B00994AD3589F464046984B984740
:102CC0000390EEE78B4B0093964A8C4903308C4C73
:102CD000A047039A00238B488B498847FEE7039C53
:102CE00020008C4B9847C50F2D186D10AD1B2DB2D1
:102CF0002000894B9847C40F24186410E41B24B2A9
:102D00004046874B9847039A138A4B445D19018AC2
:102D1000691A1500528A5A441219448A121B12B2B7
:102D200009B24046804B9847482342465146D15409
:102D3000043B4946D15202335946D15215644922C7
:102D400043469B5C02210B4341468B5405B03CBC7F
:102D500090469946A246AB46F0BD75422DB27C42E4
:102D600024B2CDE703986B4B9847C50F2D186D1013
:102D7000AD1B2DB27C4224B2C2E70398654B984745
:102D8000851B2DB27C4224B2BAE775422DB203985E
:102D9000614B9847C41B24B2B2E7039C20005D4BF3
:102DA0009847C50F2D186D10AD1B2DB220005A4B42
:102DB0009847C41B24B2A3E7039C2000554B9847B7
:102DC000851B2DB22000544B9847C41B24B297E7B3
:102DD00075422DB20398504B9847C40F24186410C5
:102DE000E41B24B28CE7039C20004A4B9847851BC8
:102DF0002DB22000484B9847C40F24186410E41BE0
:102E000024B27DE775422DB27C4224B278E7039864
:102E1000404B9847C50F2D186D10AD1B2DB27C424D
:102E200024B26DE703983B4B9847851B2DB27C423B
:102E300024B265E775422DB20398374B9847C41BFF
:102E400024B25DE7039C2000324B9847C50F2D1834
:102E50006D10AD1B2DB220002F4B9847C41B24B220
:102E60004EE7039C20002B4B9847851B2DB220007A
:102E7000294B9847C41B24B242E775422DB27C42CD
:102E800024B23DE775422DB20398234B9847C40FF7
:102E900024186410E41B24B232E775422DB2039863
:102EA0001D4B9847C41B24B22AE70398194B984737
:102EB000851B2DB27C4224B222E7039C2000154BD7
:102EC0009847851B2DB22000134B9847C40F241838
:102ED0006410E41B24B213E7039C20000D4B9847B9
:102EE000851B2DB220000C4B9847C41B24B207E76A
:102EF000AD17000088590200950300002C5C020009
:102F000059210100205D0200B5170000D9230000FF
:102F10003D240000A1240000F524000064580200B4
:102F2000A5210000A10300007929000030B583B07D
:102F30000400174B9847002810D04923E35C9B07F7
:102F400019D54423E35E4822A25C4621615E0091CC
:102F5000216C20000F4CA04703B030BD0E4B0093F6
:102F60000E4A0F4903300F4DA847220000230E4898
:102F70000E498847FEE74423E35E4822A25C4621CF
:102F8000615E0091216C2000094CA047E4E7C04637
:102F9000AD170000312C00009C5902002A040000EB
:102FA0002C5C020059210100205D0200B5170000D1
:102FB000312B0000F8B5060000210C4B9847041E89
:102FC00012D00B4D094F2000A847002204212000F9
:102FD000E36998472000A8472000FFF7EBFF210096
:102FE0003000B847041EEED1F8BDC04615230000DE
:102FF0006928000030B583B005000C00354B9847B8
:10300000002813D0712C46D8702C22D2412C1AD80B
:10301000402C1ED2022C05D3072C1AD92300103BBA
:10302000082B16D928002C4B98472FE02B4B0093E8
:103030002B4A2C4903302C4CA0472A0000232B4854
:103040002B498847FEE7532C22D8502C01D24C2C18
:10305000E8D12800204B9847002204212800EB6982
:103060009847152C0AD3182C01D9FF2C06D12868B3
:10307000002803D0C3690022012198472800164B7D
:103080009847FF2C21D024B2002C1EDB03B030BDAA
:103090005C2CC7D1DDE77F2C0AD9164B9C4210D897
:1030A000154B9C42D5D2902CD3D0FF2CBAD1D0E76F
:1030B0007E2CCED2732CB5D3752CCAD97C2CB1D131
:1030C000C7E70E4B9C42ADD1C3E728000C4B984795
:1030D000DCE7C046AD17000069280000C4590200B3
:1030E0001D0500002C5C020059210100205D02003A
:1030F000B517000081800000808000008E800000F5
:10310000B52F000010B50400034B9847FF212000A5
:10311000024B984710BDC04625260000F52F000041
:10312000F0B5C64600B582B0070001910025214BDD
:103130009846002300931CE05A1CD2B20AE0A74232
:103140000FD0002F0DD00133DBB28B420DD01A000F
:103150000628F1D0009C8A42F1D2920034681459BA
:10316000EDE7FF210198144B98470135EDB2402D52
:103170000CD029000198C047061E07D0017900290C
:10318000F3D04379062018400023E0E7002101989E
:103190000A4B9847041E09D0084E21003800FFF75B
:1031A000BFFF21000198B047041EF6D102B004BC55
:1031B0009046F0BD49250000F52F000015230000C2
:1031C000F0B5D6464F4680B583B001900020114B34
:1031D00098478146002817D00F4B9A460F4F104E44
:1031E0004D4630352800D047041E07D021000198F5
:1031F000B84721002800B047041EF7D14846054BC8
:10320000984781460028EBD103B00CBC91469A4602
:10321000F0BDC046510E0100851E010021310000A5
:103220009D1E0100F8B504000D00817900683F4B38
:1032300098473F4B9847A1880F230B40082B19DC78
:10324000002D08D10823E25E3A4B9847A1882068F8
:10325000394B9847F8BDFF2D09D00823E65E0C23B3
:10326000E25E921B6A431212921912B2ECE70C232F
:10327000E25EE9E70B2B3CDC002D05DDFE2D05DDD4
:10328000A2892E4B9847E1E72289FAE7EDB2FF22A7
:10329000521B637BDB086B43667AF60856439E1924
:1032A00033029B19DB019B191B01DB0EA7897F05EC
:1032B000BF0E6F4326897605B60E5643BF193E02F0
:1032C000F619F601F619F600277BFF06FF0E7D437F
:1032D000277AFF06FF0E7A43AD182A025219D2014F
:1032E00052191201B60E7601D20EDB0232431A4396
:1032F000C7E70D2B11DC002D05DDFE2D05DD227B42
:103300000F4B9847A2E7227AFAE7227A237B9B1A8F
:103310005D432D125219D2B2F2E77F2D03DCA26871
:10332000084B984792E7E268FAE7C0464925000053
:1033300065690000AD5F0000F52F000035610000F9
:10334000BD6200003164000030B583B004000A4B58
:103350009847002802D0002003B030BD074B0093EF
:10336000074A08490330084DA847220000230748B0
:1033700007498847FEE7C046AD1700008C5B020096
:10338000B10A00002C5C020059210100205D0200FE
:10339000B5170000F0B5DE4657464E464546E0B547
:1033A00083B082460D00002811D0E24B98470028D8
:1033B00000D051E1E04B0093ED22E0490330E04CB6
:1033C000A04752460023DF48DF498847FEE7DF4B2E
:1033D0009847002809D1DE4B0093D74BCF22D7491D
:1033E0000230D74CA047544619E23030D94B9847A9
:1033F0000400D04B984700280CD1CF4B0093D42227
:10340000CE490330CE4DA84722000023D248CE49F2
:103410008847FEE7002C00D101E24C212000CF4B71
:10342000984722003432537830218B435370CC4B71
:10343000E361CC4B23620023A361238263820020DB
:10344000C94B98470138A0820020C84B98470138E3
:10345000E082201D4C21C64B984700210020618648
:1034600000233022A0540132A3541732A354442322
:10347000E1520233E15221640132A35C0127BB43D4
:10348000A354A16334239846E25C4B3313400122DA
:103490009446624613437D221340793A93432700B2
:1034A00034377A780E26B2430626B1464E4632436A
:1034B0000826B3430836B3432C36A0551C3EB3430D
:1034C0002036B3434646A35563461A437A703D23DC
:1034D000E05461620C3F3800A64B9847002D00D1A4
:1034E0007BE1290028313800A34B98472900183187
:1034F000220010322B001033187810700132013383
:103500008B42F9D13222AB5E63863023EA5CE2540F
:103510000133EA5CE2541733EA5CE254043BEA5EAE
:10352000E2520233EA5EE2522B6C23644922A95C28
:1035300001239B4601273940A35C584683430B4334
:10354000A354AB69A3613423EA5CD209D101E25CE4
:1035500094467F22664632400A43E254EA5CD20730
:10356000D20FE15C81430A43E254EA5C52083A40DC
:103570005200E15C0226B1430A43E25435229446EC
:10358000AA5C210034310C361640B0464A780E262B
:10359000B243464632434A70EA5C92083A4092008F
:1035A000E65CB0460426B14646464846864332436A
:1035B000E254EA5CD2083A40D200E05C804608203F
:1035C000464686433243E254EA5C12093A4012010D
:1035D000E05C80461020464686433243E254EA5C73
:1035E00052093A405201E05C80462020464686431C
:1035F0003243E254EA5C92093A409201E75C40208F
:1036000087433A43E2540833EA5CE2546346EB5C96
:10361000DB07DB0F4A785846824313434B70A86B95
:10362000002802D02100554B98472800544B98475A
:10363000002800D1DEE05346002B00D1E6E0280050
:10364000504B9847070028004F4B9847020039001D
:1036500020004E4B9847D0E05346181D3D4B9847ED
:103660000400344B984700284BD0002C00D1D6E002
:103670004C212000394B98475346236022003432B6
:10368000537830218B435370354BE361354B2362C4
:103690000023A361534612229B5E638253465F8AD6
:1036A00000203B4B98473223434350334022FF32A4
:1036B0000120934232D8C019E0822000354B984750
:1036C00001286BD0534610229B5E238253461F8AEB
:1036D00000202F4B98476423434350334022FF324E
:1036E000012093420AD90020294B98470300642007
:1036F00058435030A021284B984780B2C019A0826F
:10370000A7E60D4B0093F0220C4903300C4DA8475F
:103710002200002310480C498847FEE700201C4B7C
:1037200098470300322058435030A0211A4B984745
:1037300080B2C0E7AD170000C45802002C5C020044
:1037400059210100205D0200B5170000750D010030
:10375000BC5C0200E51D01005458020075290100FF
:1037600021500000514A0000810D0100A90D010007
:10377000D11D0100715B0000E5690000AD1A000079
:10378000A5210000D92300003D2400007929000074
:10379000D10D010049330000A5C001005346142299
:1037A0009B5EA38253469F8A0020214B9847642347
:1037B000434350334022FF32012093420AD9002074
:1037C0001B4B98470300642058435030A021194BED
:1037D000984780B2381A20823BE65346002B04D02B
:1037E00002212000144B984707E001212000124BD2
:1037F00098470BE05346002B08D05346DB69220064
:1038000001215046984720000C4B98470C4B0093E1
:103810000C4B8822FF320C4901200C4DA847200098
:1038200003B03CBC90469946A246AB46F0BDC046AC
:10383000D10D0100A5C00100E5400100692800008C
:103840000C5D0200C45802002C5C020059210100EA
:10385000F0B585B004000D001600314B98470028E4
:103860000CD1304B0093304A30490330304DA847DB
:10387000220000232F4830498847FEE720002F4BC5
:103880009847A8423BD020002D4B984702A9200022
:103890002C4B9847013E638A9E19E68220002A4BF2
:1038A0009847012831D0013D238AED18A58202AA4C
:1038B00002212000E36998472000244B9847002804
:1038C00003D0C369220001219847261D3000204BF8
:1038D0009847051E0AD01F4F02AA03212800EB6952
:1038E000984729003000B847051EF5D12000144B39
:1038F00098474923E35CDB070DD405B0F0BD2000F9
:10390000154B9847B042BED1F7E701235B1BA58A50
:10391000ED182582CBE72000104B9847EDE7C04615
:10392000AD17000054590200E50200002C5C0200B3
:1039300059210100205D0200B5170000A1240000FC
:10394000692800007D23000049330000A521000004
:10395000851E01009D1E0100F52400002D2F000092
:1039600030B583B004000D000D4B984700280CD1F2
:103970000C4B00930C4A0D4903300D4DA847220013
:1039800000230C480C498847FEE720000B4B984762
:1039900001002A0020000A4B984703B030BDC04602
:1039A000AD17000064590200270300002C5C0200E0
:1039B00059210100205D0200B5170000A12400007C
:1039C0005138000030B583B004000D000C4B98470F
:1039D000002807D03C23E05C2840431E9841C0B239
:1039E00003B030BD074B0093074A08490330084D28
:1039F000A84722000023074807498847FEE7C0463A
:103A0000AD170000A05B0200D70A00002C5C02008A
:103A100059210100205D0200B517000070B584B087
:103A200005000E00104B9847002805D03F2E10D8F7
:103A30003D23E85C04B070BD0C4B00930C4A0D496B
:103A400003300D4CA0472A0000230C480C4988473E
:103A5000FEE703AC267000236370220009212800D2
:103A6000084B98476078E5E7AD170000B45B0200AB
:103A7000DE0A00002C5C020059210100205D0200DA
:103A8000B51700008D200000F0B5DE4657464E46C3
:103A9000C0B584B006000D001700130A019300287A
:103AA00030D0244B9B46244B9A46244B99460CE03D
:103AB00002AB06330020185E04B01CBC91469A4647
:103AC000A346F0BD0025002E1DD029003000D847A8
:103AD000009029003000D04704023C19A4B202AB88
:103AE0009A1D21000098C8470128E1D06B461B7938
:103AF0005BB2002B07DA002DE4D13000104B984761
:103B00000600DFE714000F4B1C40222C10D007D812
:103B10000620032CD0D0072C08D180204000CBE712
:103B20000F20312CC8D00130C02CC5D00020C3E7F5
:103B3000FF20C1E7492500001D3A0000616B00002D
:103B4000A5210000FF80FFFFF0B5DE4657464E4638
:103B5000C0B584B006000D001700130A01930028B9
:103B600028D01C4B9B461C4B9A461C4B994605E0A3
:103B700003AB188825E00025002E1CD0290030005A
:103B8000D847009029003000D04704023C19A4B265
:103B900003AA21000098C8470128E9D06B461B7989
:103BA0005BB2002B07DA002DE5D130000C4B9847B3
:103BB0000600E0E714000B4B1C40293C0020012CC0
:103BC00005D904B01CBC91469A46A346F0BD064BED
:103BD0001888F6E7492500001D3A0000356C000002
:103BE000A5210000FF80FFFFB8580200F0B5DE46B7
:103BF00057464E46C0B584B006000D001700130AA4
:103C00000193002829D01E4B9B461E4B9A461E4B03
:103C1000994605E002ABD8792AE00025002E1DD098
:103C200029003000D847009029003000D047040216
:103C30003C19A4B202ABDA1D21000098C847012844
:103C4000E8D06B461B795BB2002B07DA002DE4D17C
:103C500030000E4B98470600DFE714000C4B1C4069
:103C60006D2C0BD00B4B9C4208D02C2C06D0FF2087
:103C700004B01CBC91469A46A346F0BD0020F7E76D
:103C8000492500001D3A0000016D0000A52100003B
:103C9000FF80FFFFAD800000F0B5DE4657464E4680
:103CA000C0B584B006000D001700130A0193002868
:103CB0002CD01F4B9B461F4B9A461F4B994609E041
:103CC000039804B01CBC91469A46A346F0BD00255B
:103CD000002E1CD029003000D84700902900300069
:103CE000D04704023C19A4B203AA21000098C84797
:103CF0000128E5D06B461B795BB2002B07DA002D5B
:103D0000E5D130000D4B98470600E0E714000C4B5E
:103D10001C40BE2C09D00B4B9C4203D07E2C01D002
:103D20000020CEE7084B9847CBE70848C9E7C046D4
:103D3000492500001D3A0000D56D0000A5210000B6
:103D4000FF80FFFF8E800000D94001004CA70200D9
:103D500070B50468A5880F232B40082B13DD0B2BAF
:103D600018DD0D2B1DDDA1792A002068104B984726
:103D7000A0600023A380A17923002A0020680D4EB3
:103D8000B047A58070BDA1792A0020680A4B9847EA
:103D90002081EEE7A1792A002068084B984720810E
:103DA000E7E7A1792A002068054B98472072E0E7F1
:103DB000993C000079250000893A0000493B000049
:103DC000ED3B0000F0B5DE4657464E464546E0B5B1
:103DD0009FB004008B463D23C35C8B4200D13EE282
:103DE000D64B9847002808D03D23E25C91465A46BE
:103DF000E25400230293CA46E8E1D14B0093D14A32
:103E0000D1490330D14DA84722000023D048D149E1
:103E10008847FEE773790422134373713D23994663
:103E20005246E2542A0002992000CB4FB84709902D
:103E30004B465A46E2542A0002992000B847804671
:103E40007379042293437371099B83424BD03D26BF
:103E50005346A3552A0002992000BF4B9847020001
:103E600081465B46A35529000398BC4B9847012D1A
:103E700000D196E0BA48BB4B98470600AF4B984735
:103E8000002800D1A2E0002E2DD04B4633814346BE
:103E9000B3813460B5806B461B7AB3710EA8B24B08
:103EA00098470E96B14B0F93B14B1093B14B1193B2
:103EB00000231493FF331593089B1693079B5B42D3
:103EC0001793069B1800083012AA19781170013256
:103ED00001338342F9D10EA83622835C01218B4342
:103EE0008354A54B9847049B023304930C2B00D1B9
:103EF00066E10BAB049AD55A002DF4D005989F4B80
:103F00009847029920009E4B984706009D4B984782
:103F100003900F232B40082B00DC7BE70B2B63DD8A
:103F20000D2B00DDBBE073790422134373713D2335
:103F300099465246E2542A0002992000924FB8470F
:103F400080464B465A46E2542A0002992000B84760
:103F50000700737904229343737143468342C2D0AE
:103F60003D265346A3552A0002992000864B9847C8
:103F7000020009905B46A35529000398834B98479C
:103F80007748784B984706006C4B9847002879D0C3
:103F9000002EA8D06B4624229B181B7833723773EF
:103FA00077E77B4B994500D160E1984500D061E708
:103FB0002000784FB847C60F3618761036B220006A
:103FC000B847C30F1B185B101BB267E1724B00931D
:103FD000EB2212015C4903305C4CA0473200002305
:103FE0006E485C498847FEE7737904221343737176
:103FF0003D2399465246E2542A0002992000684B1C
:1040000098469847071C4B465A46E2542A000299A4
:104010002000C0476B4698847379042293437371E0
:10402000BFB283B29F4200D15DE73D265346A35500
:104030002A00029920005A4B9847071C5B46A3555B
:10404000021C29000398574B98474548454B984711
:1040500006003A4B9847002807D0002E00D142E7CF
:1040600037816B469B8CB38113E74B4B00934E4AD1
:1040700035490330354CA0473200002347483549C5
:104080008847FEE7444B0093484A2F4903302F4CA2
:10409000A0473200002341482E498847FEE73D23D0
:1040A00099465246E25473790422134373712A00ED
:1040B000029920003E4FB8470A904B465A46E254B8
:1040C0002A0002992000B84707000E907379042255
:1040D000934373710EA90AA8364B9847002800D164
:1040E00001E73D265346A3552A0002992000304B94
:1040F000984781460A905B46A35502002900039821
:104100002D4B98471648174B984706000B4B98477E
:10411000002806D0002E00D1E5E64B46B360F760DC
:10412000B7E61D4B0093254A07490330074CA047CB
:1041300032000023194807498847FEE7AD17000001
:10414000085A0200370600002C5C020059210100C9
:10415000205D0200B5170000893A0000AD5F000045
:10416000C44D0020E51D0100B911010025320000F9
:10417000513D00007D26000079120100AD6A00006B
:104180004925000065690000ED3B0000BD620000AC
:10419000FF7F0000A12400001C5C020054580200B4
:1041A000493B000035610000C40E0000D90E00003C
:1041B000993C000041C6010031640000ED0E000092
:1041C000029B0133DBB20293402B44D002992000C2
:1041D000364B9847059000283DD043791B07EFD414
:1041E000B022029E31002000314B98470890B12246
:1041F000310020002E4B98470790BE22310020004E
:104200002C4B98470690B22231002000284B98474B
:104210000BAD2880B32231002000254B98476880E1
:10422000B42231002000224B9847A880B5223100EB
:1042300020001F4B9847E880B622310020001C4B1D
:1042400098472881B72231002000194B9847688190
:10425000002304934DE6FF212000174B98471FB021
:104260003CBC90469946A246AB46F0BD2000134F99
:10427000B847C60F3618761036B22000B847C30FBD
:104280001B185B101BB2711C5A1C8A4200DD0A000D
:1042900012B291460A4A904500D0EBE5013601334F
:1042A000B34200DD33001BB29846E3E54925000028
:1042B000893A0000993C0000F52F0000A12400007D
:1042C000FF7F000030B583B004000D000D4B984710
:1042D00000280AD03D23E35C290019438B4202D019
:1042E0002000094B984703B030BD084B0093084AA3
:1042F00008490330084DA847220000230748084911
:104300008847FEE7AD170000C53D00001C5A0200BB
:104310007E0600002C5C020059210100205D020095
:10432000B517000030B583B004000D000D4B984761
:1043300000280AD03D23E35C1900A9438B4202D038
:104340002000094B984703B030BD084B0093084A42
:1043500008490330084DA8472200002307480849B0
:104360008847FEE7AD170000C53D0000305A020047
:104370008F0600002C5C020059210100205D020024
:10438000B517000030B583B004000A4B98470028E9
:1043900002D0E06903B030BD074B0093074A0849DB
:1043A0000330084DA84722000023074807498847E3
:1043B000FEE7C046AD170000C85B0200F50A00002A
:1043C0002C5C020059210100205D0200B51700009D
:1043D00030B583B004000A4B9847002802D0606AC9
:1043E00003B030BD074B0093074A08490330084D1E
:1043F000A84722000023074807498847FEE7C04630
:10440000AD170000E05B02001E0B00002C5C0200F8
:1044100059210100205D0200B517000030B583B0BE
:1044200004000A4B9847002802D0A06B03B030BDAF
:10443000074B0093074A08490330084DA84722005C
:104440000023074807498847FEE7C046AD1700002C
:10445000F45B02006F0B00002C5C0200592101008C
:10446000205D0200B5170000F0B583B00500002202
:1044700015213E4B984728003D4B9847071E02D018
:1044800028003C4B9847002128003B4B98470023CD
:10449000FF22FF212800394CA0472B1D0193180053
:1044A000374B9847041E0AD0364E21000198B0477A
:1044B00000902000FFF7D8FF009C002CF5D1324B74
:1044C0001B68002B09D0012202E09B68002B04D05E
:1044D00019688D42F9D11A71F7E700202B4B9847E4
:1044E000041E22D02A4E0DE029002000B047E36BC5
:1044F0009D420ED0A36D9F420ED02000234B9847C3
:10450000041E12D0636B9D42EED0A36B9D42EED190
:10451000EAE70023E363EDE71E4B98478542ECD1C1
:10452000290020001A4B9847E7E7002200212800C5
:10453000EB6998472800184B984700280DD00430A5
:104540002900164B9847686A002801D0144B9847F9
:104550002800134B984703B0F0BD2800114B984733
:10456000303029000D4B9847EDE7C046DD1F0000B5
:104570001D4400008D1B0000FD1101007925000085
:10458000851E01009D1E0100F0260020B90E0100CD
:10459000711C0000011D0000A52100006D1F01001D
:1045A000C92301004D22000070B582B00400194BF0
:1045B000984700280DD1184B00939422FF321749D9
:1045C0000330174DA8472200002316481649884794
:1045D000FEE72000154B98472000154B9847051E15
:1045E00008D02000134B9847EB69002201212800D6
:1045F00098470CE02000104B9847051E07D0C66B6B
:1046000020000C4B9847B44201D10023EB630020FB
:1046100002B070BDAD170000D45802002C5C02003F
:1046200059210100205D0200B51700006928000033
:10463000A5210000694400004D22000030B583B080
:1046400004000F4B984700280AD0A06B002814D014
:104650000C4B9847201A44426041C0B203B030BDB1
:10466000094B0093094A0A4903300A4DA847220022
:104670000023094809498847FEE70020EEE7C046C5
:10468000AD1700003D1C0000085C02007F0B00001D
:104690002C5C020059210100205D0200B5170000CA
:1046A00010B582B03023C35C028AD21A6C462280D5
:1046B000828A9B18A3803123C35C428AD21A62800B
:1046C000C28A9B18E38000226846024B984702B0DA
:1046D00010BDC046C514010010B50368002B0DD0F5
:1046E000021D01231468002C04D00133DBB2043214
:1046F000072BF7D19B001950012010BD0023F9E7CB
:10470000F0B5CE4600B582B005000E0014000122BF
:10471000C84B98472080C84A31002800C74B9847AB
:1047200001900700052835D9237B002B3FD1237D3D
:10473000002B00D06CE0237F002B00D08FE03623CD
:10474000E35C002B00D0AFE02823E35C052B00D90D
:10475000F7E04423E35C052B00D923E1F92F22D8AD
:104760006B469B88227B5A43120A2273227D5A434E
:10477000120A22752821625C5A43120A62540E31D1
:10478000625C5A43120A62544422A75C5F433F0AA8
:10479000A75408E00023237323752822A3540E3264
:1047A000A3540E32A35402B004BC9146F0BD2C2297
:1047B00031002800A14B984720730528B7D929223A
:1047C000310028009E4B984760802322310028004A
:1047D000984B9847C0B2A071002806D12022310022
:1047E0002800944B98476073A1E72A2231002800E3
:1047F000934B9847A0802122310028008D4B994689
:1048000098472081222231002800C8476081E5E7CF
:10481000302231002800874B98472082002800D1A1
:1048200089E73C2231002800844B984720750528F1
:1048300006D83222310028007E4B984760757AE70F
:104840003122310028007B4B9847FF2318406082BB
:104850003922310028007A4B9847E081E9E740226D
:1048600031002800734B98472083002800D166E769
:104870004C2231002800714B98472077052806D834
:104880004222310028006B4B9847607757E741225E
:1048900031002800674B9847608349223100280087
:1048A000674B9847E082EBE76E2231002800654BAA
:1048B0009847E062002800D146E76C2231002800CA
:1048C0005E4B98473623E054052800D83CE76D221C
:1048D00031002800594B98473723E05461223100BA
:1048E0002800544B98470300581E83413822A05C8F
:1048F000012188431843A054E06A534B984702288B
:104900000BD03723E35C052B14D86022310028003C
:10491000484B98473923E05416E7692231002800B4
:10492000474B9847A086494A31002800454B984795
:104930002063EAE7692231002800414B9847A086AE
:10494000E3E75022310028003A4B984720840028A2
:1049500000D1FEE65C2231002800384B984728231E
:10496000E054052800D8F4E6512231002800314BEC
:10497000994698476084522231002800C847A08495
:10498000532231002800C847E08459223100280012
:104990002B4B9847E083542231002800C847292335
:1049A000E054D6E67F2231002800264B9847E0638A
:1049B000002800D1D2E67C22310028001F4B984706
:1049C0004423E054052800D8C8E6732231002800AB
:1049D000184B994698474823E0527422310028002A
:1049E000C8474A23E052792231002800144B9847E7
:1049F0004623E0527E2231002800124B9847206463
:104A0000702231002800C8474C23E0527122310047
:104A10002800C8474E23E052752231002800C847BD
:104A20005023E054722231002800C8475123E0543B
:104A300094E6C046893A00000C800000ED3B00007F
:104A4000493B0000993C0000899500008E800000E1
:104A5000F0B59BB004000E00022A07D0002A61D0F6
:104A60000020012A00D1B5E01BB0F0BD0021814B30
:104A7000984703000320002BF6D1012200212000DB
:104A80007C4FB8470190042200212000B847050060
:104A9000052200212000B84727001037002305A970
:104AA000FA5C5A540133082BFAD1ADB205A90B8830
:104AB0005B1B0B808B88ED188D8080B24B881B1A96
:104AC0004B80CB88C018C880019A30006A4B984749
:104AD00003000220002BC7D02C2200212000674BAE
:104AE000984703000220F92BBED920220021200084
:104AF000604B9847C3B20220002BB5D1322200216F
:104B000020005C4B9847C3B20220002BACD15C4A1A
:104B100000212000594B98470023F92282425B4133
:104B2000581CA1E705A8574B9847332200212000C5
:104B3000504B9847002802D0002205AB1A7505AAF1
:104B400000212000504B9847042200212000494FAB
:104B5000B8470500052200212000B847270010377C
:104B6000002303A9FA5C5A540133082BFAD1ADB2E1
:104B700003AB1A88521B1A809A88AD189D8080B2A8
:104B80005A88121A5A80DA888018D88005AA31000B
:104B900018003E4B9847022200212000354B9847D1
:104BA000002801D100205FE71C20394B9847050001
:104BB0000122002120002F4B9847020000233900DA
:104BC0002800344EB04798239B00E1182800324B50
:104BD0009847E7E7013200212000264B984700283C
:104BE00040D1332200212000224B984703000020AF
:104BF000002B00D138E705AD2800224B9847002351
:104C00002B733622AB540E3AAB542A0000212000FD
:104C10001D4B9847042200212000164FB84705007D
:104C2000052200212000B8471034002303A9E25CCC
:104C30005A540133082BFAD1ADB203AB1A88521B78
:104C40001A809A88AD189D8080B25A88121A5A80AC
:104C5000DA888018D88005AA310018000B4B9847D5
:104C6000002001E798239B00E0180C4B98470C4B61
:104C70009847B6E7893A000099160100ED3B00001D
:104C80000C800000CDBF00000147000071C0000093
:104C9000A127010001BD000075BA000041BB000062
:104CA00065240100F8B505000E001400214A224BCE
:104CB00098472072052800D8F8BD204A3100280006
:104CC0001D4B9847F92803D8237A5843000A2072CD
:104CD000237A052BF0D91A4A31002800194B98473E
:104CE0002080194A31002800184FB847A081184A7F
:104CF00031002800B8476081164A31002800B847C3
:104D00002076154A31002800B8476076134A3100F2
:104D10002800134B98476060E289124B9A42CBD02F
:104D2000228A9A42C8D0104A31002800054B984781
:104D30002080C1E78C800000ED3B00000C8000006B
:104D400089800000493B000080800000893A000013
:104D50008180000082800000838000008E8000003F
:104D6000993C0000FFFF00008A80000070B505003C
:104D70000E0014001F4A204B98472070052800D8C9
:104D800070BD1E4A310028001B4B9847F92803D8F4
:104D900023785843000A20702378052BF0D900238C
:104DA00063800133FF332381AB8A01332A8A9B1A44
:104DB0001BB2DA0FD3185B10A380EB8A01336A8A27
:104DC0009B1A1BB2DA0FD3185B10E3800C4A310038
:104DD0002800094B9847A0720A4A310028000A4B64
:104DE0009847A081094A31002800094B9847A073D1
:104DF000C6E7C046AC800000ED3B00000C80000020
:104E0000AD800000A9800000493B0000A0800000A8
:104E1000893A0000F0B5DE4657464E46C0B58AB026
:104E2000040004915022784B98470600051E30D1AB
:104E30007F22049F39002000744B9847061E06D03D
:104E40007C2239002000724B9847052850D8402218
:104E5000049920006C4B9847061E00D0C0E0042245
:104E600004992000684FB8470600052204992000E5
:104E7000B847031CB04200DA331C1AB2002A01DD25
:104E8000ED182DB228000AB01CBC91469A46A346E4
:104E9000F0BD5C22049920005D4B98470025052851
:104EA000C6D95322049D29002000574FB847F30F5D
:104EB0009E19761001363618B6B251220495290093
:104EC0002000B8470500522204992000B847EA178D
:104ED000AB185340C21780185040984200DA1800AF
:104EE0003018031C020401D41DB2A1E70023FBE724
:104EF0007022049F39002000434B99469847059043
:104F0000702239002000C84783467E22049739006A
:104F100020003E4B9847020006AF00218A460291CE
:104F20003C4B019359460091059B310038003A4EA5
:104F3000B04708AE5346338073803B88013BB38053
:104F40007B88013BF3807522049F39002000C8470D
:104F50000590732239002000C84782467422390028
:104F60002000C847814607AA13006A46127D200028
:104F7000103005933100294FB847059A13885344E0
:104F80009BB252884A4492B21020215E36889E1904
:104F900036B28E1BAE4200DA2E001221605E08A9E6
:104FA0004988511809B236B2411AB14200DA3100CB
:104FB00008A880881B181BB21425605F09B21B1A51
:104FC0008B4200DA0B0008A9C988521812B21620C9
:104FD000215E1BB2521A9A4200DA1A0015B236E765
:104FE0004C22049920000A4B9847052800D836E740
:104FF000412204992000044B98478619AE4200DAFA
:105000002E0035B22BE7C046893A0000993C0000DB
:10501000ED3B0000187C00003D3F01003D17010002
:1050200010B5040008291BD0072924D0012927D056
:1050300006292BD0032935D004293DD00B293FD098
:105040000B000D3B012B40D9162943D0172957D00F
:10505000012000290AD120002C4B9847012005E0AF
:105060001378002B03D128345460012010BD002395
:1050700053600120FAE726491000264B9847F5E7D0
:10508000254B984701235840C0B2EFE70021234B3E
:105090009847638E1A1C1BB2834200DA021C628698
:1050A0000120E3E74923C35C0120DB07DED52000B4
:1050B0001B4B98470120D9E71A4B98470120D5E7A9
:1050C0000531194B98470120D0E71021174B98471D
:1050D0000120CBE7164B9847164B9847002805D080
:1050E00006212000104B98470120BFE70221200035
:1050F0000D4B9847042120000C4B98470120B5E741
:1051000011390A4B98470120B0E7C0462526000018
:105110008C5D0200D9460000C5390000154E000024
:105120002D2F00004D210000C54200002543000046
:105130001D440000531C0000F0B5CE4600B582B0FF
:10514000040001900D00103100221F4B98470028E9
:1051500027D03423EB5CDB0625D42B6A002B28D028
:105160000222210028009847814603281DD02E1DC9
:105170003000164B9847041E0BD0154F21000198A4
:10518000FFF7DAFF002808D121003000B847041EDD
:10519000F4D100204B46012B09D002B004BC91464B
:1051A000F0BD0020F9E70020F7E70020F5E7280030
:1051B000F3E72E1D3000054B984704000223994663
:1051C0000028DAD1E9E7C04699160100851E0100E2
:1051D0009D1E0100F0B5D6464F4680B58DB0070044
:1051E0000D003423C35CDB0604D50DB00CBC914626
:1051F0009A46F0BD3223C65E06AC21002E4B98477E
:10520000B3B22288D21A22806288D21A6280A2881F
:105210009A18A280E2889B18E3802200290008A83F
:10522000264B98470028E0D03B6A002B03D0002291
:1052300008A93800984706A938001F4B984706AAC6
:1052400029000AA81D4B9847002807D13B6A002B6C
:10525000CBD0012208A938009847C6E73B1D01932F
:105260001800174B9847051EF0D0134B9A46134B66
:105270009946144E04E029000198B047051EE5D078
:1052800004AC21002800D0476B8E2288D21A2280DD
:105290006288D21A6280A2889A18A280E2889B183B
:1052A000E38022000AA902A8C8470028E3D002A987
:1052B0002800FFF78FFFDEE77D2300000B140100BD
:1052C000911E0100C51E0100F0B5D64600B582B0A2
:1052D000041E01910DD0019920001A4B984720001F
:1052E000194B9847051E0AD0184B9A46154E1F00B9
:1052F00010E0174B1868174B9847041EEBD102B00B
:1053000004BC9246F0BD28000F4B98472C000028A3
:10531000F5D005002B1D009321001800D047041E76
:1053200007D001992000B04721000098B847041E1B
:10533000F7D12B6A002BE6D001220199280098476B
:10534000E1E7C046D5510000A5210000C51E0100BF
:10535000F82600204518000070B51C4D28681C4B2D
:105360009847040028681B4B984700280DD101235B
:10537000A361164B186843681A6AD2070FD51B6AD7
:105380009B070CD50123E3610BE0104D2868A3694E
:10539000002BECD0C369002BF9D09847F6E7002327
:1053A000E361C368002B03D021001031A268984745
:1053B0002368002B06D06268002A03D0A1688B42C4
:1053C00001D0A36070BDA260FCE7C046F8260020B3
:1053D000750E0100790E010070B582B005001C4EFB
:1053E00030681C4B9847040030681B4B98470028D6
:1053F00009D1174E3068A369002B04D0C369002B74
:10540000F9D09847F6E72200103229006846134B7E
:1054100098470F4C2068124B984701006846114B83
:1054200098476946104DA8472068104B9847694631
:10543000A84720680E4B98476946A84720680D4B3F
:105440009847002801D002B070BD0B4B9847FAE78F
:10545000F8260020750E0100790E01000B140100E2
:105460004518000039510000C9520000851800009D
:10547000C5180000910E010059530000704700004C
:10548000F0B585B005000E00002857D0002E5AD088
:1054900002AC0023238063802800374B98470138F3
:1054A000A0802800354B98470138E0802200310069
:1054B0006846334B984700284BD02B69002B02D00D
:1054C000694628009847B4235B00EB5A9B059B0D67
:1054D000002B14DD002100242A4EB4277F0009315F
:1054E000C900691800226846B047002831D101344C
:1054F000A4B22100EB5B9B059B0D9C42EFDB1F2BB5
:1055000029DC0933DB00EB1800226946515C995411
:105510000132082AF9D1B42149006B5A9A0580203A
:10552000C00384466244920D9B0A9B0213436B5254
:10553000E86A6639FF39144B98470AE0134B9847DD
:10554000051E06D0A2E7B4225200AB5A9B0A9B026A
:10555000AB5205B0F0BDB4225200AB5A9B0A9B027D
:10556000AB5228004830002302A95A5CC2540133D0
:10557000082BFAD1CFE7C046810D0100A90D01002B
:105580000B140100991601008D380100750D010002
:10559000014B18687047C046F8260020F0B5DE467B
:1055A00057464E464546E0B58DB00500D04B98476E
:1055B0000990D04CEB68236000212800CE4B98471F
:1055C0002068C36B002B0ED0B4235B00C35A9B052D
:1055D00048270026002B00D19EE2C64B9846C74BB9
:1055E0009A46C34656E0B4225200835A9B0A9B0255
:1055F000835287E22D194935FF35073B2B70013463
:10560000BC4B1868B4235B00C35A9B059B0D9C429E
:1056100035D203194933FF331B78002BEFD1A64253
:10562000EDD025000935ED004119C019D0470028FB
:10563000E5D05B4619684A19C9190AA8B04B9847C2
:105640000AA8B04B9946984703905B461B68D81947
:10565000C84704905B461B685819C847049B9C4682
:105660006044039B8342CAD2A24B1D68E819002301
:105670000AA95A5CC2540133082BFAD1BAE70136A1
:105680009C4B1868B4235B00C35A9B059B0D0837DD
:105690009E420FD280194930FF300378002BEED1A3
:1056A00043461868B4235B00C35A9B0500D115E23A
:1056B0000024AEE70021944A1160B4225200825ABD
:1056C000920500D112E21A00013A07922DD40799EF
:1056D00042184932FF321278002A0DD04733FF3387
:1056E000C3180A00013A05D3013B59780029F9D1C2
:1056F000079201E00023079341682023CA5C01243C
:10570000A243CA544168CA5C02208243CA54794BFE
:105710001C68B4235B00E35A9B0500D1E6E14823F3
:10572000069300230493270045E000230793E3E753
:10573000796820228B5C012003438B5446E06D4C3A
:105740002068724B98470500002606822068704B3F
:1057500098470138A8826E8220686E4B98470138BE
:10576000E8822368596820228B5C022003438B5413
:105770000398694B98475F4B18688369002B09D0E1
:10578000069B9C4660445F4B98475F4B1A68944663
:1057900060441860049B01331A000493554B1F6842
:1057A000069B08330693B4235B00FB5A9B059B0DB5
:1057B0009A4200DB9AE1049ABB184933FF331B7805
:1057C000002BE7D1079B19009142B1D079682022C4
:1057D0008B5C022083438B54069B9C46BC446346EF
:1057E000039338004D4B98470028A8D1414B9A4667
:1057F0001868464B98470600049BDB00FF184C23B3
:10580000FC5A0134043BFB5AE41A23B298464E2357
:10581000FC5E651C4A23FB5AED1A2DB253461868EC
:105820003C4B984784423CDA4E23FB5E9946414606
:10583000F0683B4B9847A846854200DD80462D4BDB
:105840001B681B69002B3DD00AAB00221A809A808E
:105850005A8043461BB29A460AAD264B9B46534696
:10586000B2464246B84617001E00741E24B2EC80B1
:105870005B4618680369290098470623E95E4B1CBC
:105880006A889B1A1BB29F4213DA261EEDDC254B59
:105890000093254BA022FF3224490220244CA0472C
:1058A00069E7144B18681B4B9847013803B29946B7
:1058B000BDE74746330056469A464B1C984653462A
:1058C000002BE4DD4A23FC5E4B4605934346E31878
:1058D000013B4B4571DC43466A465384538C9A46E0
:1058E00001235B4253449B464B46B9461F002EE0C2
:1058F000F90E0100F82600208D3801005516010030
:1059000079140100EF130100FC260020750E010040
:10591000810D0100A90D0100D9530000910E010075
:10592000A5C00100D85D0200945D0200A45D0200E4
:1059300059210100AF421CD003987D4B9847544435
:1059400024B24346E318013B059A93421ADC4823EC
:105950004A46D35E33824C234A46D35EB382748276
:10596000A4B25B46E5182DB2F582AF42E2DAF782C7
:105970003D00704B1B68596820228B5C022003435A
:105980008B54D9E73B004F469946A94500D1F2E632
:105990004823FB5E33824C23FB5EB38274824B460A
:1059A000F382644B1B68596820228B5C02200343FE
:1059B0008B5403985E4B9847DDE60025E5E75E4B88
:1059C0009847002804D05B4B18684369002B1FD010
:1059D000584C2068483080214900584DA84720681D
:1059E0004930FF302021A8472168B42252008B5A49
:1059F0009B0A9B028B520998514B984701002068E3
:105A00008369002B00D179E04E4A1268984775E00F
:105A10004D4B984704004D4B9847A369002BFCD190
:105A2000A3689B46236899469B4501D163689946C4
:105A3000404C2068464B984703902368B42252009C
:105A40009A5A9205C4D042009246002635000BE0D7
:105A50000136B6B23500374B1B68B42252009A5A51
:105A60009205920D9642B3DA5A194932FF321278F2
:105A7000002AEDD1EA009B184A229F5E48229A5ED6
:105A8000039C7C43A41864004C215B5A01339B1A8D
:105A90001BB25B0004932B000933DB00254A12681C
:105AA00005929446634406229B5EBB42D0DBA0462F
:105AB000D8444C440935ED00049A21004046254B5A
:105AC000984701373FB2D04454441A4B1B680593A2
:105AD0005B1906229B5EBB42EEDAB9E70022194B46
:105AE0001A60B4235B00C35A9B0512D1114B18688E
:105AF000B4235B00C35A9B0500D060E7164B984760
:105B0000164B98470DB03CBC90469946A246AB4612
:105B1000F0BD00230793EFE500220A4B1A60B4237F
:105B20005B00C35A9B05E9D000230793E4E5C04618
:105B3000D9530000F8260020910E010075290100BC
:105B4000150F0100FC260020750E010059530000BE
:105B5000810D010045250100ED2401007D0B0100B0
:105B600010B50421014B984710BDC04675290100AE
:105B700010B50821014B984710BDC046752901009A
:105B800070B582B004000D000679002E25D00068A3
:105B9000036899420CD0031D721ED2B201329200EA
:105BA00082189A4219D00433191F0968A942F8D102
:105BB000012E14D0711E8900214B98470600214BFD
:105BC0009847002815D0002E21D0217900220023EB
:105BD00000292BD101392171266002B070BD1A4B0A
:105BE00098470023236023716379012293436371F3
:105BF000F3E7164B00938222520015490330154CEF
:105C0000A04732000023144814498847FEE7144B8C
:105C100000930E4B832252000D4902200D4CA047E9
:105C2000DBE70133DBB221799942D3D999002068AF
:105C300009588D42F5D0900081510132D2B2F0E77F
:105C4000FD260100AD170000C9230100445E0200DB
:105C5000585F02005921010054580200B517000096
:105C60008C5F020070B582B005000C00002830D0B7
:105C7000274B98472B79002B2DD10420254B984793
:105C800006003000244B984700282BD0002E36D039
:105C90006B795908012211401A4200D001312A794A
:105CA000914210D21D4BD3189B00F3181C481018BA
:105CB000013A521AD2B2821A9200B2181868586089
:105CC000043B9342FAD189008C512B7901332B711B
:105CD0002E6002B070BD013399002868114B9847BF
:105CE0000600CEE7104B0093D02210490330104C31
:105CF000A047320000230F480F498847FEE70F4BAB
:105D00000093094BD22209490220094CA047E0E741
:105D1000815B0000DD220100AD170000FFFFFF3FA7
:105D2000FEFFFF3FFD260100285E0200585F0200D3
:105D30005921010054580200B5170000E85E020026
:105D400030B583B005004279D30710D50623134040
:105D5000063B5A425341DBB20279002A33D09A42C1
:105D600033D902689B009C58200003B030BD04204A
:105D7000174B98470400174B984700280DD0002C6C
:105D800018D02000144B984721002800134B984747
:105D90006B79012213436B71E6E7114B0093114AB3
:105DA00011490330114DA847220000231048114922
:105DB0008847FEE7104B0093094B104A0A4902201E
:105DC0000A4DA847D0E70024CEE70024CCE7C04620
:105DD000DD220100AD170000615B0000655C000082
:105DE000D05E020035040000585F02005921010016
:105DF00054580200B5170000C85F020037040000C5
:105E000010B504000068024B98470023236010BDC2
:105E1000C923010010B50168002919D00B78FF2BA8
:105E200012D000200F2403E0901C0B5CFF2B0CD041
:105E30002340821C082BF7DD821C0B2BF4DD021D96
:105E40000D2BF1DC421CEFE70020023080B210BDC8
:105E50000020FCE770B506000C1E0DD00B68002B6F
:105E60000AD00800054B98470500054B984730605D
:105E700021682A00034B984770BDC046155E00009C
:105E8000DD22010045250100F0B5DE4657464E46AD
:105E90004546E0B585B0061E039100D17BE0006861
:105EA000002800D17BE0CCB20B0A9846191C03787D
:105EB000FF2B4ED0012252420292934600227F25B0
:105EC000AA464906490E8C46703DC146B0461CE0C4
:105ED000811849784F464F4056463E420DD04906FC
:105EE000490E01910F006646B74310D159450EDDAA
:105EF00009B28B4611B2029109E04346C8461E0022
:105F000015E08A1C835CFF2B0DD09C42E0D02B4017
:105F1000911C082BF5DD911C0B2BF2DD111D0D2BB7
:105F2000EFDC511CEDE74346C8461E00029A002AEA
:105F300033DB14008018437842465A401300002097
:105F40005B060AD005B03CBC90469946A246AB46DB
:105F5000F0BD01235B420293E8E73000114B984704
:105F60000F23039A134004210B2B03DD01390D2B62
:105F700000DD03310D00411A8C4206D233685A19F4
:105F8000125D1A5501348C42F8D13068064B98479F
:105F900030600120D6E70020D4E70020D2E70020BF
:105FA000D0E7C046155E0000FD260100F0B5DE46D4
:105FB00057464E464546E0B589B006000E2302A876
:105FC00084466344198005AB1A803468002C58D08D
:105FD000CDB20B0A9A46191C2378FF2B4DD0012213
:105FE00052429046944600227F2083464906490E3D
:105FF0008946703804961AE0A118497856464E40F2
:106000005F4637420DD04906490E03910E004F46B8
:10601000BE430ED161450CDD09B28C4611B28846F3
:1060200007E0049E13E08A1CA35CFF2B0DD09D4269
:10603000E2D00340911C082BF5DD911C0B2BF2DD07
:10604000111D0D2BEFDC511CEDE7049E4246002A8A
:1060500017DBA3185B7855465D406B0611D1023201
:10606000A41805AB1A7822705B78637009B03CBC49
:1060700090469946A246AB46F0BD01235B42984646
:10608000E4E7FF22162302A98C4663441A803000FD
:10609000204B9847002800D10230043085B22900F7
:1060A00020001D4B984730601C4B9847002822D099
:1060B000002EDBD0AB1F3268944663440E2202A947
:1060C0008C4662441178197052785A702B1F3268CE
:1060D0009446634405AA1178197052785A70023DAB
:1060E00033685D19162302AA944663441A782A700D
:1060F0005B786B70BAE70A4B0093C32252000949E0
:106100000330094CA04732680023084808498847F3
:10611000FEE7C046155E0000FD260100AD17000039
:10612000605E0200585F02005921010054580200CD
:10613000B5170000F0B5DE4657464E464546E0B579
:1061400089B0060005AB1A800E2302AA9446634468
:1061500019800468002C58D0CDB20B0A9A46191C3D
:106160002378FF2B4DD001225242904694460022C4
:106170007F2083464906490E8946703804961AE006
:10618000A118497856464E405F4637420DD0490621
:10619000490E03910E004F46BE430ED161450CDD02
:1061A00009B28C4611B2884607E0049E13E08A1CAF
:1061B000A35CFF2B0DD09D42E2D00340911C082B25
:1061C000F5DD911C0B2BF2DD111D0D2BEFDC511CAD
:1061D000EDE7049E4246002A17DBA3185B7855467C
:1061E0005D406B0611D10232A41805AB1A782270FB
:1061F0005B78637009B03CBC90469946A246AB46BA
:10620000F0BD01235B429846E4E7FF22162302A972
:106210008C4663441A803000204B9847002800D1F8
:106220000230043085B2290020001D4B98473060B1
:106230001C4B9847002822D0002EDBD0AB1F3268C1
:10624000944663440E2202A98C4662441178197068
:1062500052785A702B1F32689446634405AA11780D
:10626000197052785A70023D33685D19162302AADC
:10627000944663441A782A705B786B70BAE70A4BCD
:106280000093B622FF3209490330094CA047326817
:106290000023084808498847FEE7C046155E00000D
:1062A000FD260100AD170000745E0200585F020079
:1062B0005921010054580200B5170000F0B5DE4620
:1062C00057464E464546E0B589B0060003920E2378
:1062D00002AA9446634419800468002C55D0C8B2C1
:1062E0000B0A9A46191C2378FF2B4AD001225242EE
:1062F0009046944600227F25AB464906490E8946C2
:10630000703D04961AE0A118497856464E405F4603
:1063100037420DD04906490E02910E004F46BE434A
:106320000ED161450CDD09B28C4611B2884607E0FA
:10633000049E13E08A1CA35CFF2B0DD09842E2D090
:106340002B40911C082BF5DD911C0B2BF2DD111D50
:106350000D2BEFDC511CEDE7049E4246002A14DBB6
:10636000A3185B785046584043060ED1A2186B46DE
:106370001B7B937009B03CBC90469946A246AB4645
:10638000F0BD01235B429846E7E7FF22162302A9EE
:106390008C4663441A8030001D4B9847002800D17A
:1063A0000230033085B2290020001A4B9847306034
:1063B000194B984700281DD0002EDBD06B1F326888
:1063C000944663440E2202A98C46624411781970E7
:1063D00052785A7033685B19033B6A46127B1A7015
:1063E000023D33685D19162363441A782A705B787E
:1063F0006B70BFE7094B0093F2225200084903304B
:10640000084CA04732680023074808498847FEE740
:10641000155E0000FD260100AD170000885E020039
:10642000585F02005921010054580200B5170000BE
:10643000F0B5DE4657464E464546E0B589B0060003
:1064400004920E2302AA9446634419800468002C27
:106450005CD0CDB20B0A9A46181C2378FF2B51D082
:10646000012252429046944600227F218B464006EC
:10647000410E89460F2103961AE0A018407856462F
:1064800046405F4637420DD04006400E029006005F
:106490004F46BE430ED160450CDD00B2844610B2BB
:1064A000804607E0039E13E0821CA35CFF2B0DD007
:1064B0009D42E2D00B40901C082BF5DD901C0B2B6D
:1064C000F2DD101D0D2BEFDC501CEDE7039E424664
:1064D000002A1BDBA3185B7855465D406B0615D17F
:1064E0000232A41804AB1A7822705A7862709A7833
:1064F000A270DB78E37009B03CBC90469946A24696
:10650000AB46F0BD01235B429846E0E7FF2216232D
:1065100002A98C4663441A803000224B9847002819
:1065200000D10230063085B2290020001E4B98476A
:1065300030601E4B9847002827D0002EDBD02B0060
:10654000083B3268944663440E2202A98C4662449A
:106550001178197052785A70AB1F326894466344B0
:1065600004AA117819705178597091789970D2787D
:10657000DA70023D33685D19162302AA944663441B
:106580001A782A705B786B70B5E7094B0093094A5B
:1065900009490330094CA0473268002308480949DB
:1065A0008847FEE7155E0000FD260100AD170000DC
:1065B0009C5E020013020000585F02005921010096
:1065C00054580200B5170000F0B5DE4657464E4657
:1065D0004546E0B585B08146039200285BD005684A
:1065E000002D5BD0CEB2090A081C2B78FF2B4ED0B1
:1065F000012252420292934600227F24A246400684
:10660000400E84460F2788461AE0A8184078444672
:106610004440514621420DD04006400E01900400F6
:1066200061468C430ED158450CDD01B28B4611B248
:10663000029107E0414613E0821CAB5CFF2B0DD0BA
:106640009E42E2D03B40901C082BF5DD901C0B2BAA
:10665000F2DD101D0D2BEFDC501CEDE74146029AD8
:10666000002A1EDB931CED182B78039803706B78BF
:1066700043704B461B689A1850784906490E0840EB
:1066800005B03CBC90469946A246AB46F0BD0123FE
:106690005B420293E3E701204042F1E701204042E0
:1066A000EEE701204042EBE7F0B5DE4657464E46A6
:1066B0004546E0B585B081460392002858D005686C
:1066C000002D58D0CEB2090A081C2B78FF2B4BD0D6
:1066D000012252420292934600227F24A2464006A3
:1066E000400E84460F2788461AE0A8184078444692
:1066F0004440514621420DD04006400E0190040016
:1067000061468C430ED158450CDD01B28B4611B267
:10671000029107E0414613E0821CAB5CFF2B0DD0D9
:106720009E42E2D03B40901C082BF5DD901C0B2BC9
:10673000F2DD101D0D2BEFDC501CEDE74146029AF7
:10674000002A1BDBAD18AB78039803704B461B681F
:106750009A1850784906490E084005B03CBC90464E
:106760009946A246AB46F0BD01235B420293E6E7A1
:1067700001204042F1E701204042EEE70120404283
:10678000EBE7F0B5DE4657464E464546E0B585B0E8
:106790008146039200285BD00568002D5BD0CEB205
:1067A000090A081C2B78FF2B4ED00122524202927C
:1067B000934600227F24A2464006400E84460F27BF
:1067C00088461AE0A8184078444644405146214281
:1067D0000DD04006400E0190040061468C430ED15E
:1067E00058450CDD01B28B4611B2029107E04146DB
:1067F00013E0821CAB5CFF2B0DD09E42E2D03B40ED
:10680000901C082BF5DD901C0B2BF2DD101D0D2BC1
:10681000EFDC501CEDE74146029A002A1EDB931C78
:10682000ED182B78039803706B7843704B461B6808
:106830009A1850784906490E084005B03CBC90466D
:106840009946A246AB46F0BD01235B420293E3E7C3
:1068500001204042F1E701204042EEE701204042A2
:10686000EBE7F0B5DE4657464E464546E0B585B007
:106870008146934600285FD00668002E5FD0CFB2D5
:106880000A0A111C3378FF2B52D00120404203909A
:1068900002900024803082464906490E8C460F2122
:1068A00090461BE032195078424642405546154208
:1068B0000ED04006400E01900500624695430FD170
:1068C000029A90420CDD02B2029222B2039207E0D9
:1068D000424613E0941C335DFF2B0DD09F42E1D064
:1068E0000B40A21C082BF5DDA21C0B2BF2DD221D98
:1068F0000D2BEFDC621CEDE74246039C002C21DBF4
:1069000020000234361900235C46F15CE154013367
:10691000042BFAD14B461B681B1858785206520EAE
:10692000104005B03CBC90469946A246AB46F0BD2F
:1069300001235B420393E0E701204042F1E701209D
:106940004042EEE701204042EBE74379DA0707D502
:106950009B0702D403681868704703685868FBE710
:106960000020F9E743799B0702D503681868704750
:106970000020FCE770B5041E26D04379DB0708D55C
:10698000144B9847051E04D0134B98472800134B0F
:10699000984763799B0709D52000114B9847051E3E
:1069A00004D00D4B984728000C4B98472379002BB7
:1069B0000BD10023236023716379012293430132B9
:1069C000934302329343637170BD2068034B984731
:1069D000EFE7C0464B690000015E0000C9230100DB
:1069E0006569000070B505000C002B4B98472368C3
:1069F000002B3ED06379DA071FD49B0710D520798E
:106A000001388000254B984728602279013A92008E
:106A10002368191D224B98472379013B2B7128E0ED
:106A2000207980001D4B98472860227992002168C8
:106A30001B4B984723792B711BE09B071AD52079B4
:106A400002388000154B984728602279023A92005C
:106A500021680831124B98472379023B2B7128009B
:106A6000104DA84706002000A847010030000E4B3B
:106A7000984770BD207901388000084B98472860FE
:106A80002279013A92002368191D054B9847237912
:106A9000013B2B71E3E7C04675690000DD22010070
:106AA00045250100415D0000555E000030B583B012
:106AB000050043799B0705D51C4B9847040020002F
:106AC00003B030BD04201A4B98470400194B984777
:106AD000002815D0002C20D02000174B984721000B
:106AE0002800164B98476B79022213436B71DB0722
:106AF000E5D52B681A68596819602B685A60DEE77B
:106B00000F4B00930F4A10490330104DA847220045
:106B100000230F480F498847FEE70F4B0093084BAF
:106B20000E4A09490220094DA847C8E765690000D7
:106B3000DD220100AD170000615B0000655C000014
:106B4000B05E0200CD020000585F02005921010032
:106B500054580200B5170000185F0200CF02000071
:106B6000F0B5D6464F464646C0B584B0051E0191E5
:106B7000914658D00368002B57D00B0A9846002244
:106B800002ABDA800279002A42DD00240126764237
:106B900006239A46264F16E00131C9B219E002AB2E
:106BA00006331B884A461380012036E0B34205DDD8
:106BB00002AB06331B884A4613800600013424B218
:106BC0002A79944226DAE1B26B7950460340062BCB
:106BD000E2D00020002A04D0914202D289002B6822
:106BE000C85802AB9A1D0199B84703008045D6D01A
:106BF0006A799107DAD50028D8DB002CD6D1520764
:106C0000D4D402AB06331B884A461380012004E02B
:106C100001267642F04380B2C00B04B01CBC904603
:106C20009946A246F0BD0020F7E70020F5E7C046F0
:106C3000C9650000F0B5D6464F464646C0B584B09B
:106C4000051E0191914654D00368002B53D00B0AC6
:106C50009846002203AB1A800279002A3EDD002408
:106C60000126764206239A46244F14E00131C9B228
:106C700017E003AB1B884A461380012033E0B34280
:106C800004DD03AB1B884A4613800600013424B29E
:106C90002A79944224DAE1B26B7950460340062BFC
:106CA000E4D00020002A04D0914202D289002B684F
:106CB000C85803AA0199B84703008045D9D06A791A
:106CC0009107DCD50028DADB002CD8D15207D6D4C6
:106CD00003AB1B884A461380012004E0012676425C
:106CE000F04380B2C00B04B01CBC90469946A2464B
:106CF000F0BD0020F7E70020F5E7C04683670000FD
:106D0000F0B5D6464F464646C0B584B0051E019143
:106D1000914658D00368002B57D00B0A98460022A2
:106D200002ABDA710279002A42DD002401267642A4
:106D300006239A46264F16E00131C9B219E002AB8C
:106D400007331B784A461370012036E0B34205DD55
:106D500002AB07331B784A4613700600013424B295
:106D60002A79944226DAE1B26B7950460340062B29
:106D7000E2D00020002A04D0914202D289002B6880
:106D8000C85802ABDA1D0199B84703008045D6D038
:106D90006A799107DAD50028D8DB002CD6D15207C2
:106DA000D4D402AB07331B784A461370012004E0A9
:106DB00001267642F04380B2C00B04B01CBC904662
:106DC0009946A246F0BD0020F7E70020F5E7C0464F
:106DD000A9660000F0B5D6464F464646C0B584B019
:106DE00005000191170000284CD00368002B4BD000
:106DF0000B0A98460279002A39DD002401267642E2
:106E000006239A46214B994610E00131C9B213E09E
:106E1000039B3B6001202FE0B34202DD039B3B60FC
:106E20000600013424B22A79944222DAE1B26B7965
:106E300050460340062BE8D00020002A04D091429F
:106E400002D289002B68C85803AA0199C8470300D9
:106E50008045DDD06A799107DED50028DCDB002C87
:106E6000DAD15207D8D4039B3B60012004E001260D
:106E70007642F04380B2C00B04B01CBC90469946E9
:106E8000A246F0BD0020F7E70020F5E763680000A8
:106E9000F0B5051CCB06DB0E4F05BF0E0904C90E6D
:106EA000052A3DD92804C00E40181F2800D91F20EC
:106EB0001F240440A4466E05B60EF6193F2E00D9D5
:106EC0003F263F242640ED06ED0EED181F2D00D97C
:106ED0001F251F242C40FF2A27D0FF25AD1A54431D
:106EE0006B43E3181802C018C001C01800015643D4
:106EF0006F43F7193E02F619F601F619F600B60EC1
:106F00007601C00E63465A4369435218110289182C
:106F1000C9018A18D20DD2B2D20230431043F0BD5B
:106F20007801C90218430843F9E770016346DA02A1
:106F300020431043F3E7F0B5C64600B5051CC8066C
:106F4000C30E98464F05BF0E0904C90E052A41D944
:106F50002804C00E081AC343DB1718401F23034040
:106F60009C466E05B60EB81BC343DB1718403F2680
:106F70000640ED06ED0E43465D1BE843C017054095
:106F80001F242C40FF2A2BD0FF25AD1A5443404626
:106F90006843241820020019C0010019000156435B
:106FA0006F43F7193E02F619F601F619F600B60E10
:106FB0007601C00E63465A4369435218110289187C
:106FC000C9018A18D20DD2B2D2023043104304BC98
:106FD0009046F0BD7801C902034318000843F6E764
:106FE00076016346D80234432043F0E7F0B5DE462D
:106FF00057464E464546E0B593B004000D0069463D
:107000008A8206931CAB1F781DAB1B789B461EAB78
:107010001E785B46042B01D9002F06D113B03CBC6F
:1070200090469946A246AB46F0BDBF4B9847824674
:10703000BE4B98478046836804932A00210010A81D
:10704000BB4B98470028E9D043461A8A10AB1988F1
:10705000891A89B20B918C4608B20A901880404672
:10706000418A5D886D1A2DB25D809888801A80B241
:107070009880DA88521A12B29146DA80069A002A6B
:1070800018D053461B7ADB0714D4411C6346C91A37
:1070900009B200290EDD13009446614480240A9A47
:1070A00094461A78944292411A7001338B42F8D177
:1070B00063460A9353465B69002B00D18CE06B4614
:1070C0009E8A994B9847050043469B8A0133424666
:1070D000128A9B1A1BB20593012F46D010AA0023D7
:1070E000D15E069B5B1A9846938801335B1A1BB2EC
:1070F00008930221535E190007930623D35E994239
:1071000000DD8BE710AF01AB9A46B146464600233F
:10711000FC5E0422BB5E9C421BDC6B461C229B5E19
:107120009846069623B2069A125D59464A43120AB9
:10713000029252464946118042460092059A0499AD
:1071400028006E69B04701340422BB5E9C42E9DD31
:10715000069E089B9C466644079B01331A000793D2
:1071600006217B5E9A42D2DD58E710AB02215A5EBF
:10717000924606229B5E9A4500DD4FE710AC01ABBC
:107180009946B0460023E75E0422A35E9F421BDCC3
:1071900053461EB2424669460A83B0463BB25A463F
:1071A00002924A466946098B118042460092059A2E
:1071B000049928006E69B04701370422A35E9F42FC
:1071C000ECDD6B461B8B984601239C46E24406226D
:1071D000A35E9A45D6DD21E7002E01D000F027FC02
:1071E0006B469B8A6A4613844F4B9847040043467C
:1071F0009D8A01351B8AED1A2DB210A80023C15EAD
:10720000838801335B1A1BB20B930A930623C25E79
:107210000223C35E561CF61A36B20E960C936B43CD
:107220005B185B0004998C4663440793012F1ED0C2
:107230005B46FA2B00D927E10C9B934200DDEDE67B
:10724000079B1A886B46998A0B04DB0E05934B0546
:107250009B0E0893CB06DB0E9C466B000F9313002E
:107260000026002089B20E9102009946D0E35B46C9
:10727000FA2B24D9636A002B04D010A82D4B984711
:10728000F02812D86D0000240E9B002B00DCC5E610
:10729000294E079F0B9A6B46198C3800B0477F190F
:1072A00001340E9BA342F5DCB8E66B469A8A1A803D
:1072B000666A10AB2A0004992000B047AEE6236A44
:1072C000002B3DD010A81B4B9847F02838D90A9BBB
:1072D000002B09DD6B469E8A184B0B9A52009A18B8
:1072E0001E8002339342FBD110AB02229E5E062227
:1072F0009B5E9E4200DD91E66D00104B984610AFFC
:10730000AA465B4600930B9B42460799894620009C
:10731000256AA847CC46D444634607930136062223
:10732000BB5E9E42EDDD79E691550000750E0100D1
:107330000B140100EF130100311A01000027002097
:1073400000236A461383928AD306DB0E9C46131CE5
:107350001A005705BF0E1C04E40E5B466343180277
:10736000C018C001C018C00D1F23984618405A46C7
:107370007A4313029B18DB019A18D200930E9A46A7
:107380005946634659430B025B18DB015918C90D76
:10739000434619405B466A461382138A5C43059450
:1073A0005F43089764465C4309945B46DF43FFB242
:1073B0000E9B002B00DC31E66B000E93731C0D93CB
:1073C0000B9B5B000F9301230C93BFB21F263E3330
:1073D0000B93634B984607239946524648E02B7817
:1073E000B3430B432B70049B5B012F88424617402D
:1073F0003B432B80C7001B0A4A4613401F436F7054
:107400000234544526D025006B461B8B2788BB428F
:10741000E5D06B461F836078C00863465843059BE0
:107420009B465844000A30407A05920E63465A4300
:10743000089B9B465A44120A0B9B1A4004922178DF
:10744000C906C90E63465943099B9B465944090A1C
:107450003140C4E7049A6746079B0E9CA4466344E8
:1074600007930C9B01330C930D9C9C4200D1D5E5F6
:107470000A9B002BF0DD079B1C000F9DAA4653447E
:1074800004929A46BC46BEE70E9B002B00DCC5E585
:107490000B9B043B05936B000F93069B0993002302
:1074A0000D936B461A8C1704FB0E049353059B0E29
:1074B0009A46D306DB0E9B4613E26A46128C328054
:1074C00001340133984501DC00F0F1FB0236A207DC
:1074D0003FD020780028F3D0FF28EED0FF22151AE5
:1074E000049F47437178C90869437F183A02D2194B
:1074F000D201D219D20D49460A4006925746474357
:1075000031884905890E69437F183902C919C901B3
:10751000C919C9005F4678433778FA06D20E554339
:10752000451928024019C0014019C00D4A461040B3
:10753000974338433070890E48013188084D2940FF
:1075400001433180069AD2004905490F0A437270FF
:10755000B6E722000599994200DBADE35EE1C04643
:107560001FF8FFFF6946098C21806180A180E180BE
:107570000432043308340599994200DA49E111686C
:107580000029F5D00131EDD01578002D46D0FF2D22
:1075900000D12EE1FF21491B8C4604986843617895
:1075A000C90866467143401801020918C901091843
:1075B000C90D39408A4628000699484381462088EB
:1075C0004005800E70438144484600024844C00193
:1075D0004844C0005E4675432678B046F606F60E6F
:1075E000B146664649464E43B446AC4461460D0238
:1075F0006544ED016544ED0D3D404646BE433543CF
:107600002570800E45012088BE490840284320800F
:107610005146C9004005400F014361705578002D67
:107620004AD0FF2D00D1E8E0A11CFF20401B84467A
:10763000049868438946E178C90866467143401852
:1076400001020918C9010918C90D39400C91280017
:10765000069E7043824660884005800E66467043F1
:107660008244504600025044C0015044C0005E466F
:107670007543A678B046F606F60EB2466646514603
:107680004E43B446AC4461460D026544ED01654489
:10769000ED0D3D404646BE433543A570800E40018A
:1076A000658898490D40284360800C99C9004005C1
:1076B000400F0143484641709578002D4AD0FF2D78
:1076C00000D19EE0211DFF20401B844604986843A2
:1076D00089466179C9086646714340180102091854
:1076E000C9010918C90D39400C912800069E704344
:1076F0008246A0884005800E66467043824450460C
:1077000000025044C0015044C0005E4675432679D3
:10771000B046F606F60EB246664651464E43B446AD
:10772000AC4461460D026544ED016544ED0D3D40FC
:107730004646BE4335432571800E4001A5887149F8
:107740000D402843A0800C99C9004005400F01431B
:1077500048464170D578002D00D109E7FF2D54D05F
:10776000A11DFF20401B8446049868438946E179A7
:10777000C90866467143401801020918C901091871
:10778000C90D39400C912800069E70438246E0885E
:107790004005800E664670438244504600025044C5
:1077A000C0015044C0005E467543A679B046F60657
:1077B000F60EB246664651464E43B446AC44614668
:1077C0000D026544ED016544ED0D3D404646BE4366
:1077D0003543A571800E4001E5884A490D40284394
:1077E000E0800C99C9004005400F014348464170B4
:1077F000BEE66946098C218010E76946098C6180E4
:107800005AE76946098CA180A4E76946098CE180A2
:10781000AEE606998A460A99994250DD5E000799BC
:107820008C466644D21A90460A9A914606E06A4609
:10783000128C328001330236994540DD4246D05CDD
:107840000028F7D0FF28F2D0FF22141A049A4243EE
:107850007178C908614351180A025218D2015218AE
:10786000D20D1F273A4006925546454331884905B7
:10787000890E61436D1829024919C9014919C900C6
:107880005D4668433578EA06D20E54430419200257
:107890000019C0010019C00D07401F2085432F4368
:1078A0003770890E48013188164C214001433180E0
:1078B000069AD2004905490F0A437270BAE7079B3E
:1078C0000F9A944663440793099B0B9A944663442A
:1078D00009930D9B01330D930E9A9A4201DCFFF739
:1078E0009DFB0A9A002A00DCEEE1099B990700D172
:1078F000EDE1079E984600231F21894644469046A5
:10790000E7E5C0461FF8FFFF0D9EFF2A65D0FF2E5A
:1079100067D0FF239B1B4A78D20899465A43059BA0
:107920007343D21813029B18DB019B18DB0D1F2237
:107930001A4004920A885205920E4B465A43089BFD
:1079400073439A46524413029A4692445346DB01CB
:107950009A465244D20D0B78DB06DB0E9A464B4614
:10796000544663439A46634673439946CA44534612
:107970001B029946D1444B46DB019946D1444B4604
:10798000DB0D1F2423409946099BA3439A464B468F
:107990005446234399463F231A4052014B464446DE
:1079A00023401A43049BDB025205520D13436A46DF
:1079B00093849BB20A8891460B802A0001300231E1
:1079C000B84210D00578002DF8D0954205D0FF2D93
:1079D0009AD05E466E43360A99E70A884A4596D1A0
:1079E000EAE70E9BE6E707990F9880464144079126
:1079F00006990B988046414406910C990131080084
:107A00000C9110A90624095F884201DDFFF706FBEF
:107A10000A990029E7DD0799069804000B9DA846FE
:107A200044442700AB4CA0465C460D94CAE76B4625
:107A30009C8A012E4ED0022E41D1A74B09936B4652
:107A40009A8AD306DB0E0E9353059B0E0C931604F5
:107A5000F30E0D9343469B8A01334246128A9B1ACA
:107A600019B208954D436D00049B9C46AC44634697
:107A70000793012F31D001300B9BC01A03B29846F7
:107A8000069B0A9A9E1A079B1A88089B4B4501DDA4
:107A9000FFF7C4FA4B000A93100000210C9B5B0116
:107AA0009A4643460B93099B98460D9B99466B4615
:107AB0001C8234005B4606930E9B9B46E9E0874B95
:107AC0000093874B8422920086490220864CA0476F
:107AD000FFF7A4FA854B0993B1E700236A46938226
:107AE0005B460D9F7B431802C018C001C018C00D33
:107AF0001F2528405A460C9B5A4313029B18DB0152
:107B00009B18DB009A0E92465A460E9E7243130251
:107B10009B18DB019B18DB0D1D40089A4A4501DDCF
:107B2000FFF77CFA4A00914633001F221340984623
:107B30004A460B92B9466B461C832C005A460A9261
:107B40000C9B9B4650E02B781F229343049A1343CF
:107B50002B707A012B889C465E4B61460B40134389
:107B60002B80C2005B055B0F13436B700134023640
:107B700010AB04229B5E9C4224DC35006B469B8A42
:107B800032889342DFD011006B469A8206981F23F9
:107B90009843434618435B465B014E4F38401843B9
:107BA0004B46DB024005400D18436B4618830A9A8A
:107BB000099B9847C106CB0E04934705BF0E0004EE
:107BC000C00EC0E7049CBA46079B0B9A94466344D8
:107BD0000793089B01331A00089310AB06215B5EE4
:107BE0009A4201DDFFF71AFA10AB00229E5E3700C1
:107BF00004229B5E9E42E7DC7600079B9C4666441F
:107C000004943C005746B8E73A889446059A944550
:107C100024D115E01F23049898435B4618432D4B4D
:107C20001840534618434B46DB024005400D1843AD
:107C30006B4618823988C04780B2A15D3B880593A6
:107C400038800135023710AB04269B5F9D420CDC67
:107C50002E00635D002BF4D08B42D5D006990A002C
:107C6000F92BD7D85A43120AD4E7059A079B0A9DE5
:107C7000AC46634407930B9B9C466444089B0133CA
:107C80001D00089310AB06269B5F9D4201DDFFF7A8
:107C9000C5F910AB00255F5F3D0004269B5F9F4246
:107CA000E4DC7F00079B9C4667440592D0E72200F6
:107CB0000599994200DA02E65C0007998C46644413
:107CC0001F27514606915AE4099A0023F0E7099AC2
:107CD00000233FE41FF8FFFF376F00004C600200F5
:107CE000F85F02001460020059210100916E00004B
:107CF000F0B5DE4657464E464546E0B593B00C001B
:107D000007921D001CAB1F781DAB1B789B461EAB5A
:107D10001E785B46042B01D9002F06D113B03CBC62
:107D200090469946A246AB46F0BD0A00010010A855
:107D3000D74B98470028F1D0D64B98478046D64B72
:107D40009847814683680593028A10AB1988891A7F
:107D500089B209918C4608B2824618804846418A09
:107D60005888401A80B20A9000B2089058809888CB
:107D7000801A80B29880DA88521A92B20B9212B2AC
:107D80000C92DA80002D14D043461B7ADB0710D406
:107D9000411C6346C91A09B200290ADD2B00691883
:107DA000802294461A78944592411A7001338B428E
:107DB000F8D143465B69002B00D1C3E0B54B98472F
:107DC0000C904B4610229B5E98464B469B8A013393
:107DD00042469B1A1BB2069310A90023C85E0023DB
:107DE000E25EA38801339B1A1BB20226895F0991C8
:107DF0000226A45FA4464E461224365F6446A41BA6
:107E00000C1B5C434646921BA41A6400079A9446D6
:107E1000A44462460892012F53D02A1A904610AA11
:107E20000624125F099C944200DD77E710AA04241F
:107E3000125F5B000A93099110AB079301AB9A465E
:107E40000132131A1BB20B930C9E079A13000025E4
:107E50005D5F2C00130004229B5E9D421FDC6D00C1
:107E6000089B9C4665446B4624229B5E994623B240
:107E70004246125D59464A43120A02922A885146E6
:107E80000A804A460092069A059930007769B847F9
:107E900001340235079B04229B5E9C42E7DD0B9B6D
:107EA0009C46E044089B0A9A944663440893099BC5
:107EB00001331A000993079B06215B5E9A42C4DDD9
:107EC0002CE710AA0620125E8A4200DA26E75B0041
:107ED00009938A4610AB079301AB99460C9E079A0B
:107EE00013000027DF5F3C00130004229B5E9F42CB
:107EF0001ADC7F00089B9C46674453461BB2984699
:107F000023B25A4602923A8849460A804246009273
:107F1000069A059930007569A84701340237079B16
:107F200004229B5E9C42EBDD089B099A94466344C5
:107F3000089301239C46E244079B06229B5E9A45D8
:107F4000CDDDEBE6002E01D000F0FDFB4B4610220C
:107F50009B5E1A004B469B8A01330D929B1A1BB203
:107F600098460130099BC01A03B20C9306930B98F4
:107F700001300A9BC01A03B20B930023E25EA6886D
:107F80000136B61A36B20898030041464B435344B3
:107F90005B0005998C469C44634608930221635E0E
:107FA00049461224095F5B1AC31A73430D99521A8A
:107FB00051468A1A9B185B00079A94469C44634674
:107FC0000993344B98470400012F15D05B46FA2BD8
:107FD00000D9EBE00B9B002B00DC9FE643465B00E7
:107FE0000E9373000F93A94600230D931F339846F9
:107FF0005B4607930A939AE3036A002B2AD010A8E2
:10800000264B9847F02825D910AB02229F5E062206
:108010009B5E9F4200DD81E643465B00984676000A
:1080200010AB05935B4600930C9B099A9246089906
:1080300089462000256AA8474B4643440893D44606
:10804000B444634609930137059B06229B5E9F4219
:10805000E8DD63E65B46FA2B24D80B9B002B00DCA3
:108060005CE643465B000A9373000D930C9B5B0038
:108070000C9300230793FF275B46FF1A1F239C46A0
:1080800020339946064B9A46B8465F463BE0C046C9
:108090000B14010091550000750E0100EF13010053
:1080A0001FF8FFFF0B9B002B00DC37E60C9B5C00EE
:1080B00043465B00984676000025804F2200099BCE
:1080C0009A461900089B99461800B8474B46434406
:1080D0000893D446B4446346099301350B9BAB42E5
:1080E000ECDC1BE6089B0A9A93465B440893099BC9
:1080F0000D9A93465B440993079B013307930B9AB0
:108100009A4200DC0AE6069B002BEBDD099B1E0071
:10811000089D0C9A93465B449B4641467378DB0866
:108120007B436A78D2084A439A1813029B18DB01F2
:108130009B18DB0D62461340059332885205920E60
:108140007A432C886405A40E4C4314192202121998
:10815000D2011219D20D3478E406E40E7C4328785B
:108160008046C006C00E4843201804022418E401CB
:108170002418E40D60460440404663469843044397
:108180002C704B461A4054012A8853461A40224309
:108190002A80059BDB00120A0720024013436B7004
:1081A000023602355E45B9D188469BE70C9B043BFD
:1081B00007930B9B002B00DCB0E543465B000E935E
:1081C00073000F930A9500230D931F339B46069B64
:1081D0009946B8E303880B8001370136059BB3420B
:1081E00000DC93E30230023103231F4253D03D7879
:1081F000002DF1D0FF2DEDD0FF235B1B9946437876
:10820000DB086B434A78D2084C4662439A18130243
:108210009B18DB019B18DB0D5A461340069302881E
:108220005205920E6A4394460A885205920E6243A2
:1082300062441402A44694446446E401A4466244A1
:10824000D20D0478E406E40E65430C78A446E406F7
:10825000E40EA0464C4643465C43A046A844434631
:108260001D024544ED014544ED0D5B461D4064464D
:108270009C4325430D703F231A4055010A885346FD
:108280001A402A430A80069BDB00120A0724224078
:1082900013434B70A0E7059B9946079BB34200DC54
:1082A00021E37000099B1C18089B9C466044044B0A
:1082B0009A464B460693059616E0C04645250100B2
:1082C0001FF8FFFF2388038063884380A38883808F
:1082D000E388C3800437059A0432059208340830D5
:1082E000079B934200DC4BE13B68002BF2D001334B
:1082F000E8D03978002949D0FF2900D134E1FF23A3
:108300005D1A6278D20813004B434278D2086A4360
:108310009A1813029B18DB019B18DB0D5A46134079
:1083200022885205920E4A43944602885205920EC4
:108330006A4362441602B44694446646F601B44663
:108340006244D20D2678F606F60E71430678B446DE
:10835000F606F60E75434D1929024919C901491946
:10836000C90D5D46294065465E46B5432943017007
:108370003F210A405101028855462A400A430280A3
:10838000DB00120A07210A40134343707978002961
:108390004BD0FF2900D1EAE0831CFF22551AE27876
:1083A000D2084A439846C378DB086B43D2181302BD
:1083B0009B18DB019B18DB0D5A461340628852055F
:1083C000920E4A43944642885205920E6A43624492
:1083D0001602B44694446646F601B4466244D20D91
:1083E000A678F606F60E71438678B446F606F60EC3
:1083F00075434D1929024919C9014919C90D5D462D
:10840000294065465E46B543294381703F210A40B5
:108410005101428855462A400A434280DB00120A35
:1084200007210A40134342465370B97800294BD0C4
:10843000FF2900D19EE0031DFF22551A6279D20860
:108440004A4398464379DB086B43D21813029B18C2
:10845000DB019B18DB0D5A461340A2885205920E91
:108460004A43944682885205920E6A436244160239
:10847000B44694446646F601B4466244D20D267969
:10848000F606F60E71430679B446F606F60E754307
:108490004D1929024919C9014919C90D5D462940DB
:1084A00065465E46B543294301713F210A405101AB
:1084B000828855462A400A438280DB00120A07213F
:1084C0000A40134342465370F978002900D101E76E
:1084D000FF2952D0831DFF22551AE279D2084A4360
:1084E0009846C379DB086B43D21813029B18DB0153
:1084F0009B18DB0D5A461340E2885205920E4A4300
:108500009446C2885205920E6A4362441602B446EB
:1085100094446646F601B4466244D20DA679F60646
:10852000F60E71438679B446F606F60E75434D197C
:1085300029024919C9014919C90D5D4629406546F5
:108540005E46B543294381713F210A405101C288EB
:1085500055462A400A43C280DB00120A07210A401E
:10856000134342465370B5E6238803800EE76388C1
:1085700043805AE7A3888380A6E7E388C380A9E6FF
:10858000069B99461600934200DCC5E13B0077004C
:10859000099A9046B844089A944667449B1B0593F1
:1085A000D24B9A4607239C46444607E023883B80EB
:1085B000013602340237B14500DCADE1059B995D1F
:1085C0000029F5D0FF29F1D0FF23581A6278D2088C
:1085D0004A4315007A78D2084243AD182B025B1942
:1085E000DB015B19DB0D5A461340069325886D05A8
:1085F000AD0E4D433A885205920E4243AD182A0201
:108600005219D2015219D20D2578ED06ED0E6943AB
:108610003D78EB06DB0E5843081801020918C90122
:108620000918C90D5B4619409D43294339703F2302
:108630001A4051013A8853461A400A433A80069B31
:10864000DB00120A61460A4013437B70B0E7FF2348
:108650001D1A4B78DB0843437278D2086A439A1894
:1086600013029B18DB019B18DB0D42461340059358
:108670000A885205920E4243914632885205920E64
:108680006A434A441302994691444B46DB0199469A
:108690004A44D20D0B78DB06DB0E43439946337810
:1086A0009C46DB06DB0E5D43A9444B461D024D4450
:1086B000ED014D44ED0D43461D4063464046834366
:1086C0001D4335703F231A4055013288874B1A40AD
:1086D0002A433280059BDB00120A584602401343AE
:1086E0007370013702310236069BBB4209DDE55D3E
:1086F000002DF6D00798F92DA9D80A9B5D43280ACA
:10870000A5E7A146089B0E9A9446634408930C9BE8
:108710009C46E144099B0F9A9446634409930D9B40
:1087200001330D930B9A9A4201DCFFF7F7FA069B8F
:10873000002BE7DD099B9C46089E002707239B46EC
:1087400061464C46D3E7012E55D0022E49D1684BE5
:108750000A934B4610229B5E1A000B934B469B8A52
:1087600001339B1A1BB29C460023E25E0D92A38844
:1087700001339B1A19B2089E624672435300059A50
:1087800090469844434606930222A35E4A4612242A
:10879000145F1B1BF31A4B435B00079AD418012F7D
:1087A0002CD05346EB1A1A0053465B00E31A994645
:1087B000089B0C9CA34201DDFFF7B0FA63465B0007
:1087C00098464B00079310AF5B4605930130099B19
:1087D000C01A03B209930A9B9A4643460A939046ED
:1087E00072E0444B0093444B444A45490220454CB7
:1087F000A047FFF793FA444B0A93AAE70B9B0D9A05
:108800009B1A5B00A14699440C9A964201DDFFF742
:1088100085FA63465B009A464B00984610AF5B466C
:108820000593D3460A9B9A460023FD5E2E00042240
:10883000BB5E9D420FDC6D00069B5C194D44218898
:108840002888059AD0472080013602340235042258
:10885000BB5E9E42F3DD069B5B440693C144089BCE
:1088600001331A00089306217B5E9A42DCDDFFF794
:1088700055FA31882888D0473080013402360235D5
:108880000422BB5E9C420ADC43461B5D002BF4D0F5
:10889000059AF92BEDD85A4653431A0AE9E7069B85
:1088A0000A9A944663440693099B9C46E044079BBE
:1088B0009C46E144089B01331A00089306217B5E25
:1088C0009A4201DDFFF72AFA0023FD5E2C00042204
:1088D000BB5E9D42E3DC6D00069B5E194D44D3E711
:1088E0000A9F0026D9E43B0051E6C0461FF8FFFF6F
:1088F000376F00004C600200086002005303000064
:108900001460020059210100916E0000059B9946F8
:10891000079B9E4200DAC4E4089B0E9A9446634487
:1089200008930A9B0C9A944663440A93099B0F9AF6
:108930009446634409930D9B01330D930B9A9A421D
:1089400001DCFFF7EBF94B46002B0FDD0A9B0322FE
:108950001342C5D0099A9046089A1F000026054B7D
:108960009A464B4605934046110040E40A9F002674
:10897000CEE7C0461FF8FFFFF0B5DE4657464E462D
:108980004546E0B5BFB01C900800249190460A937C
:1089900048AB1B780B9349AB1B78079300233CA98A
:1089A000C25C5A540133082BFAD1B74B9847B74BE6
:1089B00098471990048A3CAB1A88121B1A80408A87
:1089C0005A88121A5A809988091B9980DA88121AD3
:1089D000DA80AF4B98471A90002808D10A9A53883A
:1089E000002B04D10133FF3312899A4272D0079BC6
:1089F0005A1E9341023399461C9B0022995E8C4675
:108A00009F8801377F1A3FB23CA902228D5E199AD6
:108A10001226945FCA4600200E5E1020125E0220CD
:108A20001B5E1B1BEB1A7B436046801A301AC01872
:108A30004B465843030043441593B6B2B21892B262
:108A400028A802808B8801339B1B9BB21EB217960D
:108A5000013BD3188380ADB22C1924B24480C4806A
:108A6000CB8801335D1B2DB20A984388002B00D0C0
:108A700044E30289531EFF3B591E8B41DBB29B46E8
:108A80001A9B002B00D0D5E00133FF339A4200D06F
:108A90003AE30B9B002B05D1837A002B02D1079B75
:108AA000002B34D13CA87B4B9847F0235B009842C5
:108AB00000D8CAE0F0208000774CA0471B90F02639
:108AC00076003000A047189048212AA8734B984799
:108AD0001D9655E30B9B002B89D1079B002B13D1CF
:108AE0000A9B9B7A02229146002B85D10A9A937B9E
:108AF00002931378019301230093002342461C99AB
:108B00002498674CA047DDE20323994674E73CA80C
:108B1000604B9847F0235B00984219D83CA85D4B06
:108B200098470790079E70005B4CA0470590300067
:108B3000A0470690002D61DD53467B439A466B1C8F
:108B40009B46012398460027179D3E004C4631E086
:108B5000F0235B000793E5E7013312190237AB42BC
:108B600009DA9178C1540029F6D056783602117886
:108B700089193980F0E76646179B9C466644159B29
:108B80005344159324AB64229B181B88013324AAF9
:108B90006021521812889B1A1BB29B19079A9A429D
:108BA00017D928AAD3880133D38001239C46E044F7
:108BB000D84523D0179B002BE1DD7700059B9C4611
:108BC0006744159A002306998C46B4446046B4461F
:108BD000C7E728AF0A9A937B029313780193022385
:108BE0000093069B059A390024982D4EB047FB88C8
:108BF00001331BB27B80FB800026D6E728AA062122
:108C0000535E0221525E9A420ED028A9013BCB80CE
:108C10000A9A937B02931378019302230093069B95
:108C2000059A24981E4CA04706981E4CA04705980C
:108C3000A04747E23CA8174B9847F0235B009842B7
:108C400003D9F0235B001D9303E03CA8114B984728
:108C50001D901D9E7000104CA0471B903000A04737
:108C6000189048212AA80D4B98475B46002B00D14D
:108C700086E260E2002314931293119397E21D9908
:108C80001898094B9847A9E291550000750E01000C
:108C90006DBB0000EF130100A12701007529010041
:108CA000F17C000065240100192A01000D9BF318D6
:108CB0001BB22AA908200A5E9B1A0A200A5E0E9897
:108CC000821A80204000C989814259D02AA90C20EB
:108CD000095E00296BD12AA9C88E43431D00339B2E
:108CE0009A46AA444243349BD3180C9353461B1212
:108CF00098462AAB04229B5E984500DBB0E04246D2
:108D0000002A00DAACE00C9A1212100016922AAA7D
:108D10000621525E904200DBA2E0002800DA9FE0CC
:108D200034222AA9895C4A076AD52A9A890758D425
:108D3000434343445B00D21810782AA9087552783F
:108D40004A75022134222AA8825CD2070FD51F223D
:108D500022989043FC22D20002435205520D6846ED
:108D60008825401902802AA8808A904278D02AAAB1
:108D7000D27C002A60D12AAB9A7D22709B8A80E047
:108D80003699359805000C91080058432900514345
:108D9000411AC9113398169082468A446B430C9845
:108DA00042439B18DB11349A9B180C939EE72AA927
:108DB000C88E43431D004243369858438046359839
:108DC00050434346181AC013339B9A468244359B3E
:108DD0006B43369850431B18DB13349A9B180C9343
:108DE00084E716994B4343445900CB18D2181078A6
:108DF0002AA908755078487592788A750321A1E7E9
:108E0000434619B26B4658229B1800229A5E24AB47
:108E10001B8D2692259130A8AE4DA84724AB98858E
:108E2000269A259930A8AC4B984724AB2E229B1844
:108E300018700023002185E72AA8524602876A4657
:108E4000128E4287424682876A46582552191288F6
:108E5000C28703644423C154A04B984700288AD199
:108E60000023237042E0FF2323707A7812023B78BC
:108E70009B189BB20B9A002A03D0994A12889A42F7
:108E80004AD00A9A927A002A2ED06A464C21521869
:108E90001288D90A94465143119A90464144C90414
:108EA000C90E5805800E62465043129A90464044BF
:108EB0008004DA06D20E63465A43149B9C466244F1
:108EC000D204D50E1F23089A9A4313002A001A438E
:108ED000800E4001834B13400343C9025B055B0DC9
:108EE0000B436A4613849BB2059A13800136069B96
:108EF0009C4667440134059B023305934E450EDAC8
:108F00005B46002B00D0D1E6079B002BABD0BB7893
:108F10002370002BEAD0A8E700232370E6E7179B15
:108F20000F9A944663441C001A9B002B48D1159B52
:108F30001F9A94466344159324AB64229B181B88A4
:108F4000013324AA6021521812889B1A1BB21B19E4
:108F50001D9A9A426CD928AAD3880133D3800F94E2
:108F6000109B01331093209A934200DB8FE0199BF2
:108F700010229B5E24AA602152180021525E9B1889
:108F80001C9A0021525E9B1A0D93179A9146002A53
:108F900014DD189B98460F9A9446E04453001B9AA0
:108FA00092469A44159F0026219B109A944663444A
:108FB0001BB20E93444653460593A1E70F9CB3E7BB
:108FC0000F9B189A944663441D0024AB60229B18A3
:108FD000198824AB04329B181B8801335B1A1BB21F
:108FE00024AA622012181288199E708A12181098EA
:108FF0008446624412B2308A091809B228003A4EF7
:10900000B047002803D0022891D11E908FE724ABEF
:1090100064229B181988013124AB043A9B181B88E1
:10902000C91A09B22800314B984702231E937EE7E4
:1090300028AC0A9EB37B0293337801931E9B009366
:10904000189B1B9A21002498294DA847E3880133D7
:109050001BB26380E38002231E93279B002B09D160
:109060007388002B06D13389013BFF3B5A1E934185
:1090700001331E9300230F931A9B002B00D16FE73F
:109080001D9918981B4B984700230F9368E728AA4F
:109090000621535E0221525E9A420ED028A9013B5E
:1090A000CB800A9A937B0293137801931E9B0093C3
:1090B000189B1B9A24980E4CA04718980E4CA0475A
:1090C0001B98A0473FB03CBC90469946A246AB4691
:1090D000F0BDC046D5E50000F5E60000FDEA000061
:1090E000726002001FF8FFFFD1BA0000752901006D
:1090F000F17C0000192A01006524010001239B4630
:109100001A9B002B00D095E53CA8414B9847F023D3
:109110005B00984200D898E5F02080003D4CA047C5
:109120001B90F02676003000A047189048212AA80E
:10913000394B98471D960522079B002B04D1013A15
:109140000B9B002B00D002322AA80A9C63888381E3
:109150002389C38143462A9387801C99CB88013396
:1091600049885B1AC3808274A3880381E3884381A2
:10917000A3890382E37BDB07DB0FC374274B98478C
:109180000A998B7ADA43D2B21392002B00D171E59F
:109190009BB24A7BD2085A4311928A895205920E99
:1091A0005A4312920A7BD206D20E5A4314920B9B58
:1091B000079A1343279302221E92002B0AD10A9A80
:1091C0005388002B06D11389013BFF3B5A1E934164
:1091D00001331E931A9B002B00D050E5199B1222DD
:1091E0009B5E3CAA0221525E9B181C9A0221525E91
:1091F0009B1A21932095002D00DC48E753467B43C2
:109200001F93002310930F934B460693AFE6C0467F
:10921000EF130100A127010075290100F9E7000003
:10922000F0B59FB005000E00170009AC20000B4BF5
:1092300098470B4B1B886380220031002800094BA4
:10924000984702A8084B9847002300933B0002AAC6
:1092500031002800054CA0471FB0F0BDCDBF000075
:10926000A060020071C00000ED9500003D96000076
:1092700010B5040010210A4B9847237B1F2293430B
:109280002373A389074A1340A38100236373FF3329
:10929000237001332381E37B01221343E37310BD69
:1092A000752901001FF8FFFF0438C3B20A2B0FD83D
:1092B0009800084B1B589F4610200AE0182008E031
:1092C000012006E0022004E0042002E0082000E083
:1092D0000020704774600200032805D002D30638CE
:1092E000042801D9002070470120FCE7052807D099
:1092F00003D8022804D00020704707380728FAD87E
:109300000120F9E7F0B5DE4657464E464546E0B542
:1093100091B0040003911E00002A09D01B78052B90
:1093200014D811B03CBC90469946A246AB46F0BD5D
:10933000814B0093814B4D3281490220814DA847DA
:10934000814A03992000814B9847EAE7B1891000D0
:109350007F4B9847071E00D1B0E0057BED06ED0E70
:1093600028007C4B98470490069028007A4B984739
:1093700005900790BB69002B0DD0784B0093784B7C
:10938000F7226F4902206F4DA847BA690399200060
:109390006E4B9847C5E73B69002B45D000230CA9CD
:1093A000E25C5A540133082BFAD17388002B04D1A4
:1093B000802252003189914223D01BB2E2880132CF
:1093C0006188521A12B2A18801312088091A09B2A3
:1093D0000CA80500301D01903089009006952800EA
:1093E000604DA847228806980388D31803806388B5
:1093F000418859184180818852188280C2889B1800
:10940000C3800CAA03990EA8574B9847002800D197
:1094100087E73A69059B0193049B009333000EA9EB
:109420002000524CA0477CE7220003990AA84E4B2B
:109430009847002800D174E70AAA9388013312885C
:109440009B1A1BB2059358009C466044484B9847B2
:10945000049000230CA80AA95A5C1A540133082B63
:10946000FAD101210CA8434B98470AAA0021535E68
:109470009C460020215E0220155E0223E05E281A31
:109480000623D25E954253DC374A934663465B1A05
:109490001BB208930994B246804623E0099C380029
:1094A000354B9847354B00932D4B9A225200244957
:1094B0000220244DA8470498314B9847274B00932E
:1094C0001E4B58221E4902201E4DA8471E4A0399D2
:1094D00020001E4B984724E701350AAB06229B5E0D
:1094E0009D4225DC0CAA03990EA8D8470028F3D08A
:1094F00043461AB2049B0093059B08993800214CFF
:10950000A0470128CAD10CAC079B0193069B00938E
:109510005346049A0EA92000144EB04763880133C5
:109520006380E3880133E38001239C46E044D3E772
:109530000498134B9847F4E6FC600200A460020014
:10954000C460020059210100146102002192000050
:1095500051EF0000D9920000ED9200001C61020062
:10956000B06002002DE900000B14010079890000B1
:10957000A1270100E51301005DFD0000306102003C
:109580006524010039FD0000002808D003781A0086
:10959000203A01205F2A01D9D809400070470320F2
:1095A000FCE700000300303BDBB21A00092B18D99E
:1095B000602801D92038C0B24138C3B2052B0DD87C
:1095C0009800094B1B589F460B220AE00C2208E02A
:1095D0000D2206E00E2204E00F2202E0002200E04D
:1095E0000A2210007047C0465061020010B5040006
:1095F0001C210F4B9847FF23237223781F2293438C
:10960000237022880B490A402280002363700A4B92
:10961000636001235B42E3812382A2781F231A4304
:10962000A27063880B4063800023E370A37510BDB4
:10963000752901001FF8FFFF30000020F0B5DE465D
:1096400057464E464546E0B5DBB011900F911700E6
:109650001A000E93649B07933B7A052B02D913786B
:10966000002B06D15BB03CBC90469946A246AB4667
:10967000F0BD7B6805930A000400010058A8CF4B99
:1096800098470028EED0FA7D910724D4A3880133AF
:1096900022889B1A1BB2059A0826965F0A217A5ED9
:1096A0009146B144119A0020115E24910220105E6F
:1096B00012217A5E21921422B95E421892B215B23A
:1096C000079C002C52D0002954D1002814DB13959C
:1096D000002206922EE00C217B5E3CAD0292B84A3D
:1096E00001920A217A5E00927A680E992800B54E9E
:1096F000B0470022AB5ECEE7A168081AC117401838
:109700004840802189004C46091B4900884207DDFA
:109710000122524207990A6013950022069209E03D
:1097200007980168002929DB069141688C4662444C
:1097300012B213921BB2190017930C23FA5E0E9B00
:109740001800069CA4466044FB7D00930B0005991D
:109750009D4DA847A44660449B4A92469B4A90462A
:1097600008960600139DBB46079F11E01395002243
:109770000692DFE7139500220692DBE7139500229D
:109780000692D7E706962378002B00D16AE70600F9
:10979000089BEB180F9A0221525E934220DA0E9B2F
:1097A0009C195B460C229A5E5B46DB7D0093179BFF
:1097B00005992000D04780194D442DB2002FE1D0EB
:1097C0004545DFDB3B68002BDCDA3E60119A022165
:1097D000535EEB1A7B60130002229B5EBB60D1E7F5
:1097E0000B9613955F46FA7D53072ED4130748D482
:1097F0003B7A1093FB891E003A8A9246534501D961
:1098000056469A463B7E9B0755D13FAC2000704B95
:1098100098477B886380109BFA2B01D96D4B1B788E
:10982000DBB21E934B466A469383938B1F936B4622
:109830004C229B181B881893249D00232093B0462C
:1098400053460C933E0000F00EFE0C217B5E069CFE
:10985000311B89B20E98A44660440092059A5E4C72
:10986000A047119A9388013312889B1A1BB2181AC9
:10987000C30F1B185B10249A944663441BB22493B5
:10988000B6E70C217B5E0B98069C011B89B20E98F3
:10989000A44660440092059A4F4CA047119A9388C1
:1098A000013312889B1A1BB21B1A249A94466344F4
:1098B0001BB224939CE755AC2000484B98473B884B
:1098C00023807B680820185E05300A21444B9847A6
:1098D00060803B7A23727A7E03231A40637A0321E5
:1098E0008B431343637290E70025C5E0089B002B70
:1098F00007D134AB80229B181B8820930123089347
:10990000A2E0089B012B01D100F02DFE022B01D11A
:1099100000F070FD4B461E88CFE0202C00D093E075
:10992000549B209A9B1A072B05D04B461B881993F2
:109930000223089388E00D9B94466344180000239B
:109940003CA9C25C5A540133062BFAD13CAD2878AD
:10995000244B9846984704006878C047240124188F
:10996000A878C0470600E878C0473601361828793D
:10997000C04782466879C04753461B011818C2B2D7
:10998000D2081F23349999430B001343F6B2B6084B
:109990007601154A13403343E4B2E408E4025B0560
:1099A0005B0D23436A46D021521813809BB2199352
:1099B0000223089348E0199E7FE0C0460B14010083
:1099C000187C00003D3F0100213C010000FCFFFF2E
:1099D000CDBF000068610200993E010089A500002A
:1099E000B9C10100A59500001FF8FFFF3CA8099A26
:1099F0000280139941804B469B89013B9446634406
:109A00000A9A9446634483801F9B013B8C466344BF
:109A1000C3803FAA0F997D4B98475FE07C4B009332
:109A20007C4B9822FF327C4902207C4CA047079B4C
:109A3000002B09DD4B469B89099A944663440A9A98
:109A4000944663441BB2099354990B9B069A9B1A44
:109A50008B4201D800F0D2FC714B9F4200D143E70A
:109A600000250C9A9A4207D0069B9C4661440E98AA
:109A70005B461B68984785B26A4E54A90D9B984671
:109A800018003368984704004346549A9446634448
:109A900018003368002198474B46DB7DDB0706D56D
:109AA000232C00D122E7089B012B00D135E74B4640
:109AB0001E88089B022B00D17DE70200210005983B
:109AC000594B98470A900790554B9F4206D00C99E6
:109AD000994203D0AF4201D8A94287D8109B042BEA
:109AE000A5D9059B002B99D04B465B7E159300238F
:109AF00022003CA905984D4DA84700280BD11F2CEA
:109B000095D94B4B0093434BA222FF32424902307E
:109B1000424CA0478BE73CAB9A88002A02D15B8875
:109B2000002B84D03CAB06215D5E09998C46290050
:109B300061445B8812918C4663440F980025415F15
:109B40008B4200DA73E701000423CB5E6146994241
:109B500000DD6CE7059908254B5F0A25495F5B1A14
:109B600013998C466344991A3CAB08255B5FCB1A6A
:109B700098464244010002200B5E9A4200DA56E702
:109B800006228B5E984500DD51E721000598294BA0
:109B900098471B90002823D0059B1B7B9B0700D177
:109BA00070E26B4648229B181B881BB214934346F5
:109BB0001BB216936B4644329B181E803CAB9B7ABB
:109BC0001E00032B00D10EE1022B3BD012D8012B3B
:109BD00000D00EE1012680232293174B259335E018
:109BE000164B00930B4BB822FF320B4902200B4C53
:109BF000A0471CE7042B00D1F6E0082B00D0F8E0CA
:109C00000826FF2322930E4B25931FE071C000000E
:109C1000F46202006C610200BC6202005921010082
:109C2000FFFF00005C00002091FE000089FE0000A4
:109C30001463020081FE0000A46102003C63020084
:109C4000BC610200C0232293D94B25933CAB5A88B8
:109C50001D929B881C93724392460F9B00229B5E31
:109C600000222D921499994203DA5B1A5A00D318F4
:109C70002D930F9B04241C5F03211D9D2800CD4BB9
:109C80009847149A944660441A95A04204DDA41A99
:109C9000013463001B191A930F9B02229B5E002262
:109CA0002B921699994201DA5B1A2B930F9B06228D
:109CB0009B5E1C990A00169CA44662442E919A420F
:109CC00002DD1B1B01332E936B468C229B181A88D6
:109CD000D306DB0E289353059B0E2A931304DB0E49
:109CE000299353462B9A53432D9A72439B18DC10A9
:109CF0001B9A9446644407221A4092461C9B1D9A64
:109D000053431A002F93F0235B009A4200DD2F93F8
:109D10002F9D2800A84B984726906800A64B98478F
:109D20002790A64B9847A64B984705001021425E06
:109D3000838A01331C929B1A1BB21B938168239167
:109D400003212D989B4B98472B0012255B5F169D96
:109D5000EB1A1B994B43149DAC4663441C9A9B1A07
:109D60002B9A4A4312189B185B0023998C469C44FB
:109D700061461C916B4648229B181D88281834A9FF
:109D8000088303211A988B4A9047013D451934AA4C
:109D900095832B9D2B0043441BB25383D383894B64
:109DA000984730902B002E9DAB4200DB4FE11A9973
:109DB0002D980A1A31921D9D6B1A8446634419002E
:109DC000714332910321494210007A4B98471B9B03
:109DD0009C4660444300339300232C9336974B46B4
:109DE0003793A146CBE00426F0232293764B2593AC
:109DF0002CE7764B0093764B764A77490220774CD6
:109E0000A04714E6082E0BD063461840259B1B5C28
:109E100006E0634603401E994B431B0A00E0002303
:109E200016998B540132032A21D014981B99884229
:109E30007BD23318F54001341A99A1427BD0149398
:109E40001299087828400821CB1A9B1BD840C3B22E
:109E5000002BE4D01E99FF29D4D0082ED9D0634618
:109E60001840259B1B5C1E994B431B0AD8E70F002B
:109E700008781C994B78DB086246121A5343299ADA
:109E800042439B181B0A1F221A402392BB78994613
:109E90000A78D206D20E63464F46DB1B5A43289BF4
:109EA0007B43D218120A1F231A40169B5B789846F0
:109EB0000B885B059B0E61464746C91B4B432A999D
:109EC00079438A4653441B0A3F210B409A46002897
:109ED00008D1002F06D14B46002B03D1269B1D999C
:109EE000585403E0269B1D99604658541D9948001C
:109EF000279FB846404407781F239F433A43027088
:109F000053465B010288364F3A4013430380239A3D
:109F1000D2001B0A07273B40134343704B1C1D9381
:109F20001C9B02331C9300227FE7129B0133129388
:109F3000229D00237FE7129A91469A46309B002B80
:109F400050D1319B1D998C4663442F9A9A4266D911
:109F50003AAAD3880133D3802C91329B5344DA1030
:109F6000914407221A4092461C9B339A94466344BC
:109F70001C932B9B01332B932E9A934264DA229DE0
:109F80005346DD402D9C1A9A94420DDA2C9B1D936A
:109F90000022FF239C4639AB169308239B1B1B937F
:109FA0004B46129353464AE72C9B1D93C6E7C04687
:109FB000A8610200B9C10100A1270100915500006C
:109FC000750E01006DBB0000AC6102006C63020005
:109FD000906102007A020000BC6202005921010077
:109FE0001FF8FFFF2C9B269A944663441C003AAA54
:109FF0000023D15E938801335B1A1BB20620125EE8
:10A000002000CF4DA84700289BD13AAB9988013159
:10A010001B88C91A09B22000CA4B984791E73AAC8D
:10A02000159B02931E9B019302230093269B279A64
:10A0300021000F98C44DA847E38801331BB2638009
:10A04000E38000232C9388E7369F379B99463AAAF2
:10A050000621535E0221525E9A420DD03AA9013B7D
:10A06000CB80159B02931E9B019302230093269B9A
:10A07000279A0F98B44CA0472698B44CA04727982D
:10A08000A047D4E46B4648229B181B881CB2434669
:10A090001BB29C466B465C329B181E803CAB9B7A85
:10A0A0009A46032B30D0022B17D009D8012B33D17D
:10A0B00001239A4602217F331493A54B1D9311E08F
:10A0C000042B23D0082B27D108239A46802149004E
:10A0D000F73314939F4B1D9304E00421C023149382
:10A0E0009D4B1D931E9AF92A3DD89C4B1B78934299
:10A0F0001CD0002200292BD01E9B99481697129D38
:10A100001F0012931D9E1BE004239A461021F0238A
:10A110001493944B1D93E5E7934B0093934BE622E6
:10A12000FF3293490220934CA04780E4924B1B6876
:10A130009A45DED10CE0129B135401328A4205D0BD
:10A14000B35CFF2BF7D07B431B0AF5E7169F1295F4
:10A15000824B6A467821521812781A70864B524602
:10A160001A607F4B1D933CAB5A88279299885046C2
:10A1700050430F9B00229B5E002216929C4201DA04
:10A180001B1B16930F9B04229B5E279D2A191C956F
:10A190009A4202DD1C1B631C1C930F9B02229B5ED8
:10A1A00000221A929C4502DA62469B1A1A930F9B70
:10A1B00006229A5E6346CB182391934203DD6346E1
:10A1C000D21A531C2393169B28931A9A5043544631
:10A1D0005C430019C6081B9B9C4666440724044048
:10A1E000279B4B431A002593F0235B009A4200DD26
:10A1F00025932598614B984722906B4648229B18DF
:10A200001D883AAB169AAA181A80013D1C998C46F3
:10A2100065449D801A98050045442AB25A80DA8028
:10A22000574B98472690082355465D1B279B169A47
:10A23000944663441C995B1A52465A4327921A98D3
:10A24000239B984200DBB8E000231B932A971D9BB9
:10A2500098461D954B462B9339E00023137012E06E
:10A260000136149900240132129B934210D03378A6
:10A270000B40281BC340D8B20028EED0484603400C
:10A280004046C35C1370A542EAD9E419F940EAE7F5
:10A29000BA461D956746269B002B33D11C9B169A08
:10A2A0009B1ADB19259A9A426CD93AAAD3880133B2
:10A2B000D3801B97279B9C466444E308F61807232A
:10A2C0001C401A9B01331A93239A934272DA149911
:10A2D000E140169B1A001C98824211DA229F3A0034
:10A2E0001B9DAC466244030028981B1A9C443B000B
:10A2F00063441800FF239946129057461D9DB6E708
:10A300001B9FC8E71B9B229A9446634499463AAA2E
:10A310000023D15E938801335B1A1BB20620125EC4
:10A320004846074DA8470028B8D13AAB9988013173
:10A330001B88C91A09B24846024B9847AEE7C04687
:10A34000D1BA000075290100F17C000065240100EC
:10A35000A4610200BC610200A8610200C42B0020BD
:10A36000C02A0020AC610200946302007C610200FC
:10A37000BC62020059210100C02B0020A12701006E
:10A380006DBB00003AAF159B0293FF230193FD3B89
:10A390000093229B6A46A4215218128839000F9814
:10A3A000734DA847FB8801331BB27B80FB800023E1
:10A3B0001B937FE72A9F2B9B99463AAA0621535E5F
:10A3C0000221525E9A4210D03AA9013BCB80159BE4
:10A3D0000293FF230193FD3B0093229B6A46A42036
:10A3E000121812880F98624CA0472298614B984728
:10A3F000FFF71DFB00230893FFF726FBB8464E46E8
:10A40000337E9B0747D4337EDB0765D40E9B1F004A
:10A410000B9DAC4667440C23F25EF37D0093179BC3
:10A4200005993800544CA0474419119B00255D5FE5
:10A43000F27D530770D4130700D582E0139B1F9958
:10A440008C466344189A624492B218920B9A069210
:10A450001BB21A0013930F9B06215B5E934201DA35
:10A46000FFF700F90B940E9B069A944663440D93F4
:10A470001B78002B01D1FFF7F5F8219B9C46654422
:10A480002BB209930023549308933C4B9B464746B9
:10A49000B146FFF7D9FA3AA86B4690229B181B8861
:10A4A0000380736808229B5EDA0FD218521055ABF6
:10A4B00002215C5EE10F09194910521818998C4667
:10A4C000624412B242803CA96C46A48C0C804A8043
:10A4D0000F9A2B4CA04796E73AA86B4690229B1800
:10A4E0001B880380716855AB02229C5EE20F121933
:10A4F000521001320C8912194989521A18998C4646
:10A50000624412B242803CA96C46A48C0C804A8002
:10A510000F9A1B4CA04779E70C21735E0092059AB5
:10A5200001003800174FB847119A938801331288F9
:10A530009B1A1BB2181AC30F1818401045192DB2D8
:10A540007CE70C21735E0092059A010038000D4FE4
:10A55000B847119A9388013312889B1A1BB2181AB4
:10A5600045192DB26AE700230893FFF7D3F9C046D7
:10A57000ED6F000065240100213C0100580000201F
:10A58000B9A50000993E010010B504000A21084B4E
:10A59000984701236380FE33237223781F2293435D
:10A5A00023702388034A134023800023637010BD67
:10A5B000752901001FF8FFFFF0B5DE4657464E46ED
:10A5C0004546E0B5CBB005900E00069107921C0001
:10A5D00002229B5E002B01D100F046FC227A052A64
:10A5E00001D800F041FC02000020115E0025705FE0
:10A5F000814200D12BE1DA0FD3185B109BB20A1C09
:10A60000814200DD021CD21A48AD2A800A1C814218
:10A6100000DA021C9A1848A98A80069A0221525E22
:10A6200005990220085E111C824200DD011CC91A36
:10A6300048AD6980111C824200DA011C5B1848AAEF
:10A64000D380079A48A90800D54B9847002801D124
:10A6500000F00AFC059B02269E5F069B02255D5FBB
:10A66000AE4200D1FCE0059B00229A5E11000892E8
:10A67000069B00229B5E9A46514500D106E2AE42FF
:10A6800006DB33002E001D00089B524608929A46B6
:10A690005346089A9B1A0993AA1B0A92D9175B186A
:10A6A0004B409946D11753184B409B460222A35E5C
:10A6B0009846D94500DCD0E25B4658014946B94B83
:10A6C0009847B94B1B5C42465A4313003F229046C1
:10A6D00098444346DB111F009BB2524608988245BE
:10A6E00000DD021CD21A0EA90A8052460898824543
:10A6F00000DA021C9A180EA98A802A1CB54200DDD5
:10A70000321CD21A0EA94A802A1CB54200DA321C29
:10A710009B180EAAD38048AA0EA90800A04B984700
:10A72000002800D19CE343461B12984601233B407E
:10A7300043440B93D94500DCBAE2099A002A00DCB5
:10A7400091E2B2B241466B4619868BB2A9B29346EA
:10A75000D21A12B2002001908946CB1A1BB2009384
:10A760005346089912A8914FB8476B469B8D5A469D
:10A77000D21812B2012101914B441BB200935346EF
:10A7800008991DA8B847002112A8894B98469847F8
:10A790000B9000211DA8C0470C90637ADB0600D403
:10A7A000ACE201235B420D930A93824B9847824BA4
:10A7B00098478146028A0EA80588AD1AABB203807D
:10A7C0004946498A45886D1A45808588AD1AADB2DB
:10A7D0008580C288521AC2800135ED1A2DB2774B9E
:10A7E0009847E023FF33984200D8B3E2F0235B00A0
:10A7F0009B465846724B984780464B461B8A0EAF85
:10A800003A889A1812B21100099210AA1180B988D8
:10A810005B1893807B884946498A5B181BB253803A
:10A82000D3805946674B98474B4612229A5E0223C3
:10A83000FE5EB61806217B5E9B189E4200DDECE2B0
:10A840000027614B9A46230044469846D0E20225F1
:10A85000555F32000226925F954200D0CBE603E3BB
:10A86000237A9846534B9847534B98478146022288
:10A87000A35E013B5E1001251D40AD190623E25E7B
:10A880000023002A04D00422A35E5A1E9341DBB2A7
:10A890001F0009934D4B98470021002801D1013139
:10A8A0007940069B00229B5E059A0020105E1A1CD0
:10A8B000834200DD021C28AF3A801A1C834200DA72
:10A8C000021C013A28AB9A80059B5B8828AA5D1B75
:10A8D00055809E19D68000290ED02288637A9B0766
:10A8E0009B0F02934346019301230093002328A961
:10A8F00048A8374DA847B3E228AA48A91000284B1A
:10A900009847002800D1ABE228AA0023D75E4B4627
:10A9100010215B5E9B4669460B840B8CF91A89B249
:10A92000884609B28A4611800220115E4D466D8A22
:10A93000AC464D1B55800420165EF31A9BB29380E3
:10A94000D58860462D1AD580013342469B1A1BB22A
:10A950000B9333AB1F809E805980D9800021099BC7
:10A96000002B08D0504658440623E15E0422A35E23
:10A97000C918184B98470BB20C930B980700104B53
:10A980009847089028AB02229E5E06229B5EB34247
:10A9900000DA77E00B4B9B460B4B9A460A9750E048
:10A9A0000B140100B9C10100B063020091BB0000AB
:10A9B00075BA000091550000750E0100EF130100FB
:10A9C000A1270100192A0100D1BA00006DBB0000C7
:10A9D000ED6F000085C301000626A55FED180B0092
:10A9E000AA4202DA089B19541300013001331AB24B
:10A9F000874207D90425635F9342EDDB9A1A12B2AE
:10AA00008018F2E70A9766460220228833AD637AFF
:10AA10009B079B0F0293237A01930090089B2900C8
:10AA200048A8D14FB8476B8801336B80EB8801335E
:10AA3000EB8001360AAB7E229B1800229B5E9E4271
:10AA400020DC0A9F3900089D2800D8474B465A8AC7
:10AA5000921912B2198A0AAB78201B181B88C918E0
:10AA600009B20B9B2800D047099B002BCDD00028B2
:10AA7000CBD0002F04D00C9A00200021B446B9E7B7
:10AA80000220C2E70898B94B9847E9E1237A984633
:10AA9000B74B9847B74B984707000222A35E013B8C
:10AAA0005E1001251D40AD190623E25E0023002A39
:10AAB00004D00422A35E5A1E9341DBB299460A9346
:10AAC000AD4B98470021002802D101314B46594037
:10AAD0000598028828AB551B1D8096199E80069A02
:10AAE0000225525F0225455F101CAA4200DD281C8A
:10AAF0005880131CAA4200DA2B1C013B28AAD380E1
:10AB000000290ED02288637A9B079B0F029343464D
:10AB1000019301230093002328A948A8924DA84738
:10AB20009EE128AA48A91000944B9847002800D11C
:10AB300096E128AA0021535E9C463B8A6146C91AC9
:10AB400089B211800225505F7D8AA846451B558039
:10AB50000425565FF31A9BB299469380D5884346E5
:10AB6000ED1AD5804B460133591A0BB21A000B93DC
:10AB700033AB614619809E805880D8800C921000BB
:10AB80007F4B9847089000210A9B002B0CD0102384
:10AB9000F85E28AB00229B5EC0180623E15E04220B
:10ABA000A35EC918774B98470BB2994628AB02228F
:10ABB0009E5E06229B5E9E424BDC734B9B46734B14
:10ABC0009A46B8464B4609931DE0099F01373BB2B0
:10ABD0000993228833AD00230293237A01930090D6
:10ABE000089B290048A8604FB8476B8801336B80E9
:10ABF000EB880133EB8001360AAB7E229B180022E2
:10AC00009B5E9E4225DC0C99089D2800D847434650
:10AC10005A8A921912B2198A0AAB78201B181B881B
:10AC2000C91809B20B9B2800D0470A9B002BD0D033
:10AC30000028CAD00423E25E099B9A4200DA002071
:10AC40000621635E9B18099A9A42BEDB0023099392
:10AC5000BBE70898454B984702E14B4658015946D7
:10AC60004B4B98472DE5B2B26B469B8DA9B29346EC
:10AC7000D21812B2002001900B918C4663441BB293
:10AC800000935346089912A8424FB84743466A4674
:10AC90001386138E5A46D21A12B2012101910B99D2
:10ACA000CB1A1BB20093534608991DA8B8476AE512
:10ACB0006B461A8C998D534668468385838D9B46D7
:10ACC000CB181BB20B929446614409B20022019248
:10ACD0000095320012A82F4FB84743466A461386A4
:10ACE000128E5B469B1A1BB20B998A1A11B2012273
:10ACF0000192009532001DA8B84744E56B461B8DB4
:10AD000099466B469B8C98464B460899CB1A1BB2CA
:10AD1000032201924246921912B20092320028A8F0
:10AD20001C4EB04753464A469B1A1BB20222019260
:10AD30004246521912B200922A00514633A8B04737
:10AD4000002128A8144DA8470A90002133A8A8473D
:10AD50000D902AE50EA8114B9847834649E5290036
:10AD600008980F4B98474CE0ED6F000065240100F8
:10AD700091550000750E01006DBB00000B14010021
:10AD8000A127010085C30100192A0100D1BA0000E2
:10AD9000B9C1010091BB000075BA0000EF130100BA
:10ADA0007529010043461A885B7A9B079B0F029323
:10ADB00043461B7A019302230093230048A910A85D
:10ADC0004D4FB8470AABDB8B01331BB20AAA538342
:10ADD000D38359462000494B9847002701360EABD4
:10ADE00006229B5E4A461221525E9B189E4211DC4F
:10ADF000E3191800089332B22B000999D0470028B4
:10AE0000ADD07F19EB199B45CCD910AAD38801335B
:10AE1000D380E3E74346A0461C0010AA0621535EF8
:10AE20000221525E9A420FD010A8013BC3802288B3
:10AE3000637A9B079B0F0293237A0193022300936B
:10AE4000434648A92C4DA84740462D4B98470B98A0
:10AE50002C4DA8470C98A8470A98A8470D98A847D2
:10AE6000637A0C221A4206D14BB03CBC90469946FC
:10AE7000A246AB46F0BD33AD2800234B984723884C
:10AE80006B80224B2B80237A2B730222A35E5E10F1
:10AE90000122534001251D40637A5B0717D4637A72
:10AEA0001B07E1D506990A88B6B228A8931B038030
:10AEB00049888B1B4380ADB29219521B8280761851
:10AEC000761BC68033AA0799114B9847CCE7059F9C
:10AED0003A88B3B228A8D11A01807F88F91A418034
:10AEE000A9B2D218521A8280DB195B1AC38033AA26
:10AEF0000799074B9847D2E7ED6F0000192A010028
:10AF00006524010025BB0000CDBF0000FF7F0000CD
:10AF100071C00000F8B5DE4657464E464546E0B5DE
:10AF20000A9CA58A521B12B2658A4D1B2DB2216A5A
:10AF3000002940D12831615CC90711D5217C032348
:10AF40000B40012B00D8C5E1022B06D00024032BB7
:10AF500045D1D417A41AE40F41E00132D40F3EE0EA
:10AF6000217C03220A40911E012900D8B4E1012A64
:10AF70000FD0002A10D1E91800D5AFE16D42002DA5
:10AF800000DAADE10224AB4229DD4019BD4B984700
:10AF900025E00124002D22DC1A00DD4200D5A1E1CC
:10AFA0006942CB43DB17194000248A4217DDB54BB9
:10AFB0009847023413E02821615C8B46C90715D4F9
:10AFC000A7691100794389128C46F917C91BC90F6B
:10AFD00061448D4200DC96E05B469C07E40F200054
:10AFE0003CBC90469946A246AB46F8BDE1692F00AD
:10AFF0004F43BF12002906DD974200DC76E15B4635
:10B000009C07E40FEBE7974200DBABE15B469C0754
:10B01000E40FE4E75B465E08012466400124344007
:10B02000DDE75B465E080124664001243440D6E734
:10B03000002190E100214B46C154636AD21A0135C8
:10B04000BD4243DA636A9A421ADD002DF5DBBD4248
:10B05000F3DA5B10D31ADBB24146615C0E4201D0D9
:10B06000DB43DBB2A946415DF92BE4D8052BE1D9DE
:10B070004B431902C918C901CB18DB0DD9B2DAE765
:10B08000BD4223DA002D21DBA36953439B125343B6
:10B090005B12DBB2E269002A13DB2822A25C920772
:10B0A00001D5DB43DBB246193278F92B0DD8052BDD
:10B0B0000AD953431A02D218D201D318DB0DDAB2DF
:10B0C00003E0DB43DBB2E8E7002232702823E35CD5
:10B0D0009B070CD50024674500DA80E702346346FD
:10B0E000002B00DA7BE76146664B984777E701352E
:10B0F00000D5F9E00224BD4200DD70E7791B40195C
:10B10000604B98476BE79846E9188C4506DD5B462F
:10B110005C08012666400124344060E7110279434F
:10B120008E14B4468903090E013212027A43961432
:10B13000B2466646761BB146D4455CD0002F52DB42
:10B14000FF22511AE5694D43AD12002E19DBC845A7
:10B1500017DD69434912CAB25946890701D4D2435F
:10B16000D2B2494646183178F92A09D8052A00D8BA
:10B1700099E04A4311028918C9018A18D20DD1B247
:10B1800031704A46511C1DD488451BDDFF22551BDA
:10B19000A2696A43921255436D12EAB22825655D91
:10B1A000AD0701D5D243D2B241180D78F92A08D89B
:10B1B000052A7AD96A431502AD18ED01AA18D20DF5
:10B1C000D5B20D702822A25C920770D50024C84524
:10B1D00000DA04E702344B46002B00DAFFE649466A
:10B1E000284B9847FBE6002900D0CCE001398C467B
:10B1F000E1440131FF314E46002E1BDBC84519DD0D
:10B200009203120E521852085946890701D5D243AB
:10B21000D2B2494646183178F92A0AD8052A07D900
:10B220004A4311028918C9018A18D20DD1B200E02F
:10B23000002131702822A25C92070CD55346591B7D
:10B240000024884500DCCAE60234002900DAC6E69C
:10B250000C4B9847C3E6494601311A00884500DD8A
:10B260000A000024002A00D1B9E60234002A00DCDA
:10B27000B5E6991A8018034B9847B0E60025A1E07F
:10B280000025C2E0752901004A460132012490459B
:10B2900000DAA4E60134002A00DAA0E6991A801840
:10B2A000624B98479BE600216AE7002589E74946FB
:10B2B00002311A00884500DD0A000024002A00D16E
:10B2C0008DE60234002A00DC89E6991A8018574B73
:10B2D000984784E6012482E6012480E601247EE684
:10B2E00000247CE600247AE6002478E61F00EB18B0
:10B2F000594389128A4200DD8CE61202A3695A433F
:10B3000092121112FF231A4039D09C469B1A98467C
:10B31000636A424653431B126246D21A491B8C464B
:10B320001AD4B94218DA41464B435B12DBB2594694
:10B33000890701D4DB43DBB2614645182978F92B34
:10B3400009D8052B00D873E64B431902C918C90167
:10B35000CB18DB0DD9B2297063465D1C28239846B3
:10B3600002266FE61F005B1959438912914200DDE6
:10B3700057E601321202A3695A439212C1E74D1BEC
:10B38000AC46FF22EAE7E26952424A439212002E9B
:10B3900019DBC84517DD51434912C9B25D46AD07F7
:10B3A00001D5C943C9B24D4646193578F92909D89E
:10B3B000052900D862E769430D026D18ED0169188F
:10B3C000C90DCDB23570494601391FD488451DDD00
:10B3D000FF25AA1AA5696D425543AD126A43521260
:10B3E000D2B22825655DAD0701D4D243D2B246184A
:10B3F0003578F92A09D8052A00D841E76A431502A9
:10B40000AD18ED01AA18D20DD5B235702822A25C74
:10B41000920700D438E70224884500DADFE50029E6
:10B4200000DCDCE5014B9847D9E5C04675290100F1
:10B43000F0B5DE4657464E464546E0B58DB0019024
:10B4400089460093169DAC7CE407E40F1023EE5E62
:10B450002F00083700230AA8F95C19540133082B80
:10B46000FAD1002C45D10AAB02215B5E0020934249
:10B470004ADC0AAB06215B5E934245DBB4460AAB6D
:10B4800000201B5E9A46F318994508DB009B4B444D
:10B4900018000AAB04215B5E9B1B98420BDD0AA8D7
:10B4A0000227C05F8719BA4262DB0AAF06217F5EBE
:10B4B000BF1BBA425CDC002C3CD153464A469C1A66
:10B4C000009D0020AC421FDC002C03DB2100019812
:10B4D000A24B98470AAB0420185E4B46C01A0130B5
:10B4E000002800DC0BE2854215DC002C1ED0022077
:10B4F0000AE00AAB02215B5E0120934204DC0AAB46
:10B5000006215B5E9342B9DA0DB03CBC9046994689
:10B51000A246AB46F0BD009B191A019B9C466044B5
:10B520008E4B9847002CE2D10220EDE78542DED118
:10B530000120E9E753464A469B1ADA43D2171340E3
:10B54000009A02209342DFDC0AA90420095E4846E3
:10B55000091AC91A01315818824200DAD11A022098
:10B560000029D1DB019AD0187C4B98470220CBE709
:10B570000AAB04215F5E80B2DB8801331B1A1BB269
:10B58000121A30007043804612B2944500DDE0E1AB
:10B59000981B0138824200DDB3E10220B4E76B8BD7
:10B5A00006AA53802B8B1380E9E1802109010291C7
:10B5B000AFE107AB6A8B5A802A8B1A80B8E107A9E2
:10B5C0004988002900D0F5E107A9013A0A80FF2245
:10B5D0004A80EFE106A9498807AD6D8849194910ED
:10B5E000CFB2002C01D0FF43FFB2F31A013BC118C8
:10B5F00012D4009DA9420FDA019D6E183578F92FFB
:10B6000009D8052F36D97D43AC462D026544ED019E
:10B610006544ED0DEDB23570D21A013A151811D40A
:10B62000009B9D420EDA019B5A191378F92F08D816
:10B63000052F21D95F433B02DB19DB01DF19FF0D29
:10B64000FBB21370002C19D0481CC343DB17184001
:10B65000009A1300111A954200DC291A984200DB67
:10B660002DE1002900DA2AE1019B9C4660443B4B16
:10B67000984724E10025CEE70023E2E7009CA142A1
:10B6800000DD3AE1002902DB0198344B9847681C41
:10B6900000D532E1A04200DD11E1009B191A019BA7
:10B6A0009C4660442D4B984709E109AD059B180065
:10B6B00058434346181A029A2900294B98476A882A
:10B6C00006AB5988FF23591A9B1A4B435B12DBB216
:10B6D000002C01D1DB43DBB2039D002D14DB00986D
:10B6E000854211DA01990800AC4660440178F92BD3
:10B6F00009D8052B2BD959430D0009024919C90155
:10B700004919C90DC9B20170049D002D13DB0098C1
:10B71000854210DA01990800AC4660440178F92BA3
:10B7200008D8052B15D94B431902C918C901C918E6
:10B73000C90DC9B20170039B013B0393049B013304
:10B74000049308AB5A80059B0133059376E10021F1
:10B75000D9E70021EEE700223FE0C046752901004D
:10B7600015220100002201984254013C0122944616
:10B77000E24401372E005F4546D83509029B9C46BE
:10B780006544380078434346181A00022B006B4387
:10B79000C01A6900B44B984745192B119BB22D0173
:10B7A000FF22154076197610F6B24A46002A01D0DB
:10B7B000F643F6B2002C12DB009AA2420FDD200005
:10B7C000019A125DF92E08D8052EC4D972431102D0
:10B7D0008918C9018A18D20DD2B201990A54524669
:10B7E000002AC2DB009A5245BFDD5146019A525CE5
:10B7F000F92EB8D8052EB5D9564332029219D20186
:10B800009619F60DF2B2AEE74C465A46D243059E63
:10B81000B446624403998C469444624603925A4665
:10B82000501C049A94466044821B049208AA5580D6
:10B8300009AA1380558008AB5B88002B3DD007AA6E
:10B84000528853435B12DBB2002C01D0DB43DBB2E6
:10B85000039A002A14DB00990800904210DD019938
:10B860009446614408000A78F92B08D8052B28D99A
:10B870005A4311028918C9018A18D20DD2B2027036
:10B88000049A002A13DB0099080090420FDD019909
:10B89000944661440A78F92B08D8052B13D95343F1
:10B8A0001A02D218D201D318DB0DDAB20A70039B48
:10B8B000013B0393049B01330493002C05D0022029
:10B8C00022E60022DBE70022F0E703990131009C29
:10B8D000A14212DC002902DB0198644B9847049BCB
:10B8E000002B0ADBA342EADA009AD11A019A9C469D
:10B8F000624410005D4B9847E1E7002004E6002019
:10B9000002E680204000844500DC4EE680210902EA
:10B9100002919A1AB01A431C9B466B69984200D157
:10B9200047E640434346181A029A07A9504B9847E6
:10B93000584640434346181A029A06A94C4B98476A
:10B940005B466B6106AB5B886B8306AB1B882B8306
:10B9500028E080235B009C4500DD81E080231B0103
:10B960000293B31A9B466B699B4500D117E6584674
:10B9700040434346181A029A06A93D4B98475B4636
:10B98000013B1800039358434246101A029A07A934
:10B99000374B9847039B6B6106ABDB886B8306AB29
:10B9A0009B882B8306AB1B8807AA1288511E8B42EB
:10B9B00000D104E652464946501A0137BA1A12B26B
:10B9C00007A90988994200D104E60133F61A8319C0
:10B9D00019000393961B013E33181D000493002C9D
:10B9E00012D0481CC343DB171840009E3300311AA5
:10B9F000B54200DC291A984206DA002904DB019BD3
:10BA00009C466044194B984706AB1888431C059325
:10BA100008AD40434346181A029A2900144B984730
:10BA20006B88002B05D108AB1A88013A1A80FF22D7
:10BA30005A8008AB1B889B4500DC36E607AB1B88A9
:10BA40009B46059F5F4500D9F5E608AB1A881201B1
:10BA500002925E88049B9A46039BA1461C008CE6DA
:10BA600080231B0202937CE7B9C101007529010004
:10BA70001522010010B582B0104B1B68002B14D0AA
:10BA80000E4A01239468002C10D00133DBB2083237
:10BA9000102BF7D10A4B00930A4B57220A49022078
:10BAA0000A4CA0470120404206E00023034ADC0084
:10BAB000A0501219516018B202B010BDF44D002010
:10BAC00020640200D4630200E863020059210100EF
:10BAD000F0B587B00390049116001F00104B1B684F
:10BAE000002B1BD00E4C0022059203E00834236883
:10BAF000002B0DD000931D683B0032000499039881
:10BB0000A847002808D00228F0D101230593EDE7CB
:10BB10000598431E9841013007B0F0BD0120FBE7B6
:10BB2000F44D0020431C07D0044AC300985800215C
:10BB30009950D318596070470020FCE7F44D00205D
:10BB400030B50100084B1A0080320020002402E0CA
:10BB50000833934206D05D688D42F9D118681C60A5
:10BB60005C60F5E730BDC046F44D0020074B1A007D
:10BB70008032002002E00833934205D01968002982
:10BB8000F9D00130C0B2F6E77047C046F44D00204E
:10BB9000F8B5CE46474680B504000F00150098461C
:10BBA00008AB00269E5F09AB1B7899462C21514BB0
:10BBB0009847B54205DD2B0035001E003B00474687
:10BBC0009846278165814346A381E68103234A463F
:10BBD0001340227C03218A431A4322746782A58280
:10BBE0004346DF1B761BFB17FA185A40F1177318F0
:10BBF0004B4001259A4200DC0025282101222B0020
:10BC00001340655C012085431D4365540023E361B7
:10BC1000A3613949216023712A4227D0002F07D020
:10BC2000390080204003354B984770438012E06113
:10BC3000002E07D0310080204003304B9847474307
:10BC4000BF12A761E3692362227C0323134024D13E
:10BC50002822A35C02218B43A354236A9A10002B51
:10BC600045DB62620CBC90469946F8BD002E07D0B9
:10BC7000310080204003214B984778438012A06117
:10BC8000002F07D03900802040031C4B9847704399
:10BC90008012E061A3692362D6E7012B0CD0022B4E
:10BCA00010D0032BD9D1236A002B1ADD2822A35CE4
:10BCB00002218B43A354D0E72822A35C02210B432B
:10BCC000A354CAE7236A002B05DD2822A35C0221C6
:10BCD0000B43A354C1E72822A35C02218B43A35446
:10BCE000BBE72822A35C02210B43A354B5E75242D1
:10BCF0006262B7E77529010015AF0000B9C1010004
:10BD0000F0B5CC8801344D88641B8E8801360D88CF
:10BD1000761B251C24B237B2BC4200DD351C2DB287
:10BD20006D10AA4200DD2AB20E0008360400083465
:10BD30000D782570013401318E42F9D10282012241
:10BD40001A40837C01218B4313438374054B0360AA
:10BD50000223037180231B06436100234383038373
:10BD6000F0BDC04631B40000F0B5DE4657464E4641
:10BD70004546E0B591B00D9002910C924B101E001B
:10BD80000F9301230B405A425341F31A1D000E93A7
:10BD9000040047003800884B98470590231E00DCBC
:10BDA000DBE0B91E0391013B06938C46604407908B
:10BDB0001900491B0891290028000A957F4BA446C9
:10BDC00063445B1A5D000B9549000A0009967100F7
:10BDD00088460C9B99460023009302256D422B1A3E
:10BDE00001979B46CA46914624E09B1A002E10DB21
:10BDF0002A88D318023F023D013E5E450CD03B80AD
:10BE0000811900228C42F0DD4A46AA184244528829
:10BE1000EBE752461288ECE7019D2A00059950464F
:10BE2000674B9847AC46E244009B01330093A34222
:10BE300000DBAAE0029A0492534603995B5A5343EB
:10BE4000069A002AE8DB0B9A52441500089A561EFF
:10BE5000079F099A501C0A9A94466044CFE701361E
:10BE60000235A64207D268882B888342F7D004990E
:10BE7000C8476880F3E74446002C00DC7BE00C9B5D
:10BE800003930E98421C13007B4308930F9D6B4253
:10BE90007B439B460D994B005B425A4300920B003B
:10BEA000013B4B435B0002930023069303000122F6
:10BEB000944663449A46B8465B460193AB4637E0E6
:10BEC00000210FE04846008816E041460298095AD2
:10BED000CB180132B944F6190234624512DA002B4C
:10BEE000EEDB9911218011005846101A0028E9DD77
:10BEF00001988019009D405B1B1A51446145E4DAAA
:10BF00003188E5E74546B846079F64460023414629
:10BF10003A882A8001336D180237A342F8DB88463D
:10BF2000069B01330693039A02320392A34222DA5C
:10BF3000039A1500138804994B4308990E00944600
:10BF40006644059A17009446A9460022079747467B
:10BF5000210064468C46A846C1E7029B04930C9DD1
:10BF600028881900174B984728800D9A13005343CF
:10BF70009846012B17D80598134B984711B03CBC35
:10BF800090469946A246AB46F0BD019F0C9D28887D
:10BF900004990C4B984728800D9A130053439846F8
:10BFA000012B00D86BE70C9D0126064B99464346B2
:10BFB000A0461C0057E7C046A1270100FEFFFF7FF7
:10BFC00045250100B9C101006524010010B5040038
:10BFD0005421234B9847234B1B88638023791F22CE
:10BFE00093432371A188204B1940A18000216171E6
:10BFF000A17B9143A173E1891940E1810021E173A3
:10C000003420215C91432154A18E1940A186210046
:10C010003431002048704621605C90436054605A7F
:10C02000184060522100463100204870A17F9143A2
:10C03000A177E28B1340E3830023E377FF3363812F
:10C040002373237723753622A354084A226344219D
:10C05000635422642822A354F03B638210BDC0467F
:10C0600075290100486402001FF8FFFF300000201E
:10C07000F0B5DE4657464E464546E0B5B1B081467E
:10C0800004919346C4884588631C5B1B1BB2002B3C
:10C0900001DC00F0CEFF86880788731CDB1B1BB217
:10C0A000002B01DC00F0C5FF130020229B5E9846A8
:10C0B000002B01D100F0E1FE28235A46D35C069301
:10C0C000052B01D800F0D9FE136A012B00D1E2E064
:10C0D0005B46598CDA8C8B1AFF18BFB214AB1F80E9
:10C0E00089187618B6B29E805946898C881A2D1800
:10C0F000ADB25D805218A418A4B2DC804346DB0FB9
:10C1000043445910C94389B216AA781810805B10AD
:10C1100001339BB2F018908069185180E318D380E6
:10C12000069BFA2B01D9FF2306939F4B98479F4B01
:10C1300098478246049A16A918A89D4B984700284C
:10C1400001D100F09AFE53461B8A9C4618AB1A8810
:10C150006146521A1A805246508A5A88121A5A80D8
:10C1600099886246891A9980DA88121ADA8000233F
:10C170001AA94846C25C5A540133082BFAD18146A9
:10C180001AAB198801318AB294461A805888013056
:10C1900082B205926A46928A5A809888421E9A8094
:10C1A000DA88511ED9805B4600215B5E6146411AE8
:10C1B00009B20598101A00B20200814200DA0A00A2
:10C1C00052100F929A4200DD0F930136F61BB2B265
:10C1D000924611B20134651BADB22AB214009142ED
:10C1E00000DA0C0064109C4200DD1C00A0444346B1
:10C1F00009934046584340006E4B98470E905B466B
:10C200002027DF5F22B2B846D3190793002322A864
:10C2100014A95E5C1E540133082BFAD1FB0FDB1905
:10C220005B109BB2012139400E001091591E7042E3
:10C230007041091A0C19A4B222A98C8001339BB257
:10C240004B805046241A0C80ED18CD80002329A87D
:10C25000594CA0474346012B01D102F079F97B10DC
:10C260000D93079C0C942000524B98470A90002C89
:10C2700061DD0C9B5B000B93079B504A9446634423
:10C280005B000E9A9246002290464D4F524608920D
:10C29000CA4699461CE05B4624229B5E002B00D0D8
:10C2A00016E75B4626229B5E002B00DD10E700F0C0
:10C2B000E4FD0B990898434B9847089B0B9A9446CA
:10C2C0006344089301239C46E044079B434531DDCA
:10C2D0000C990A9C20003C4B98476B461C229B5EA5
:10C2E000424612B229A9009100212000299CA047B2
:10C2F0000028DED00D9B05930A9D28788001190047
:10C300002F4B9847089B1880079A012AD5DD1C00FF
:10C310004B441E0005E02388638001350234A642A9
:10C32000CBD068782B788342F5D080010599B84747
:10C330006080F2E7D1460A98244B98470D9B012B69
:10C3400001D102F014F96B461C229B5E08930E9CEF
:10C3500022000D9D290018001D4B9847109BAC46EC
:10C3600063441FB2012F3ADD059720888001390010
:10C37000134B984720800C9D6D43012D2AD90F4AFD
:10C38000944665446D00A44665440D4E02E00234B7
:10C39000A5421FD0608823888342F8D08001059988
:10C3A000B0476080F3E7C04691550000750E01006C
:10C3B0000B140100A127010001BD0000FFFFFF7F5A
:10C3C000B9C1010075290100192A01006524010085
:10C3D00069BD00000E9A39000898B54B9847079F31
:10C3E0007F43002F0AD00E9A1300780094466044D1
:10C3F00019881170023301328342F9D116A94A8893
:10C40000CB8801339B1A1BB2D80FC3185B10D3180B
:10C410009BB210931BB20C930A888B8801339B1A32
:10C420001BB2D90FCB185B10D3189BB211931BB260
:10C430000D93A04B984700230893002810D15B462A
:10C4400022229B5E002B0BD15B4624229B5E002B9D
:10C4500006D15B4626229A5E53425341DBB20893D3
:10C4600016ACA08801302388C01A00B2924B9847BE
:10C4700005906B463C229A5E01231AA929A88F4D8C
:10C48000A847002129A88E4B98470F900422A35E4D
:10C490001CA98B806A46928C0A9201339B1A0B80EE
:10C4A0000220235E4B80013B94466344CB80049A78
:10C4B0001EA8844B9847002871D01EAB06229B5EB5
:10C4C0000C998B4201DD1EABD9801EAB00229B5E16
:10C4D0000D9A934203DC119B01331EAA13801EABFD
:10C4E00000215A5E9B8801339B1A1BB20B93002BD1
:10C4F00055DD1EAB06215C5E02269E5F1CAB022151
:10C500005D5E751B09994D4300215B5ED21AAD1823
:10C510000E9B9C466544002322A81EA95A5C1A540F
:10C520000133082BFAD122AB5A88DA800134A61BDA
:10C5300036B2002E33DD731C9846012622AC624BC6
:10C540009A4607955F4619E0FA8B2923FB5C029314
:10C55000069B01930090059B210004985B4DA84722
:10C56000638801336380E3880133E380099B9C4641
:10C57000079B634407930136B0450FD00B9A079988
:10C580000598534B98470221625E0025615F0B9B23
:10C590000598D0470128D7D10130D5E7BB4616AA68
:10C5A0000421535E1CA98B8001330A981B1A0B804F
:10C5B0000623D25E531C1B1A4B80CA80049A1EA805
:10C5C000404B9847002800D185E01EAB02229B5EBD
:10C5D0000C9A934203DC109B01331EAA53801EABBE
:10C5E00000229B5E0D9A934203DC119B01331EAA2D
:10C5F00013801EAB00215A5E9B8801339B1A1BB22D
:10C600000B93002B67DD1EAB06215C5E02269E5F4E
:10C610001CAB06215D5E2D1B09994D4300215B5E1D
:10C62000D21AAD180E9B9C466544002322A81EA971
:10C630005A5C1A540133082BFAD122ABDA885A809B
:10C640000134A61B36B2002E45DD731C9846012628
:10C6500022AC1D4B9A4607955F4619E0FA8B2923B9
:10C66000FB5C0293069B01930090059B21000498BC
:10C67000164DA8476388013B6380E388013BE38054
:10C68000099B9C46079B634407930136464521D08E
:10C690000B9A079905980E4B98470221625E002578
:10C6A000615F0B9B0598D0470128D7D10130D5E7B2
:10C6B00069BD00006DBB0000A127010001BD0000A5
:10C6C00075BA00000B140100D1BA0000ED6F000034
:10C6D00045250100BB4616AA0421535E1CA98B8088
:10C6E00001330A981B1A0B805388844663444B809D
:10C6F000D3881B1ACB80049A1EA8D14B98470028D8
:10C700006CD0089B002B0AD01EAA10884B469B8831
:10C71000191C1BB204B2A34200DA011C11801EAB2B
:10C7200000215A5E9B8801339B1A1BB20793002B92
:10C7300054DD1EABDF8801375B88FF1A3FB20999D1
:10C740000B00013B4B431CA90020095E521A9A18AA
:10C7500013000E998C4663440B93002322A81EA954
:10C760005A5C1A540133082BFAD122AB5A88DA806A
:10C77000002F33DD0025B34B984622AC089B9A4628
:10C780005E46BB4615E0F28B2923F35C0293282317
:10C79000F35C01930090059B21000498AA4FB847D1
:10C7A000638801336380E3880133E38001355D45AD
:10C7B00013DA079A0B990598C04702205346002BBD
:10C7C000E1D10223E25E0023E15E079B05989F4FC3
:10C7D000B8470128D7D10130D5E7B346099B002BD4
:10C7E0001FDDDF0F9C4667447F100E9D00265A1EFA
:10C7F0009446B8461F000BE0197810781870117035
:10C800000133013A9C42F7D1ED190136B74208D005
:10C810004346002BF8D02B006246AA1841466C18FC
:10C82000EAE716AA0021535E1CA90B80013B0A9C73
:10C83000A44663448B800223D35E4B80013B634458
:10C84000CB80049A1EA87E4B984700286FD01EAB61
:10C8500006229B5E0C998B4201DD1EABD9801EAB7C
:10C8600004229B5E0D998B4201DD1EAB99801EABAD
:10C8700000215A5E9B8801339B1A1BB20B93002B3D
:10C8800055DD1EAB06215C5E02269E5F1CAB0221BD
:10C890005D5E751B09994D4300215B5ED21AAD1890
:10C8A0000E9B9C466544002322A81EA95A5C1A547C
:10C8B0000133082BFAD122AB5A88DA800134A61B47
:10C8C00036B2002E33DD731C9846012622AC5F4B36
:10C8D0009A4607955F4619E0FA8B2923FB5C029381
:10C8E000069B01930090059B21000498564DA84794
:10C8F000638801336380E3880133E380099B9C46AE
:10C90000079B63440793013646450FD00B9A07995E
:10C9100005984C4B98470221625E0025615F0B9B96
:10C920000598D0470128D7D10130D5E7BB4616AAD4
:10C930000021535E1CA90B80013B0A9CA446634462
:10C940008B800623D25E531C1B1B4B80CA80049A2B
:10C950001EA83B4B9847002800D17AE01EAB02226C
:10C960009B5E0C9A934203DC109B01331EAA5380FA
:10C970001EAB04229B5E0D998B4201DD1EAB99809C
:10C980001EAB00215A5E9B8801339B1A1BB20B938E
:10C99000002B5EDD1EAB06215C5E02269E5F1CAB9B
:10C9A00006215D5E2D1B09994D4300215B5ED21A65
:10C9B000AD180E9B9C466544002322A81EA95A5C14
:10C9C0001A540133082BFAD122ABDA885A80013489
:10C9D000A61B36B2002E3CDD731C9846012622AC05
:10C9E0001A4B9A4607955F4619E0FA8B2923FB5CA0
:10C9F0000293069B01930090059B21000498124D21
:10CA0000A8476388013B6380E388013BE380099B7F
:10CA10009C46079B634407930136464518D00B9A02
:10CA200007990598074B98470221625E0025615FD0
:10CA30000B9B0598D0470128D7D10130D5E7C046D8
:10CA40000B14010045250100ED6F0000D1BA000074
:10CA5000BB4616AA0021535E1CA90B80013B0A9C11
:10CA6000A44663448B80538863444B80D3881B1B4C
:10CA7000CB80049A1EA8C54B984700286CD0089B11
:10CA8000002B0AD01EAA4B4618889388191C1BB28B
:10CA900004B2A34200DD011C91801EAB00215A5E4E
:10CAA0009B8801339B1A1BB20793002B54DD1EABEE
:10CAB000DF8801375B88FF1A3FB209990B00013B01
:10CAC0004B431CA90020095E521A9A1813000E99B4
:10CAD0008C4663440B93002322A81EA95A5C1A5467
:10CAE0000133082BFAD122AB5A88DA80002F33DDCC
:10CAF0000025A74B984622AC089B9A465E46BB464B
:10CB000015E0F28B2923F35C02932823F35C019355
:10CB10000090059B210004989E4FB847638801331D
:10CB20006380E3880133E38001355D4513DA079ABA
:10CB30000B990598C04702205346002BE1D10223F0
:10CB4000E25E0023E15E079B0598934FB8470128FA
:10CB5000D7D10130D5E7B3461CA916AB1A880A9C79
:10CB6000A44662440A809A88121B8A8002229B5E35
:10CB70004B80013B6344CB80049A1EA8834B9847AB
:10CB8000002876D0089B002B0AD01EAAD0884B46DE
:10CB90005B88191C1BB204B2A34200DD011CD180CA
:10CBA0001EAA9388013311885B1A1BB20B930221D2
:10CBB000535ED4880134E41A24B209990C911CAA5A
:10CBC0000225555F5D1B4D434B1EED180E9B9C4689
:10CBD0006544002322A81EA95A5C1A540133082B6D
:10CBE000FAD122AB5A88DA80002C42DD631C9846C9
:10CBF00001266A4B9A4622AC07955F461EE0069BCB
:10CC0000FF2B1FD1069920E0FA8B2923FB5C0293AE
:10CC1000FF2301930090059B210004985D4DA847D8
:10CC2000638801336380E3880133E3800C9B9C4677
:10CC3000079B634407930136464519D0079B197833
:10CC4000FF29DCD0069B5943090A0B9A0598D04767
:10CC50000220089B002BD7D10223E25E0023E15E75
:10CC60000B9B05984C4DA8470128CDD10130CBE74F
:10CC7000BB461CA916AB1A880A9CA44662440A80CB
:10CC80009A88121B8A8006229A5E531C1B1B4B80BB
:10CC9000CA80049A1EA83D4B9847002800D181E025
:10CCA000089B002B0AD01EAA50884B46DB88191C13
:10CCB0001BB204B2A34200DA011C51801EAA938861
:10CCC000013311885B1A1BB20B930621535E5C1C67
:10CCD0005288A41A24B209991CAA0625555FED1A98
:10CCE0004D434B1EED180E9B9C466544002322A825
:10CCF0001EA95A5C1A540133082BFAD122ABDA88E8
:10CD00005A80002C4EDD631C98460126234B9A4620
:10CD100022AC07955F46CB461EE0069BFF2B1FD13A
:10CD2000069920E0FA8B2923FB5C0293FF230193F1
:10CD30000090059B21000498164DA8476388013B8D
:10CD40006380E388013BE380099B9C46079B634427
:10CD500007930136B04523D0079B1978FF29DCD013
:10CD6000069B5943090A0B9A0598D0470220089B55
:10CD7000002BD7D10223E25E0023E15E0B9B0598D6
:10CD8000054DA8470128CDD10130CBE70B14010098
:10CD900045250100ED6F0000D1BA0000D528010043
:10CDA000D946BB461CA916AB1A880A9CA446624405
:10CDB0000A809A88121B8A805A8862444A80DB88DB
:10CDC0001B1BCB80049A1EA8C44B984700284CD04C
:10CDD000089B002B49D11EAA9388013311885B1A46
:10CDE0001BB20693D78801375388FF1A3FB200233E
:10CDF00022A811005A5C1A540133082BFAD122AB35
:10CE00005A88DA80002F30DD01370125B44B9A466D
:10CE100022ACB44B98465E46BB4614E0F28B292305
:10CE2000F35C0293FF2301930090059B210004987B
:10CE3000AD4FB847638801336380E3880133E380F3
:10CE40000135AB4510D02823F15C069A059F3800C8
:10CE5000D0470221625E0020215E069B3800C04759
:10CE60000128DBD10130D9E7B3460F989F4B984793
:10CE700005989F4CA0470E98A0475B461B7B9A469F
:10CE8000052B3FD900231AA94846C25C5A540133E6
:10CE9000082BFAD181465B4610229B5E012B1FDDD9
:10CEA0005B461B7DF92B1BD95B4600229B5E002B4A
:10CEB00016D05B46588A1AAB8108012211401C88A3
:10CEC00009191980410811405C8809195980C40862
:10CED00014409988091B99800240D9888A1ADA80FF
:10CEE0005346FA2B01D9FF239A46824B9847824B2F
:10CEF00098470700049A1AA91CA8784B984700285D
:10CF000000D09DE05B46D86A002806D036235A46FA
:10CF1000D35C052B01D900F0D7FB5B461E7D052EA7
:10CF200019D910229B5E002B15D05B4612229B5E06
:10CF3000002B10D0FA2E00D9FF266E4B98476E4B6F
:10CF400098470700049A494618A8644B9847002858
:10CF500001D000F041FD5B46D96B002906D0442387
:10CF60005A46D35C052B01D901F056F85B461B7F6E
:10CF70009846052B5DD95B4618229B5E002B58D046
:10CF80004346FA2B01D9FF2398465C4B98470A90F9
:10CF9000002316A94846C25C5A540133082BFAD123
:10CFA0005B465D8B16AB1A88521B92B292461A8072
:10CFB0005A88521B92B207925A809F88EF19BFB2CB
:10CFC0009F80DA88AD18ADB2DD805B4600229B5EA3
:10CFD00006935B4618229B5E0593002318A816A9AA
:10CFE0005A5C1A540133082BFAD16B469C8A18AE4E
:10CFF00033881B1B9BB208933380B388E3189BB222
:10D000000993B38073881B1B9BB20B937380F388C7
:10D01000E418A4B2F480374B9847374B98478146C1
:10D02000049A31001AA82D4B9847002801D001F02E
:10D030004FF831B03CBC90469946A246AB46F0BD95
:10D04000388A1CAA1188091A89B211807D8A5488ED
:10D05000641B548093881B1A9BB29380D088401B1A
:10D06000D08001335B1A1BB20A930B931800244B38
:10D0700098470690214B984783B20C930022079261
:10D08000002B06D15B469B79023B5A1E9341DBB2D3
:10D0900007931AA98C8801340B88E41A24B226005D
:10D0A0005B4600229A5ECB88013349885B1A1BB22B
:10D0B000A34200DD23005B109846934200DD9046BA
:10D0C000079B002B2FD04346002B2CD15B469B792E
:10D0D000002B17D001235B420F9333E00B140100A8
:10D0E000D5280100D1BA0000ED6F000025BB00007B
:10D0F0006524010091550000750E01006DBB000014
:10D10000A12701005B465A885B7B0293534601933B
:10D110000123009300231AA90498AE4CA0470123D1
:10D120005B420F9377E24346002B37DD43461AB24A
:10D1300000231AA929A8A84DA847002129A8A74B70
:10D1400098470F905B465B886A4613845B469B79E1
:10D1500000220D92022B25D01AAB0422995E0020EA
:10D16000185E4B1C1B1A1BB2424652009B1A0993B5
:10D170001EAA108091801CA90223CD5E7B8A5B19B8
:10D180001BB25380D38006228B5E9D4200DD32E2CB
:10D190004B461093B9465E46D346E8E001235B4216
:10D1A0000F93CFE75B465A889B889A42D4D06000A1
:10D1B0008B4B98470D90002ECEDD002542460992FC
:10D1C000B0462E005D46BB4605901EE0A978C90614
:10D1D000C80E6B885B059B0EEA78D20821781F2762
:10D1E000B94301432170590123887E4803400B4312
:10D1F0002380D2001B0A07210B40134363700136C2
:10D20000059B02330593B04558DD059C0823E95E74
:10D2100040464843001232B29042D7DA0A27EB5F09
:10D2200047465F433F12BA423FDA591A43465943D1
:10D23000301A00B20302181A09126B4B9847FF23E9
:10D240001840191A6A79D2084243EB78DB084B433D
:10D25000D3181A02D218D201D218D20D1F231A40A5
:10D26000AB885B059B0E43439C466B885B059B0E1E
:10D270004B4363441F02BC469C446746FF01BC46C7
:10D280006344DB0D3F273B402F79FF06FF0E7843B9
:10D29000AF78FF06FF0E7943401801020918C90153
:10D2A0000918C90D1F20084098E72979C906C80E3A
:10D2B000AB885B059B0E6A79D2088FE7099B98467D
:10D2C0005F46AB4648E70B99069F3800474B9847A7
:10D2D0004B465A8A521912B2198A0EAB1B8FC918C3
:10D2E00009B20A9B3800424FB8470590B379012B29
:10D2F00019D181E00B99069F38003C4B98474B466B
:10D300005A8A521912B2198A0EAB1B8FC91809B268
:10D310000A9B3800364FB8470590B379012B6BD084
:10D32000079A002A3ED1022B00D153E10C9B002B1F
:10D3300002D1099B322B0CDC737B02935B46019379
:10D34000059B0093069B6A46128C1EA90498214CEB
:10D35000A0471EAB5A8801325A80DA880132DA803F
:10D3600001350EAB3E229B5E9D4200DD3FE14B4608
:10D3700012241C5F64191AAB02229B5E43440133E2
:10D380009C42B7DD1AAB06229B5E42469B1A013BCC
:10D390009C42AFDA079B002B95D0B379012B29D0A3
:10D3A00001220592099A322A00DDA0E0022B00D169
:10D3B00010E1012BBAD1737B02935B460193059B6D
:10D3C0000093069B6A46128C1EA90498014CA04744
:10D3D000BFE7C046ED6F000001BD000075BA000058
:10D3E000A12701001FF8FFFFB9C10100192A0100A0
:10D3F000D1BA0000012305937288B3889A426DD098
:10D400001AA94A88A31A9BB20827F05F8246C988E6
:10D410000131891A09B202004A43121218B2844635
:10D42000824245DA0A27F05F07004F433F12BC45AE
:10D4300000DBB1E05746C01B41439B1A1BB21802E8
:10D44000C01A0912C04B9847FF210840091A727987
:10D45000D2084243F378DB084B43D3181A02D218A0
:10D46000D201D218D20D1F239C461A40B3885B0507
:10D470009B0E43439A4673885B059B0E4B439A442D
:10D4800053461B025344DB015344DB009B0E3779A8
:10D49000FF06FF0E7843B778FF06FF0E7943411869
:10D4A00008024018C0014018C00D6146084007E05E
:10D4B000B178C906C80E73885B059B0EF278D20856
:10D4C0001F21089F8F433900014358019F4B0B4098
:10D4D0000343D2025B055B0D13430893079B002BAC
:10D4E00000D168E70123099A322A00DC63E71AAA0F
:10D4F0000221525E42440132944208DB1AAA0621FC
:10D50000525E4146521A013A944200DC4EE71AAB91
:10D5100000229B5E22A90B80424668460287048F48
:10D52000013BE3188B801EAB5A884A80DB88CB8096
:10D53000737B02935B460193059B0093069B028CD1
:10D540000498834FB847B379012B2ED01AAB04222D
:10D550009B5E22A95A1C141B0C808B8042469B1A8E
:10D5600001334A461021525E0EA93820095E521836
:10D570009B1ADA43D2171340069A94466344727B8F
:10D5800002925A460192059A00926A46128C22A98A
:10D5900004986F4CA047DCE63179C906C80EB38801
:10D5A0005B059B0E7279D2088AE722A91AAA138812
:10D5B000E3180B8093881B1B8B80737B02935B4665
:10D5C00001930123009300236A46128C0498604F54
:10D5D000B847BBE7737B02935B460193059B0093BF
:10D5E000069B0D9A1EA904985A4CA047B1E6DA464C
:10D5F000109B9946B3465B469B79002B05D10C9B4B
:10D60000002B02D1099B322B0CDC0D9B002B02D08E
:10D610001800514B98470F98504B984706984E4B1F
:10D6200098476FE443466A469382968A1EAC1AADC9
:10D630002B88F3182380AB889B1BA3800222AB5E50
:10D640006380F318E3805B465A885B7B0293534602
:10D650000193012300930023210004983C4FB84715
:10D660000623E95E8A1B12B262800620235E9A427C
:10D6700002DC01331EAA53801EACE1805B465A884F
:10D680005B7B0293534601930127009700232100FF
:10D6900004982F4DA8471AAA138823809388A38043
:10D6A00053880133F3186380D388013B9E1BE680C7
:10D6B0005B465A885B7B0293534601930097002395
:10D6C00021000498A847A0E7254B984707000128A8
:10D6D00011D902285AD0234B0093234B234A2449C3
:10D6E0000220244CA0470023002204994846224CE3
:10D6F000A047FFF712FC29A95B46D86A1F4B984741
:10D70000012809D01E4B0093174B1E4A18490220CE
:10D71000184CA047FFF701FC299BDD026D0D6E231D
:10D720000EAA944663441E8876091EAC2000164B50
:10D73000984736235A46D35C23703723D35CA372B1
:10D74000938EA38145E0C046B9C101001FF8FFFFD9
:10D75000ED6F0000F17C00006524010025BB000096
:10D7600089950000B46402004C640200AB0500001F
:10D770005C640200592101000593000021FC0000B7
:10D7800094640200910500007192000022AC200018
:10D79000874B98475B469B8E23805B461B6B636081
:10D7A00036235A46D35C23720C22A35E29AE002294
:10D7B0000292804A01920A21625E00925A46126BDE
:10D7C0005946C96A30007C4CA0470023F55E02230D
:10D7D000F65E38235A46D35CDB073DD44B461888A7
:10D7E0005988DB8801335B1A1BB24A4692880132A2
:10D7F000121A12B2521BD40FA2185210801880B203
:10D800001CAA10809C1BE30F1B195B10C91889B25E
:10D810005180013D45199580731ECB189BB2D38072
:10D82000022F00D19AE05B4600229A5E49461CA86E
:10D83000624B984701246442002801D100F0ABFEFE
:10D840001EAB5A46D26A04991CA85D4DA847200019
:10D850005C4B9847FFF761FB5B4600229A5E002312
:10D86000494629A8584CA047002129A8574B98475A
:10D8700007904B46988801301B88C01A00B2544B61
:10D88000984629009847CB0F59184B1006934B46E2
:10D8900006229B5E9A464B465C885346581C001BEA
:10D8A00000B23100C047CB0F5B185B10E41AA4B282
:10D8B00023B21CAA5380B1B2884601396418D480BF
:10D8C0009A4546DB1400ADB2424B9A463C4E059257
:10D8D0004B46B9461F002AE0002300935B46DB6AF3
:10D8E00022AA04990598D0472388EB181BB22380FD
:10D8F000A288AA18A2804A460421525E9A4208DBF6
:10D90000022FE9D01EAB5A46D26A04990598B04757
:10D91000EAE74B46B9461F00638843441BB2638065
:10D92000E2884244E28006217A5E9A4210DB3B881C
:10D93000069A9B1A9BB21AB22280691E5B18A380BA
:10D9400004217B5E9342E7DB3B004F469946D7E7D5
:10D95000B94607981B4B9847FFF7DFFA012214409E
:10D960001CA8091941801B19C3805B4600229A5EDE
:10D970004946124B9847002816D15B4600229A5E12
:10D980000023494629A8104CA047002129A80F4B85
:10D9900098470400002300935B46DB6A22AA04999F
:10D9A0001CA80C4DA84752E701246442F2E7C04688
:10D9B000ED950000187C00003D3F01009916010024
:10D9C0000593000025BB000001BD000075BA0000F2
:10D9D00085C301003D960000388A18AA1188091AEB
:10D9E00089B211807D8A5488641B548093881B1AE5
:10D9F0009BB29380D088401BD08001335B1A1BB24E
:10DA00000A930B931800B84B98470590B74B98476B
:10DA10000025002806D15B4612255D5F0F3D6A4256
:10DA20006A41D5B25B460021595E4B469B88013363
:10DA30004A4612889B1A4A46D28801324846408894
:10DA4000121A12B21BB2934200DD13005B1009934D
:10DA50008B4200DD0991099B002B00DC84E01AB2A7
:10DA60000023494622A8A24CA047002122A8A14B8E
:10DA700098470F905B461020185E00231AA94C4669
:10DA8000E25C5A540133082BFAD1A1461AAB1A882A
:10DA90005B465B8A59076BD584B21AA912190A80B2
:10DAA0008A88190769D584B21AA9121B8A804A8804
:10DAB000990767D584B21AA912194A80CA88DB0768
:10DAC00065D583B21AA9D31ACB80099B98466A46BA
:10DAD0001383138B9A461A1A12B2012329A8844C75
:10DAE000A047002129A8834B984710905B4610203F
:10DAF0001B5E013B0D934146434500DA0D915B46A9
:10DB0000DB8911936A4693835B465B7D0693002D08
:10DB100000D1BCE11222BB5E4A460221525ED21AFB
:10DB20000D998C46624418A90620095E0C91914219
:10DB300000DD0C921CAA4946098811804946898853
:10DB4000918018A902254D5F5B191BB25380D380C9
:10DB50000C9BAB4200DA9FE01EAC08954B46B146E9
:10DB60005A460E921E0047E001235B420F9381E765
:10DB7000099944186442A4B28FE709994418644291
:10DB8000A4B291E7099944186442A4B293E7099BAF
:10DB9000C3185B429BB295E70422B35E5A1C514600
:10DBA000521A2280A380099A9A1A013210217B5EB0
:10DBB0000EA92820095E5B18D31ADA43D217134046
:10DBC000059A94466344069A02924A460192424656
:10DBD00000926A46928B21000498474DA8471CABDF
:10DBE0005A8801325A80DA880132DA80089A013282
:10DBF00008920C9B93424ADB0B99059D28003F4BF2
:10DC000098477A8A089B9C46624412B2398A0EABC6
:10DC10001B8DC91809B20A9B05952800384DA847E5
:10DC200080461CAB5A886280DB88E3800022B35EAA
:10DC30002380013B5344A380069A02924A460192F4
:10DC40000090059B6A46928B210004982A4DA847B4
:10DC50000623E25E0221735E0E991020095E5B18B6
:10DC60009A4299DA338853442380B38852469B1AE8
:10DC7000A380069B02934B4601930123009300234C
:10DC80006A46928B210004981B4DA84784E7320016
:10DC90004E460E9B9B4691461222BB5E4A4606218B
:10DCA000525ED21A0D99521A18A902254D5F95425B
:10DCB00000DA15000C990A00A94201DB01321500B7
:10DCC0005B191BB21CAA5380D38018AB06229B5E43
:10DCD0009D4200DD99E01EAC08954B46B1465A4680
:10DCE0000C921E0041E0C046A12701006DBB000060
:10DCF00001BD000075BA0000ED6F0000192A010097
:10DD0000D1BA00000422B35E5A1C5146521A228036
:10DD1000A380099A9A1A013210217B5E0EA928204D
:10DD2000095E5B18D31ADA43D2171340059A94465A
:10DD30006344069A02924A460192424600926A461B
:10DD4000928B21000498AF4DA8471CAB5A88013232
:10DD50005A80DA880132DA80089A0132110008927A
:10DD60000EAB2E229B5E99424ADC0B99059D280042
:10DD7000A54B98477A8A089B9C46624412B2398A1E
:10DD80000EAB1B8DC91809B20A9B059528009F4D43
:10DD9000A84780460022B35E2380013B5344A38002
:10DDA0001CAB5A886280DB88E380069A02924A465E
:10DDB00001920090059B6A46928B21000498914D38
:10DDC000A8470623E25E0621735E0C991020095EC7
:10DDD0005B1A9A4296DD338853442380B3885246B7
:10DDE0009B1AA380069B02934B4601930123009349
:10DDF00000236A46928B21000498824DA84781E750
:10DE000032004E460C9B9B4691466B46998E1CAC4D
:10DE10004B465A8801328A186280DB88013B5B1AC4
:10DE2000E3804B4600229B5E23805A46128A013AC9
:10DE30009B18A380069B029301960127009700235D
:10DE40006A46442152181288210004986D4DA84753
:10DE50004A460421525E59460B8AD31A0133238065
:10DE6000A280069B02930196009700236A464421F4
:10DE70005218128821000498A8471098644CA047B3
:10DE80000F98A0470598634B9847FFF764F84B46F7
:10DE90000021595E1CA801804B4604229A5E8280B4
:10DEA00018AB02241C5F7B8A1B191BB24380C38002
:10DEB0005B4612201B5E042B2BD0082B45D0002282
:10DEC00016210EA8844661440A70172161440A7025
:10DED000022B2CD10132143363441A7016230EAA7C
:10DEE000944663441B78002B04D1173363441B789A
:10DEF00001255D4001231D4014AB1D70250018ABAA
:10DF000006229B5E9C42B8DC1CAC3F4B9A46B04656
:10DF100051E00D9A944661441CAA9180002216217A
:10DF20000EA8844661440A70172161440A70012BCF
:10DF300010D0032BD2D1023B16220EA98C4662448C
:10DF40001370172262441370C8E70D99521A1CA966
:10DF50000A80E3E7012216330EA98C4663441A7047
:10DF6000BCE70B99059E3000D0477A8A521912B24D
:10DF7000398A0EAB1B8DC91809B20A9B0596300071
:10DF8000224EB047069A0292424601920090059BAB
:10DF90006A46928B210004981A4EB0476388013379
:10DFA0006380E3880133E38001350EAB2E229B5E54
:10DFB0009D4200DD61E714AB1B78002BD1D11633F5
:10DFC0000EAA944663441B78002B09D00223E25E1C
:10DFD0004B4602215B5E0D998C4663449A42C0DD3C
:10DFE00017230EAA944663441B78002BD6D0022335
:10DFF000E25E4B4606215B5E0D995B1A9A42CDDBD1
:10E00000AFE7C046ED6F0000192A0100D1BA000049
:10E0100025BB0000652401004C2398465B46424620
:10E020009B5E1CAD00260296BC4A01925A464E20C9
:10E03000125E00925A46126C2800B94CA04722ACDE
:10E04000268066802B88013BA3806B88013BE380A0
:10E050001EAD50235A46D25C2B0021004846B14FDA
:10E06000B8472A8848235946CB5AD21892B22388F7
:10E07000D31823806B884A215846415A5B189BB2BB
:10E08000618859186180A1885218A280E2889B1883
:10E09000E38029AD2800A44B98475B461B6C6B605E
:10E0A0005B4642469B5AAB815B4602329B5A6B8170
:10E0B00046235A46D35A2B804423D35C2B720096B6
:10E0C000D36B2A0004992000984CA047FEF74EFF1E
:10E0D000069B01375246BA1A01350799691A09B2E7
:10E0E00012B28A4200DD0A0052109A4200DD069AFE
:10E0F000059B9918099B013308981B1A01340B984A
:10E10000201A00B21BB2834200DD03005B100793AC
:10E110008B4200DD07914B461E8A1AA90B889B1B78
:10E1200098B208804B465C8A4D882D1B4D808B88A9
:10E130009B1B9BB28B80CD882C1BCC8001331B1A80
:10E140001BB21E00089312B2012316A922A8784D13
:10E15000A847002122A8774CA0470E90079F3AB20B
:10E16000002318A929A8A847002129A8A0470F9093
:10E1700009963000704B984705905B4618229B5ECD
:10E180005A46D28A119269460A835A46527F92466B
:10E190000A9A002A00D09BE1013B1093BB4200DAAF
:10E1A00010974B4612229B5E18A902200A5ED21AD3
:10E1B00010988446624414000C921CAA08881080AF
:10E1C000898891801AA90227CF5FDB191BB253807F
:10E1D000D380BC4200DA82E01EAC5B460D932EE099
:10E1E00018AB04229B5E5A1C551B2580A380079AFE
:10E1F0009B1A01334A461021525E0EA93020095E57
:10E2000052189B1ADA43D2171340059A9446634476
:10E2100052460292424601920A9A00926A46128B34
:10E2200021000498454DA8471CAB5A8801325A80FA
:10E23000DA880132DA8001370C9BBB424DDB099949
:10E24000059E30003E4B98474B465A8AD21912B26F
:10E25000198A0EAB1B8EC91809B2089B3000394DC4
:10E26000A8470A901CAB5A886280DB88E38018AB11
:10E270000B9300215B5E23806A46958B013BEB1874
:10E28000A3805246029242460192009033006A46B1
:10E29000128B21000498294EB0470623E25E0B9BA7
:10E2A00002215B5E0D991820095E5B189A4297DA8D
:10E2B00018AA1388EB18238093885B1BA38053460E
:10E2C0000293434601930123009300236A46128B75
:10E2D00021000498194EB04782E70D9B9B464B46A0
:10E2E00012229B5E18AA0627D75FFF1A109ABF1A40
:10E2F0000C990A00B94201DB01321700DB191BB28D
:10E300001CAA5380D3801AAB06229B5E9F4200DD7D
:10E310009AE01EAC5B460B9347E0C046187C0000B9
:10E320003D3F01003D170100ED9500003D960000C6
:10E3300001BD000075BA0000A1270100ED6F0000CB
:10E34000192A0100D1BA000018AB04229B5E5A1CA6
:10E35000551B2580A380079A9B1A01334A4610213A
:10E36000525E0EA93020095E52189B1ADA43D2176A
:10E370001340059A944663445246029242460192E3
:10E380000A9A00926A46128B21000498894DA84788
:10E390001CAB5A8801325A80DA880132DA800137A0
:10E3A0000EAB36229B5E9F424CDC0999059E3000E5
:10E3B000814B98474B465A8AD21912B2198A0EAB32
:10E3C0001B8EC91809B2089B30007C4DA8470A90E3
:10E3D0000EAB28215B5E23806A46958B013BEB18D0
:10E3E000A3801CAB5A886280DB88E380524602928D
:10E3F00042460192009033006A46128B2100049835
:10E400006C4EB0470623E25E0EAB2E215B5E0B998D
:10E410001820095E5B1A9A4296DD18AA1388EB1839
:10E42000238093885B1BA38053460293434601934A
:10E430000123009300236A46128B210004985D4E4D
:10E44000B04781E70B9B9B466B4640229B181B887D
:10E450001CAC18AD6A8801329A186280EA88013AC9
:10E46000D31AE3800022AB5E2380013B5A46128B15
:10E47000D318A38053460293434601930127009784
:10E4800000236A4644215218128821000498494EFC
:10E49000B0470423EA5E531C5946098B5B1A23805C
:10E4A000A2805346029343460193009700236A4695
:10E4B00044215218128821000498B0470E98404C0D
:10E4C000A0470F98A04705983E4B9847FEF7B1FD2F
:10E4D0001CAA18AB198811809B8893801AA9022363
:10E4E000CE5E4B465B8A9B191BB25380D3800622BB
:10E4F0008B5E9E42E2DC314B9B462E4F0999059C78
:10E5000020002D4B98474B465A8A921912B21AADE9
:10E51000198A2B88C91809B2089B05942000D8478E
:10E520001CAC52460292424601920090059B6A46FC
:10E53000128B21000498B847638801336380E38815
:10E540000133E38001360622AB5E9E42D6DDB5E79D
:10E55000079C0C9420001C4B98470A9001220D92B6
:10E56000002C01DDFDF785FE0A98164B9847079FA2
:10E570007F43002F01D1FDF741FF0E9A1100780073
:10E58000944660440B889B0913700231013281422A
:10E59000F8D1FDF733FF5B4600229A5E002349461F
:10E5A00029A80A4CA047002129A8094B9847040034
:10E5B000FFF746F9ED6F0000192A0100D1BA0000FB
:10E5C00025BB000065240100A127010001BD00005A
:10E5D00075BA0000F0B583B004000E00170001AA60
:10E5E00011781F208143117011884048014011802B
:10E5F00000215170A56821781F220A40111F0229AD
:10E600000DD9072A22D0082A34D0092A48D00A2A4C
:10E610005ED00B3A032A15D801AA138012E02078A5
:10E62000C006C00E324B98472368DB025B0D5F4388
:10E63000BE19C008C0B27043281801AB02781A7026
:10E6400042785A7001AB188803B0F0BD32400723FE
:10E650009A1A2068C002400D0730C0104743F610D8
:10E66000ED19AE19317A063B93400B40134101AAD4
:10E670001380E7E7053A3240520006239A1A2068D1
:10E68000C002400D033080104743B610ED19AE199B
:10E69000317C033B93400B40134101AA1380D1E727
:10E6A000012333409B00053AD31A2068C002400D75
:10E6B0000130401047437610ED19AD1940352978E7
:10E6C0000B329A400A401A41130001AA1380B9E79D
:10E6D0002368DB025B0D7B43AD19ED188023DB0063
:10E6E0009C4665442A7801AB1A80ABE71FF8FFFF10
:10E6F000A9920000F0B587B0040001928668007806
:10E700001F230340052B0AD00B2B12D00C2B28D033
:10E710000D2B47D0FF200E2B64D007B0F0BD23682F
:10E72000DB025B0D5A4351184A0051187118887862
:10E73000F3E707250D40043B5D1B2368DB025B0DFF
:10E740000733DB10019A5A43C910B218535C0120F9
:10E75000A84018402841C3B2584258414042C0B274
:10E76000DBE7002302A803705533437055338370F1
:10E77000FF2002ABD87003250D406D0006235D1B02
:10E780002368DB025B0D03339B10019A5A43891007
:10E79000B218525C0323AB4013402B41034002AA42
:10E7A000D05CBAE702AB9C46124B654685CB85C56B
:10E7B0001B682B6001250D40AD0004235D1B236801
:10E7C000DB025B0D01335B10019A5A434910B2180A
:10E7D000525C0F23AB4013402B41FF221340624693
:10E7E000D05C9AE72368DB025B0D019A5A437118EB
:10E7F000885C92E7E0640200F0B5DE4657464E467C
:10E800004546E0B583B004000822835E1B024362E4
:10E810000A22835E1B0283620C23C75E3E4B9B462B
:10E820000A213800984705B20A2676426E43F61947
:10E83000ABB29846584200B2384B9A469847814648
:10E840000135ADB2684200B2D04701905A27424626
:10E85000B81A00B2D04780467D1B28B2D0470700C7
:10E860000A25AD1B4B466B431800019B7343C01830
:10E870000A21D847E06243465D43300078432818B8
:10E880000A21D8472063A07C254B984734260125D0
:10E8900003002B40A05D012290431843A055A07CAB
:10E8A000204B984705406D00A05D02239843054327
:10E8B000A555A27C131F022B28D93421635C0420A8
:10E8C00083436354236823621F2313402376A38862
:10E8D0005B05DA0A144BA1690B401343A361E2887C
:10E8E0005201DB02DB0E13436383E1898020400287
:10E8F000094B9847E086FF23A375238AA38203B0C0
:10E900003CBC90469946A246AB46F0BD3421EBB2E2
:10E91000042003436354D5E7B9C10100A1210100DC
:10E92000D9920000ED920000FF03E0FFF0B5DE4653
:10E9300057464E464546E0B587B000900291059295
:10E940001D0010AB1B889B466A4F0A212800B84760
:10E9500004B2661C0A204042604345192000664B01
:10E9600099469847804630B2C84782465A3420B20A
:10E97000C84704005A3630B2C84781460A26761B7B
:10E980004046704353466B43C0180A21B84780463F
:10E9900074434B465D4360190A21B847119B00221E
:10E9A0009A5E119B0227DF5F54425B465C43241250
:10E9B00024B22300434399467B425D466B431B12BE
:10E9C0001BB24146594396B24D466D1AED13751967
:10E9D0002DB2AA46454665434343BCB20395ED18A4
:10E9E000ED130194A44665442DB2029CA21A5C4624
:10E9F0006243121212B2140044430294611AC91302
:10EA0000711809B244466243049294466344DB138E
:10EA1000019CA44663441BB2059CE71B5C4667430C
:10EA20003F123FB244467C43A0464C464246A41A9D
:10EA3000E2139146B1444A4612B291467843039F8D
:10EA40003F18FF13E34667443FB2029A4446121B45
:10EA5000D2139046464436B2049A94466044C0139A
:10EA60005A46141824B252468A4500DD0A1C101C6E
:10EA700012B24A4500DD4846021C00B2B04200DD39
:10EA8000321C0098028050468A4500DA081C011C9E
:10EA900000B2484500DA49460A1C09B2B14200DA20
:10EAA000321C00998A80291C9D4200DD191C0A1C19
:10EAB00009B2B94200DD3A1C111C12B2A24200DDBB
:10EAC000211C009A51802A1C9D4200DA1A1C131C3A
:10EAD00012B2BA4200DA3B1C1A1C1BB2A34200DA83
:10EAE000221C009BDA8007B03CBC90469946A246A7
:10EAF000AB46F0BDB9C10100A1210100F0B5DE4671
:10EB000057464E464546E0B58BB004003823C75EF5
:10EB1000FF231A003A403A21465E33406F2A7EDCDA
:10EB20003C22815E4942C917803FFFB26F2B00DD56
:10EB300087E03E23E25E5242D3179846803EF6B20B
:10EB4000257DED06EB0E0093A38A5B059B0E0193DA
:10EB5000637DDB080293A37D03933423E35C994632
:10EB60005B0700D481E023684422A25C94465143B1
:10EB7000226C92465144581809AA057815704078BD
:10EB800050700420225E60464243404650430200DB
:10EB9000206C804690449A46C24408A855462D7879
:10EBA000057055466D7845708A189818824607A8F2
:10EBB00055462D78057055466D7845704846800756
:10EBC00000D484E0604601381B18595C89464146F0
:10EBD000595C8A46985CFF21CB1B4A465A439446AF
:10EBE000039A7A4362441212434355467D43AC462E
:10EBF00063441B12DDB2AC460B408D1B6B431140CE
:10EC000071435B181B12A375D2B2052A00D9DCE050
:10EC1000002362460026052A00D9DAE0ABE0902AFC
:10EC20000CDD3C21425E01320421405E0121824222
:10EC300000DB00217F22D71BFFB277E7FF270021EF
:10EC400074E7902B0DDD3E22A35E01330622A05E09
:10EC50000122834200DB002290467F239E1BF6B2F6
:10EC60006EE7FF26002398466AE718239C46A444D3
:10EC700065468BB29B46238A3E21625EA18F594432
:10EC800009B204956046AF4DA946A84709AB188064
:10EC900042466B46DA8292B29046238AE28F424421
:10ECA00012B23C20215E049D2800C84708AB1880A2
:10ECB000238AE28F424412B2A18F594409B228003C
:10ECC000C84707AB18803423E35C9B075BD4FF2362
:10ECD000A3753B00002B00D08DE009AB1D78ED063D
:10ECE000EA0E00921A885205920E01925B78DB08B8
:10ECF0000293002F00D0B7E007AA1778FF06FF0E97
:10ED000013885B059B0E5278D208002E00D1F1E0EB
:10ED1000FF2E00D100E1FF21891B009D75434F4369
:10ED2000EF193D02ED19ED01ED192D01ED0E207DDC
:10ED30001F27B84305432575019870434B43C018FE
:10ED400003021B18DB011B18DB009B0E5B01A08A72
:10ED50007D4D28400343A382029846434A43B61898
:10ED600032029219D2019619F60DF6005B055B0F7F
:10ED70001E436675012318000BB03CBC90469946B3
:10ED8000A246AB46F0BD3E23E25EA18F594409B2D4
:10ED9000049D28006D4B98478146E28F424412B291
:10EDA0003C23E15E2800694B98478246E28F42444B
:10EDB00012B2A18F594409B22800644B98473423FA
:10EDC000E35C9B0700D506E781E76346052B00D887
:10EDD000FF263B00039A052A00D800234A46052A4D
:10EDE00000D8FF235246052A00D80027052800D95D
:10EDF00070E7FF276EE7FF2B00D17AE7FF22D21AD8
:10EE000009A84178C9085143029D5D43AC468C4432
:10EE1000614609026144C9016144C90D1F25AC4620
:10EE20000D40029501884905890E5143019D5D43BE
:10EE3000A84641440D02A84688444546ED01A8462F
:10EE40004144C900890E01910178C906C90E4A439F
:10EE5000009D5D4352191502AD18ED01AD18ED0D81
:10EE600063461D40009544E7FF2F39D0FF23DB1B8D
:10EE7000984608A84278D2087A4307A94B78DB085D
:10EE800045466B43D3181A02D218D201D218D20DBC
:10EE90001F239C461A4003885B059B0E7B439946C3
:10EEA0000B885B059B0E6B434B441D02A94699449E
:10EEB0004D46ED01A9464B44DB009B0E0078C00691
:10EEC000C00E47430978C906C90E40464143791828
:10EED0000F027F18FF017F18FF0D61460F4014E7F6
:10EEE00008AA1778FF06FF0E13885B059B0E527861
:10EEF000D2080AE7257D1F218D432F43277559012D
:10EF0000A38A114803400B43A382D2005B055B0F29
:10EF10001A43627501232EE7237D1F229343009D30
:10EF20001D432575019B5A01A38A07490B401343D2
:10EF3000A382029AD6005B055B0F334363750123FE
:10EF400019E7C046D5E500001FF8FFFFF5E6000011
:10EF5000F0B5CE46474680B585B080466B46D98130
:10EF6000614B198800290CD0604B1F683B0020338F
:10EF700001398AB2D10089188900443179185C4876
:10EF80000CE05C4B00935C4B44225C4902205C4CDF
:10EF9000A047002434E024338B4205D01A68824213
:10EFA000F9DB013A1A60F6E70025564E4E4B9946BA
:10EFB00007E001282AD00135ADB24B461B88AB4291
:10EFC0002FD9EC006419A4003C196068B0470028F0
:10EFD000EFD163684345EED120896B46DB89C01AC7
:10EFE00042424241D0B20028E5D0236A6269944689
:10EFF0006344FA229200934211DD2262002C10D069
:10F00000200005B00CBC90469946F0BD41466068B2
:10F010003D4B9847030058425841C0B2E3E7236292
:10F02000ECE7314B1A88012A13D93B002433023A0A
:10F0300091B2CA00521892004832BA183C0002E05D
:10F040002433934206D0196A206A8142F8DA1C0000
:10F05000F6E73C006368002B25D020002B4B984737
:10F060002B4B0093244B772224490120244DA847A1
:10F07000284B98470500002363616B46DA894146B7
:10F080002000254B9847002816D00023236263698F
:10F09000002BB5D12800214B984760610028AFD1E3
:10F0A00001236361ACE71E4B0093134B7A22134993
:10F0B0000120134DA847DBE71A4B00930E4B832228
:10F0C0000E4902300E4DA8472000104B98472021D2
:10F0D0002000154DA84724212000A84780231B06A7
:10F0E000236200248CE7C046C62B0020E04D0020A0
:10F0F0000200008054650200F06402001C650200FA
:10F100005921010089950000E5C601005DFD000060
:10F110007C650200F90E010075FC0000150F01006E
:10F12000B0650200E465020075290100F8B5D64615
:10F13000474680B50700154B1B689846144B1B8843
:10F14000002B1ED00025134B9A46114E0FE0002BCA
:10F1500002D02000104B984720212000D0472421C6
:10F160002000D0470135ADB23388AB4209D9EC005D
:10F170006419A40044446368BB42E8D0002FF1D175
:10F18000E5E70CBC90469A46F8BDC046E04D00202D
:10F19000C62B0020752901005DFD0000F0B5C646B4
:10F1A00000B582B00400244B1B68002B06D0002061
:10F1B000224B9847204B1868214B9847E0000019D4
:10F1C0008000204B98471C4B18601F4B9847002825
:10F1D00020D0194B1B68002B2AD01C4B1C80002C04
:10F1E00014D00024144F1A4E9846E5002D19AD0096
:10F1F0003B6858192021B0473B6858192421B04773
:10F200000134A4B243461B88A342EED802B004BC2A
:10F210009046F0BD0F4B0093A8220F4903300F4CCE
:10F22000A047054B1A6800230D480E498847FEE7A2
:10F230000022064B1A80E9E7E04D00202DF1000086
:10F24000C9230100DD220100AD170000C62B0020FC
:10F2500075290100046502001C65020059210100A6
:10F2600054580200B517000030B587B00C001500E7
:10F270000800384B9847002821D12378DB06DB0EA5
:10F28000043BDBB20A2B28D82368DB025B0D9B0210
:10F29000314A29680A4013432B6063885B095A018D
:10F2A00069881F230B4013436B802378DB06DA0E3B
:10F2B0002B781F218B4313432B7001300DE0012865
:10F2C0000DD0022836D0254B0093254B9A225200B0
:10F2D00024490220244CA047002007B030BD022260
:10F2E000210004A8214B984700280AD02B78DB0680
:10F2F000DB0E1C331F22134001200A2BEDD9002006
:10F30000EBE703AB0422290004A8194CA047040032
:10F3100004A8184B9847002C02D1039B042BE5D07E
:10F32000154B00930E4B2222FF320E4902200E4C49
:10F33000A047E4E7084A2B681A408023DB00134308
:10F340002B6020226A80C03213400B2213432B70A3
:10F350000138C2E789950000FF03E0FF5C67020007
:10F36000506602000067020059210100251C0100BF
:10F37000891B0100591B01003867020070B50D00A0
:10F38000CC69002C16D02068002804D00A4B98477E
:10F3900020680A4B98476068002801D0074B9847BF
:10F3A000A068002801D0054B98472000034B9847E0
:10F3B0000023EB6170BDC046591B0100C923010049
:10F3C000F0B5DE4657464E464546E0B587B00600E6
:10F3D0000C008B7A012B19D0002B00D0AEE14B68CA
:10F3E0009B68002B00D1A7E1087BC006C00E031F5D
:10F3F000022B00D988E063689B682361012007B075
:10F400003CBC90469946A246AB46F0BD4868D14BFD
:10F410009847D149D14B984700282ED102226168E4
:10F4200004A8CF4B984700281ED1E369002B26D0B3
:10F43000E5690820CB4B98472860CB4B98470028BC
:10F4400044D02A68002304A9002A4DD1C74B009359
:10F45000C74B6022FF32C7490320C74DA847210090
:10F460003000C64B984708E0C54B0093C04BA6221E
:10F470005200C0490220C04CA0470020BFE70C202A
:10F48000B84B9847E061B84B984700280DD1B84B6E
:10F4900000935422FF32B7490330B74DA847E269C1
:10F4A0000023B848B8498847FEE7E069002809D139
:10F4B000AE4B0093AE4B5622FF32AE490330AE4CFA
:10F4C000A047DAE70C21B14B9847B1E7A84B00936E
:10F4D0005E22FF32A7490330A74CA0472A680023C9
:10F4E000A848A9498847FEE7585CD0540133082B47
:10F4F000FAD1207BC006C00E031F022B04D8A37ACA
:10F50000002B00D177E720E1C31F032B07D90B386D
:10F51000032800D901E10023236101206FE79C4B00
:10F5200098470700E369002B17D0E5690220B8402F
:10F530008C4B984768608C4B9847002839D18C4B8E
:10F5400000939822FF328B4903308B4CA0476A68A6
:10F5500000238C488C498847FEE70C20814B984754
:10F56000E061814B984700280DD1814B0093C62262
:10F57000520080490330804DA847E269002381484A
:10F5800081498847FEE7E06900280ED1774B009358
:10F59000774BC722520077490330774DA8472100A7
:10F5A0003000764B9847002029E70C21774B98478D
:10F5B000BBE70123BB401F0018006A4B9847A860B7
:10F5C000694B9847002847D06B68002B52D0AB6836
:10F5D000002B4FD0A37A012B5BD063689868002F73
:10F5E00000D196E0002398463F339B46203B994646
:10F5F000684B9A46414603944A006B689C466244B5
:10F6000043789C0802948678F6084C462640047895
:10F61000E408A44614784B469C43A04664464346FF
:10F620001C4314705B46029C1C4063019C4613887B
:10F6300054462340644623431380F6001B0A0724E4
:10F64000234033435370C378AA68535401310430C4
:10F650008F42D1D1039C5CE0454B00939A22FF324C
:10F6600044490330444CA047AA6800234548464912
:10F670008847FEE73D4B00933D4B9C22FF323D49BE
:10F6800003203D4DA847210030003C4B9847002007
:10F69000B5E604212868404B9847002F39D0002355
:10F6A00098463E4B9B463F239A46203B9946230073
:10F6B0004446984604AE0023042231002868D84707
:10F6C00062006B689C466244737898080390B17836
:10F6D000C9084846014002913078C00811784B466D
:10F6E000994308431070534603981840400113880B
:10F6F00028490B40034313800299C9005B055B0F47
:10F700000B435370F378AA6813550134A742D1D143
:10F71000444600232361012071E621003000174B8D
:10F7200098471F4B0093124BD422FF3211490220FD
:10F73000114CA047002062E6002060E6087BC0066E
:10F74000C00E031F022B00D9DEE600232361012037
:10F7500055E6C046091D010084670200E5C60100A8
:10F76000251C0100DD220100AD170000B467020076
:10F770007066020000670200592101007DF300005D
:10F780008867020054580200B5170000752901006F
:10F79000A99200001FF8FFFFCB1B0100891B01008D
:10F7A000E0670200F0B5DE4657464E464546E0B5F6
:10F7B0008DB00D001700039316AB00269E5F0A7BE9
:10F7C0001F2313401A1F022A46D88B7A0020012BD0
:10F7D00006D00DB03CBC90469946A246AB46F0BD63
:10F7E000CB699946087BC006C00ED64B9847804629
:10F7F000E968C902490D039B4B43D9194143C9101C
:10F8000004314B461868D04B984700281AD143461C
:10F81000DB08DBB25E43002308934B46186808AB55
:10F8200032001799C94CA0470120089B9E42D0D0B6
:10F83000C74B0093C74BC84AC8490130C84CA047C2
:10F840000020C6E7C74B0093C24BC74AC3490220FA
:10F85000C34CA0470020BCE71A000B3A032A0ED97C
:10F86000073B032B00D8F6E0C04B0093C04BFE22B1
:10F870005200BA490220BA4CA0470020A9E706ABC3
:10F8800000211970FF225A7007AB19705531597059
:10F8900055319970DA7008AAB64B13CB13C21B68A6
:10F8A00013602989002E11DD080A179C721E92B27E
:10F8B00001329446520062442300A4466244039CF1
:10F8C0001970587003339A42FAD10394287BC0060A
:10F8D000C00E9C4B9847814601238340013B9BB25D
:10F8E00098462B7BDB06DB0EDAB20C2A4DD011D901
:10F8F000DAB20D2A5FD00E2A72D1EB68DB025B0D03
:10F9000099B21BB20493039C4C43E41900270023D3
:10F910009A4615E00B2A63D1EB68DB025B0DDA1027
:10F92000511C04915B0701D113B20493049B039C07
:10F930005C43F91064180723BB431F0006AB9A46CB
:10F94000EB699B4604988C4B98470590AB7A002B4B
:10F9500050D16B6899680C19002E77DD179B991CA4
:10F96000013EB6B27000801905309C4660441F26E7
:10F97000FF239C4608234A469B1A5BB20393CB465F
:10F980002B000500404698464CE0EB68DB025B0D1F
:10F990009A10511C04919B0701D113B20493049B4C
:10F9A000039C5C43B9106418BBB203279F437F00DC
:10F9B00007AB9A46C4E7EB68DB025B0D5A10511C9B
:10F9C0000491DB0701D413B20493049B039C5C43B2
:10F9D00079106418FB0709D5002708AB9A46AFE7F2
:10F9E00000270024002304939A46A9E7042708ABC4
:10F9F0009A46A5E7211D5B461868534B98475B461E
:10FA000018680023049A0599504CA047059CA3E769
:10FA1000DBB20B705B46FF1A7FB2002F13DB0331A2
:10FA2000A94213D0237899460300BB404A461340AD
:10FA30003B414246127B32400E2AE9D062461340D7
:10FA40005246D35CE5E7039F0134E8E705984B4B4A
:10FA500098470120BDE6087BC006C00E394B984789
:10FA6000814601238340013B9BB298462B7BDB06FA
:10FA7000DB0EDAB2082A4DD015D9DAB2092A00D144
:10FA80007EE00A2A00D093E0EB68DB025B0D9AB2BD
:10FA90001BB29A46039C5443E7198023DB009B4624
:10FAA000BB44002416E0072A00D081E0EB68DB02AB
:10FAB0005B0DDA10511C8A465B0701D113B29A46DE
:10FAC0005346039C5C43FB10E41808239B46A34465
:10FAD0000724BC43EF695046274B98470490AB7A04
:10FAE000002B6AD16B6899685944002E00DC8BE0CA
:10FAF0001798013EB6B2013673009E1984466644DB
:10FB0000FF239A4608224B46D21A53B20393B446B7
:10FB10004E4662E0EB68DB025B0D9A10511C8A4690
:10FB20009B0701D113B29A465346039C5C43BB101A
:10FB3000E41810239B46A344BFB20324BC436400D3
:10FB4000C8E7C046A9920000CB1B0100891B010039
:10FB500030680200B466020035020000006702004F
:10FB6000592101000C6802002E02000054680200B6
:10FB70009066020010660200A127010065240100C2
:10FB8000EB68DB025B0D5A10511C8A46DB0701D47F
:10FB900013B29A465346039C5C437B10E4184023FF
:10FBA0009B46A344012427407C427C41A40091E76A
:10FBB00000239B4600249A468CE759460431386856
:10FBC000144B98470023524604993868124DA847B1
:10FBD00004998AE70330604516D00A784346A3406B
:10FBE00013402341524613405A007D68525B027015
:10FBF000120A4270BA68D35C8370A41B64B2002CF2
:10FC0000E8DA039C0131E5E70498044B98470120AA
:10FC1000DFE5C046CB1B0100891B01006524010004
:10FC2000F0B583B001900D000A781F2313400B70CC
:10FC30000D480E4B9847041E14D00D4E05E00027CA
:10FC400021000948B047041E09D02368002BF6D0D4
:10FC50002A0001992000984707000128F0D13800B8
:10FC600003B0F0BD0027FAE72C4D0020851E0100EF
:10FC70009D1E0100F0B583B00700009102810800CD
:10FC8000254B9847B8720023FB6101280ED0009BDA
:10FC90007B602248224B9847041E36D000250C2357
:10FCA0009C46BC44634601931E4E10E0009C20001D
:10FCB0001D4B984701301D4B9847786021001C4B25
:10FCC0009847E6E721001548B047041E18D023687E
:10FCD000002BF7D06268002AF4D0019A0099200026
:10FCE000984705000128EDD10023BB613B613C60D2
:10FCF000390020006368984705000128E2D101E03F
:10FD0000002D03D0280003B0F0BD002520213800CD
:10FD1000084B9847F6E7C046899500002C4D002017
:10FD2000851E01009D1E010009C70100DD220100A2
:10FD3000F9C601007529010070B582B00568AC688C
:10FD4000002C09D0069E0196009313000A000100C2
:10FD50002800A04702B070BD0020FBE710B50400EA
:10FD60000068002807D0C368002B01D02100984705
:10FD7000A37A012B00D010BD6068024B9847002386
:10FD80006360F8E7C923010030B583B00E480F4B1C
:10FD9000984704000E4B9847002808D0002C03D049
:10FDA000102120000B4B9847200003B030BD0A4BB8
:10FDB0000093C92209490330094DA84722000023B6
:10FDC000084809498847FEE72C4D0020E51D010041
:10FDD000AD170000752901003866020000670200B7
:10FDE0005921010054580200B517000010B582B027
:10FDF00010211548154B9847154B9847002809D0F6
:10FE0000144B0360144B4360144B8360144BC3606A
:10FE100002B010BD134B0093134B4722134902301D
:10FE2000134CA0470020134B98470028F0D10E4BED
:10FE3000009348220D4903300D4CA04700220023B7
:10FE40000D480E498847FEE72C4D0020D11D0100CA
:10FE500089FD000069F20000C1F30000A5F7000071
:10FE60007DF30000DC6602002066020000670200ED
:10FE700059210100AD17000054580200B5170000C9
:10FE800010B54368984710BD10B50468A04710BD71
:10FE900010B584B013000A0001A9054CA047002347
:10FEA000002801D001AB1B88180004B010BDC0466B
:10FEB00089FE000003780A78934201D0981A7047AF
:10FEC00040784B78C01AFAE703880A88934201D039
:10FED000981A704740884B88C01AFAE700880B8848
:10FEE000C01A7047F0B587B00C000B1E18D0066919
:10FEF000B369994217D0728A9205920D002A62DD89
:10FF0000B7683B68C81A0590BB8898420DD8002393
:10FF10000393BA7C002A1AD1FB881B18B461F361E1
:10FF2000180007B0F0BDF369FAE70021013189B28A
:10FF3000914248DA8B005B189B000393FB1818680A
:10FF4000201A05909D88A842F0D81F00E1E7012AF9
:10FF50001BD0022A1ED00023032ADFD13A8AB968B7
:10FF60001B4B0093022305A81A4FB847002828D03E
:10FF7000039BB268944663441D009B68C01A400806
:10FF8000EB68185CEB88C318C8E7FB68185CFB8853
:10FF9000C318C3E73A8AB9680D4B0093022305A83A
:10FFA0000C4FB84700280AD0039BB26894466344BC
:10FFB0001D009B68C01A4008EB88C318AEE70023F9
:10FFC000ACE70023AAE7B4610023F361A8E7C046C9
:10FFD000DDFE00006D400100F0B5DE4657464E469E
:10FFE0004546E0B59BB009291CD00569D04B984720
:10FFF000002801D100F0E7FCC0006B681E182B7DC3
:020000021000EC
:100000009B0711D1002E01D100F0E0FC3068000305
:10001000030B2868C0181BB03CBC90469946A2460A
:10002000AB46F0BD1731E0E7337974795C43002CBF
:1000300001D100F0CEFCEB7C9B061B0FDAB2022A4A
:1000400000D18DE008D9DAB2032A00D18BE0042A6E
:1000500004D10134640801E0012A7ED0B54B186850
:10006000B54B984784420FD9B24F21003868B34B43
:1000700098473860B24B9847002877D0AD4B1B6843
:10008000002B01D100F0A8FC33681B031B0B2A686E
:10009000D218A84B1B68059333790F931BB21393A7
:1000A000737912931BB21093EB7C9B061B0FD9B292
:1000B00002910891032967D0A2490A60A24A1370ED
:1000C0000023A24A1370A24A1360A24A1370A24AE4
:1000D00013700F9F3800A14CA047050019903800FD
:1000E000A0470390139B002B00DC6AE2994B1B781E
:1000F0000493994B1B789A46924B1E68944B186850
:10010000914B1B789946012349468B40013BDBB25A
:100110000D9308235B1A0E9310235B1A0C938B4BE1
:100120001B789C462C003B00013B9BB20133119392
:100130002A009B465A440B92002307930A930021FE
:1001400009934B469B009B46854B5B441493534657
:100150000693A84667464D4638E00734E4087DE735
:100160000334A4087AE70134640877E77D4B0093F1
:1001700072227D4903307D4CA0476E4B1A680023E4
:100180007B487C498847FEE70131089194E70323C7
:100190009C46C308072101404A19072A2FD8F35C5F
:1001A0000E9A511A0B4162461A401300002802D0E1
:1001B000049A934231D040190493012101220992FB
:1001C000237001340B9B9C4200D150E1002F2CD1B5
:1001D0004B46082B0DD8684B5A469B5809939F46AF
:1001E00007239C46D5E70F239C46D2E7FF239C4676
:1001F000CFE70D9B9C46CCE701239C46C9E7F25C08
:1002000012029246F3185B7853449BB20C9A511A2F
:100210000B4162461A401300C8E7012207920022F0
:10022000069201320A920127C5E7012F11D000235F
:10023000022FC5D1069A013AD3B20693002B00D003
:1002400011E14B46082B00D9F6E0149B1B68049380
:100250009F46C308072101404A1C072A15D8F35CB2
:10026000C94308310B4101221340069A0132D2B230
:100270000692411C012B15D04B46082B00D9B0E04B
:100280003E4B5A469B5804939F46F25C120294469A
:10029000F3185B7863449BB2C94310310B410122D0
:1002A0001340E2E70B2A05D00800049B01220792C5
:1002B000012185E7CB08072211408A1D072A13D8A0
:1002C000F25C0223591A0A413D331A400692073064
:1002D000069B002B00D0BFE04B46082B24D8284BB0
:1002E0005A469B5804939F46F25C1202F3185B78BF
:1002F0009A1892B20A23591A0A4135331A400692C3
:10030000E5E70323C708072101404A19072A39D81E
:10031000F75D0E9A511A0F413B403EE00723F1E78B
:100320000F23EFE7FF23EDE70D9BEBE70123E9E761
:10033000E5FE0000C82B002045240100FD26010039
:10034000AD170000D02B0020CC2B0020DC2B002090
:10035000D82B0020D42B0020CD2B0020A12701007A
:10036000B4680200F06902000C6A02005921010021
:1003700054580200B517000090680200D8680200C7
:10038000FC680200F25D12029446F7197F78674418
:10039000BFB20C9A511A0F413B40401904930122FD
:1003A00007920A9200270121099209E70323CF0847
:1003B000072008404219072A17D8F75D0E9A101A2D
:1003C00007413B4048190493012207920A920027F3
:1003D00001210992F4E60723E9E70F23E7E7FF236A
:1003E000E5E70D9BE3E70123E1E7F25D12029446A6
:1003F000F7197F786744BFB20C9A101A07413B4047
:10040000E0E70323C708072101404A19072A17D844
:10041000F75D0E9A511A0F413B4040190493012297
:1004200007920A92002701210992C9E60723E9E70A
:100430000F23E7E7FF23E5E70D9BE3E70123E1E770
:10044000F25D12029446F7197F786744BFB20C9AA6
:10045000511A0F413B40E0E7049B012207920A92A8
:1004600002270121ACE6049B01220792A8E6069B25
:100470009A464546BC46099B002B14D1002901D061
:10048000CC4B18600A9B002B02D0CB4B62461A70F3
:10049000079B002B02D0C94B52461A700026029BC4
:1004A00004932F0023E0C64B6A46127C1A70E5E7DE
:1004B000042300220721314008256D1AED1A71032B
:1004C000090C059884466144012098400300013BD3
:1004D000DBB2DB43AB4008780340AA401A430A7002
:1004E000089A1300944666440137A74221D03A780F
:1004F000049B02990329DDD1072A18D89200B14B39
:100500009B589F4604230222D4E704230422D1E708
:1005100004230622CEE704230922CBE704230B227F
:10052000C8E704230D22C5E704230F22C2E70423F2
:10053000C0E7119A5A431192109B012B00DC34E260
:10054000A14B1B681E00A14B1B781A000B930123C3
:100550009340013BDBB214939246984B1B7898462C
:1005600008239B1A0E9310239B1A1093944B1B780D
:100570000493904B1868904B1978129B023B9BB2E6
:1005800001331593089C06940F9B013B9BB21D0001
:10059000169323006B431793002312930D930F932D
:1005A00009930A9393000C93894A9C4662441892DB
:1005B000139B9B4643460893199B1D008C46B146EE
:1005C000CFE100231193B7E7032308E0072306E0F8
:1005D0000F2304E0FF2302E0149B00E00123C50881
:1005E000072202409719072F1FD84F467D5D0E9FA7
:1005F000BA1A15412B40DBB2002802D0049A9A4265
:1006000021D080190493012209920A9223700134A7
:10061000644500D141E100291DD10B9B082BDBD89B
:100620000C9B6C4AD35807939F464F467F5D3F0211
:10063000BA464D446D785544ADB2109FBA1A154173
:100640002B40DBB2D8E701220D9200220892013242
:100650000F920121D5E7012911D000230229D5D11C
:10066000089B013BDBB20893002B00D011E10B9BF0
:10067000082B00D9E0E0189B1B6804939F46C30831
:1006800007220240551C072D16D84D46EB5CD2437D
:100690000832134101221340089A0132D2B2089263
:1006A000451C012B15D00B9B082B00D980E04A4B31
:1006B0000C9A9B5804939F464D46ED5C2D024B448B
:1006C0005B785B199BB2D243103213410122134075
:1006D000E2E70B2A05D02800049B01220D92099223
:1006E00094E7EB0807221540AA1D072A14D84A46AA
:1006F000D35C0222551B2B413D321A400892073031
:10070000089B002B00D0BDE00B9B082B34D8334B4B
:100710000C9A9B5804939F464A46D25C12024B4463
:100720005B789B189BB20A22551B2B4135321A402D
:100730000892E4E703239A46C508072303409A1961
:10074000072A1FD84A46525D0E99CB1A1A415346C2
:100750001340DBB28019049301220D920F92002105
:1007600009920A9252E707239A46E5E70F239A4631
:10077000E2E7FF239A46DFE7149B9A46DCE7012372
:100780009A46D9E74A46515D09024D446A785218A3
:1007900092B21099CB1A1A4153461340DBB2D9E7F3
:1007A00003231EE007231CE00F231AE0FF2318E0B9
:1007B000149B16E0D82B0020DC2B0020CD2B002032
:1007C000D42B002020690200D02B0020CC2B00204D
:1007D000646902004069020088690200AC69020095
:1007E0000123E90807222A40901907280FD8484614
:1007F000415C0E98821A11410B40DBB2A819049398
:1008000001220D920F92002109920A92FEE64846BB
:10081000405C000249444978091889B21098821A4C
:1008200011410B40DBB2E9E7032308E0072306E0B0
:100830000F2304E0FF2302E0149B00E00123C10822
:10084000072202409519072D0FD84D46695C0E9D71
:10085000AA1A11410B40DBB28019049301220D92B8
:100860000F92002109920A92D0E64D466D5C2D024E
:1008700049444978491989B2109DAA1A11410B407F
:10088000DBB2E9E7049B01220D920F92022109924B
:10089000BCE6049B01220D92B8E68C46B246119943
:1008A0000027029B07930300404662461392984636
:1008B0001EE00423002407220A400826B61AF61A6E
:1008C0004D032D0C059A9446654401229A4013006D
:1008D000013BDBB2DB43B3402A781340B4402343EF
:1008E0002B70069B9C46614401373BB29B4525DD3E
:1008F000039BDC5DC35D5C40C455079B029A032AE1
:10090000D9D1072C18D8A400354B1B599F46042376
:100910000224D0E704230424CDE704230624CAE7F5
:1009200004230924C7E704230B24C4E704230D246C
:10093000C1E704230F24BEE70423BCE70500139A94
:1009400094464046179B069A90464344119A904617
:10095000984443461193129B01331293159A934284
:100960000DD05B46002BF6DD039B98461C00169BC2
:100970005E1C4644A8466146B44656464BE6089B74
:10098000984661460A9B002B18D1099B002B01D089
:10099000144B18600F9B002B01D0134B19700D9B4B
:1009A000002B02D0114B42461A701998104CA047E8
:1009B0000398A0470F4B1868FFF72DFB0E4B6A46B4
:1009C000127C1A70E1E70020FFF725FB0020FFF7FB
:1009D00022FB0020FFF71FFB0020FFF71CFBC04697
:1009E000D0690200D82B0020DC2B0020CD2B00206A
:1009F00065240100C82B0020D42B0020F0B5DE4672
:100A000057464E464546E0B585B081460C001F006E
:100A10000025092A3AD04B461E6911004846534B1F
:100A200098478346002800D194E0F368002B00D15A
:100A30008EE0390048464D4B98470023002828D1C6
:100A40005A46D000726894466044328A5A43121162
:100A500041880909002D00D04900130008335B18B4
:100A60001B0923804379A380027962800623C35641
:100A7000E3800723C3562381F37C9B061B0FA372DD
:100A8000002D00D16FE05200628064E00135173222
:100A9000C1E74B461B69DA7C520642D4DB689846B4
:100AA000DB7A03221A401CD00023012AC8D1434616
:100AB0001B68994600025844039043469B681A02FB
:100AC000120A2B4B00930423494603A8294FB84729
:100AD000002824D04B46C01A000943465B681B56C9
:100AE000AEE743461B68994603AB9C460002584458
:100AF000188043469B681A02120A1F4B0093022378
:100B0000494660461B4FB847002806D04B46C01ADE
:100B1000400843465B681B5692E7002390E700239A
:100B20008EE7DA6853685946595C0023002987D05C
:100B30009368185C0023002800D181E70139537BBA
:100B40004B4311680918C91801390023CB5677E7C0
:100B5000002375E70025280005B03CBC9046994667
:100B6000A246AB46F0BD0125F5E7C046E5FE000014
:100B7000C9FE00006D400100B5FE000010B5054B38
:100B80001868002804D0044B98470022014B1A60D3
:100B900010BDC046C82B0020C923010010B50400B9
:100BA0002C21154B98470022E260F0235B00238044
:100BB000D03B63806260237A02218B43237226310B
:100BC000635C1F2083436354218DFC23DB000B43B4
:100BD0002385210028315B055B0F4B702389074972
:100BE000194082239B000B43238101210B43237275
:100BF00022626262626110BD7529010003F0FFFF8D
:100C0000F8B504000D0017001E002421034B98477F
:100C100025606760A560E660F8BDC04675290100E3
:100C200070B582B005004048404B9847041E56D02E
:100C3000B82149003E4B98472C22290020003D4B0B
:100C40009847200030304C213B4B98470022B62378
:100C50005B00E250394B1B68002B52D0374B1E68AB
:100C60001C60230003221E213548364DA847E06250
:100C7000354B9847002847D0E36A002B51D0B42267
:100C80005200A35A9B0A9B02A3520022B6235B0088
:100C9000E250002100202D4DA847E06300210020F4
:100CA000A847206400210020A84760640021206C30
:100CB000274DA8470021606CA8470021206C254DD6
:100CC000A8470021606CA847E06B234B98471B4B5B
:100CD0001E60E06A214B9847200002B070BD0020E2
:100CE000194B98470028F7D11D4B00937C221D49D2
:100CF00003301D4CA047002200231C481C49884794
:100D0000FEE70E4B1C60A9E7154B00938D22154999
:100D10000330154DA847E26A002314481449884758
:100D2000FEE70024D8E7C046204D0020E51D010065
:100D30007529010045250100D11D0100E02B00208F
:100D40009D5500001D390100AD17000095330000CE
:100D500005310000A51E0000692800008D39010042
:100D6000F0A6020008A70200592101005458020011
:100D7000B5170000014B18687047C046E02B0020F3
:100D8000031E05D01A7A920709D50220185E704713
:100D9000044B1B68F0204000002BF8D0F2E7002045
:100DA000185EF4E7E02B0020031E05D01A7A9207A4
:100DB00009D50020185E7047044B1B68882040004E
:100DC000002BF8D0F2E70220185EF4E7E02B0020B9
:100DD000031E03D018890005800D7047024B1B6865
:100DE0008220002BF9D0F5E7E02B002070B5051E1E
:100DF00019D028000F4B9847040028000E4B984745
:100E00000100A000001940000C4B98470200002090
:100E10001D2A07D90130312A04D94430904280413B
:100E20004042023070BD064B1D68F0246400002D66
:100E3000E3D0DEE7810D0100D10D0100A5C0010066
:100E4000E02B00204268002393614268D361704721
:100E500010B5002804D001000348044B984710BD8A
:100E60000148034B9847FAE7204D00209D1E0100E2
:100E7000851E01004068704743681A68002A04D044
:100E80005868431E9841C0B270470020FCE700003C
:100E900010B50400074B984700280AD00022A35E33
:100EA0000222A05E58436368DB68C01A434258417F
:100EB000C0B210BD790E010010B5002804D00100A9
:100EC0000348044B984710BD0148034B9847FAE785
:100ED000144D00209D1E0100851E01000022044BC0
:100EE0001A70044B1A689446604418607047C046F4
:100EF000E82B0020E42B0020044B012119701A7804
:100F0000002AFBD0024B18687047C046E82B00202F
:100F1000E42B002010B50400014B9847001B10BDC6
:100F2000F90E010010B50C00096A606A81420AD00E
:100F30008002064B9847A369E269D21A5043801297
:100F4000181800B210BD8020C000F4E7A5C0010051
:100F500010B50122094B1A7009480A4B984700281E
:100F600005D0094B18680421084B984710BD064B63
:100F700018680021054B9847F8E7C046F02B002081
:100F8000E44D0020851E0100EC2B00208D3801006F
:100F9000F0B5CE46474680B591B06548654B984759
:100FA00000280BD03C25624C634E435D02229343E4
:100FB000435501002000B0470028F6D15F4B186868
:100FC0005F4B984707005A485A4B9847041E00D178
:100FD0008CE05C4E0025B04626E0DB19002B00DAE1
:100FE0008DE0A268002A00D190E02000904728E020
:100FF0002369002B2FD02000103021009847636810
:10100000002B02D001B220689847636A226A93429B
:1010100027D243461B78002B00D171E04448454B52
:1010200098470400002C61D035703C23E35C9B079B
:1010300066D43C22A35C02210B43A354636A002BB9
:10104000CBDD636AFB186362002BE2DB226A9A4203
:10105000CED26262CCE72000103021003A4B984794
:10106000CDE73C23E35C01221340181E07D1A28E7A
:10107000002A4DD035498A4251D0013AA286A28E2B
:10108000002A1AD0236B5A426262E26A002AC0D058
:10109000002840D04342434199463C20215C012333
:1010A00099434B460B432354A169E069A061E16178
:1010B000DB0700D4A26B2262ABE7E26A002A01D010
:1010C000002828D0402221006846214B9847210063
:1010D0001748204B984720001F4B98471F4B9847B5
:1010E000039B002B95D06846984792E71C4B984786
:1010F000124B186011B00CBC90469946F0BD63626B
:1011000021000B480C4B984704008BE763629DE776
:10111000E26A002AD6D0A36A59426162BAE7236B19
:101120005A426262E26A002A00D172E7F3E7C046DF
:10113000E44D0020851E01009D1E0100F42B0020BF
:10114000150F0100F02B0020250F0100FFFF00000C
:10115000452501006D1F0100C9230100510F010049
:10116000F90E010010B540210A480B4B98470B4B74
:1011700098470B4B1860002304221E2109480A4C93
:10118000A0470A4B18600A4B98470022094B1A7077
:1011900010BDC046E44D0020D11D0100F90E010034
:1011A000F42B0020910F01001D390100EC2B0020D1
:1011B000510F0100F02B002010B5040040210D4B11
:1011C0009847FA235B0023620023A3616433E36141
:1011D000094B1A7822745A7862749A78A274DB7870
:1011E000E3740123A3863622A35C01210B43A3549D
:1011F00010BDC046752901004CA70200F0B5D646C7
:1012000000B582B006008A461548164B9847041E62
:101210001ED000230193144F0CE021001048134B03
:1012200098472000124B9847124B9847012301938F
:101230002C1E0FD021000A48B84705002368B3428E
:10124000F6D163685345E8D05346002BF0D1E4E76C
:1012500000230193019802B004BC9246F0BDC04641
:10126000E44D0020851E01009D1E01006D1F010040
:10127000C9230100510F010030B583B0050041685A
:10128000002902D000681E4B98471E481E4B984705
:10129000002821D11B481D4B984704001C4B984740
:1012A00000281FD0002C15D02B6AAB6340222900E8
:1012B0002000184B98473623E35CDB0708D56368AA
:1012C000002B05D02068002802D01822A15E984784
:1012D000114B984703B030BD104B98470138104B65
:1012E0001860D7E70F4B00936A220F4903300F4D68
:1012F000A847220000230E480E498847FEE7C04653
:10130000FD110100E44D00202D210100E51D01002B
:10131000AD17000045250100510F0100F90E010035
:10132000F42B00203CA7020054A702005921010021
:1013300054580200B5170000F8B504000F000A4821
:101340000A4B984700280DD0074E094D04E00100D4
:101350003000A847002805D00368A342F7D14368AE
:10136000BB42F4D1F8BDC046E44D0020851E01000B
:101370009D1E010010B50300891ACA178918514033
:10138000FA20800048431900054B9847054B9842C6
:1013900000D91800002800D1013080B210BDC0462D
:1013A000B9C10100FFFF000070B50023C65E042331
:1013B000C25E921BD40FA4186410A5B224B20B888D
:1013C0009B1B5B1B1BB24A884188521A521B12B2EC
:1013D00064435B4352439B18E017DA0F9C42504131
:1013E000C0B270BD4B1E4188C918C180704704232C
:1013F000C25E0021435ED21A01320621435E022101
:10140000405E181A013050437047F0B5C64600B52B
:101410000D8813881C1C1BB22EB2B34200DA2C1CA0
:1014200026B204804D8853881C1C1BB22FB2BB42CD
:1014300000DA2C1C27B244808D8893881C1C1BB2B8
:1014400098462BB2984500DD2C1C25B28480C988B3
:10145000D3881A1C1BB20CB2A34200DD0A1C13B2C3
:10146000C2800020AE4204DCF80FDA17BB425041C4
:10147000C0B204BC9046F0BD70B50D8813881C1C2A
:101480001BB22EB2B34200DD2C1C04804D88538861
:101490001C1C1BB22EB2B34200DD2C1C44808D8874
:1014A00093881C1C1BB22EB2B34200DA2C1C848021
:1014B000C988D3881A1C1BB20CB2A34200DA0A1CDA
:1014C000C28070BDF0B5DE4657464E464546E0B593
:1014D00085B00E000023CC5E0023C15E00238C4249
:1014E0005EDB0425435F98460023444558DC022315
:1014F000F45E0225435F9A460023544550DB0623E1
:10150000C35E1D0001930023AC4249DC002A00DCCD
:101510009BE0434668460380038899468CB2AFB28D
:1015200053460380008802AB19804B4601331B1BD6
:101530001BB2D90FCB185B10791C091A09B2CD0F59
:101540006D186D10191C1BB2AB4200DD291C0D1C5F
:1015500009B2914200DD151CADB22C19A4B202AB48
:101560009C8052465A80281883B200936B46002113
:101570005A5E934602AA5946D1800022310002A841
:10158000FFF7A0FF002813D02C1902AA9480009B1B
:101590009C466544D580310010002D4B98470300D0
:1015A000180005B03CBC90469946A246AB46F0BD3B
:1015B0007F1BBFB202AB5F806A469288DA8000224E
:1015C00031001800FFF77EFF00280AD02C1902AB6B
:1015D0009C807D1B5D80310018001D4B98470300E7
:1015E000DEE74B465C1BA4B202AB1C8042469A80ED
:1015F000002231001800FFF765FF00280AD0641BA5
:1016000002AB1C807D1B5D8031001800104B984799
:101610000300C5E702AB52465A805A46DA800022E0
:1016200031001800FFF74EFF01230028B8D0641BDB
:1016300002AB1C80009B9C46654402ABDD80310000
:101640001800034B98470300AAE70123A8E7C04608
:10165000A913010010B50023C45E0423CA5E002351
:10166000944216DC0423C45E0023CA5E0023944225
:101670000FDB0223C45E0623CA5E0023944208DC0B
:101680000623C45E0223CA5EE317D00F944243418F
:10169000DBB2180010BD0000F0B5C64600B582B040
:1016A00005000C0016000023C75E00228B5E0020A0
:1016B000BB4214DC0223EA5E0221635E9A420EDB27
:1016C0000423EA5E0421635E9A4208DC0622AB5ED4
:1016D0000621625ED80FD1179A424841C0B2002E4F
:1016E00003D102B004BC9046F0BD01A90F806B8805
:1016F0004B8032002000104B98470028F1D0042284
:10170000AB5E984601A90B80320020000A4B984737
:101710000028E6D001A90F80EB884B803200200022
:10172000054B98470028DCD001A943460B803200C6
:101730002000014B9847D4E7C514010030B5142AA6
:1017400027D89200B24CA25897468288013204886A
:10175000121B12B2D40FA41864108A8801320D88AB
:10176000521B12B2D50FAA185210A21A1A80C288A0
:1017700001324488121B12B2D40FA4186410CA8814
:1017800001324988521A12B2D10F8A185210A21A85
:101790005A801A88018852181A805A88418852182B
:1017A0005A8030BD00221A805A80F2E782880132C6
:1017B0000488121B12B2D40FA41864108A88013254
:1017C0000988521A12B2D10F8A185210A21A1A801E
:1017D00000225A80DDE782888C88121B0488121B45
:1017E000098852181A8000225A80D2E700221A80F3
:1017F000C288CC88121B4488121B498852185A8010
:10180000C7E7828801320488121B12B2D40FA418D1
:1018100064108A8801320D88521B12B2D50FAA18A3
:101820005210A21A1A80C288CC88121B4488121B3C
:10183000498852185A80ACE782888C88121B048829
:10184000121B0C8812191A80C288CC88121B44887B
:10185000121B498852185A809BE700221A80C288BE
:1018600001324488121B12B2D40FA4186410CA8823
:1018700001324988521A12B2D10F8A185210A21A94
:101880005A8086E782888C88121B0488121B0C8879
:1018900012191A80C28801324488121B12B2D40F66
:1018A000A4186410CA8801324988521A12B2D10FA2
:1018B0008A185210A21A5A806BE700221A80CA882E
:1018C0004988521AD2435A8063E7828801320488D9
:1018D000121B12B2D40FA41864108A8801320D882A
:1018E000521B12B2D50FAA185210A21A1A80CA8817
:1018F0004988521AD2435A804BE782888C88121B3F
:101900000488121B0C8812191A80CA884988521A36
:10191000D2435A803DE700221A80C28801324188B2
:10192000521A5A8035E7828801320488121B12B29B
:10193000D40FA41864108A8801320988521A12B28E
:10194000D10F8A185210A21A1A80C2880132418817
:10195000521A5A801DE782888C88121B0488121B39
:10196000098852181A80C28801324188521A5A8056
:101970000FE78A880988521AD2431A8000225A80B7
:1019800007E78A880C88121BD2431A80C28801326A
:101990004488121B12B2D40FA4186410CA880132F2
:1019A0004988521A12B2D10F8A185210A21A5A80BC
:1019B000EFE68A880C88121BD2431A80C288CC8832
:1019C000121B4488121B498852185A80E1E682880B
:1019D00001320188521A1A8000225A80D9E6828880
:1019E00001320488121B1A80C28801324488121BFB
:1019F00012B2D40FA4186410CA8801324988521A4E
:101A000012B2D10F8A185210A21A5A80C1E6C046EB
:101A100088A70200828801320488121B1A80C288BB
:101A2000CC88121B4488121B498852185A80B0E691
:101A300030B58DB2830702D001800230013A29040B
:101A40004919102A16D903001400196059609960C9
:101A5000D960196159619961D9612033103C102C0A
:101A6000F3D81100113909094C1C6401103A09011D
:101A7000521A0019002A04D005800230013A002AC7
:101A8000FAD130BD70B54A01521AFF24641A03041A
:101A9000DB0E63439D182B025B19DB015B191B01F5
:101AA000DB0E4505AD0E65438E01711A6D182902D6
:101AB0004919C9014919C900C006C00E60438218FE
:101AC00010028018C00180180001890E4901C00E63
:101AD000DB020843184370BD10B5FF23591A0304F5
:101AE000DB0E4B431A001B029B18DB019B181B01EA
:101AF000DB0E4205920E4A43140012021219D20163
:101B00001219D200C006C00E414308024018C0019D
:101B100040180001920E5201C00EDB021043184320
:101B200010BD421C4378002B04D109E00132137828
:101B3000002B05D03A2BF9D05C2BF7D02F2BF5D00A
:101B40001000704710B544210148024B984710BD62
:101B5000B84D0020D11D010070B504004068002878
:101B60000ED003690925002B08D02168984705008D
:101B70002068044B9847002323606360280070BDF1
:101B80000B25FBE7C923010070B584B01C1E01D0F2
:101B9000002323604568002D15D0AE690923002E6F
:101BA0000ED000230393006803AB009313000A00D8
:101BB00001002800B0470300002C01D0039A2260E6
:101BC000180004B070BD0B23FAE770B50A00446832
:101BD000002C09D0256A0923002D03D001682000BC
:101BE000A8470300180070BD0B23FBE770B5040085
:101BF00009480A4B984700280CD00378A34209D023
:101C0000054D074E01002800B047002802D0037898
